:1000000000800020BD0100000DA40000C5A3000079
:10001000C5A30000C5A30000C5A30000C5A3000040
:10002000C5A30000C5A30000C5A300000DA40000E7
:100030000DA40000C5A3000025C4000029C50000D0
:100040000DA400000DA400000DA400000DA40000EC
:100050000DA400000DA400000DA400000DA40000DC
:100060000DA400000DA400000DA400000DA40000CC
:100070000DA400000DA400000DA400000DA40000BC
:100080000DA400000DA400000DA400000DA40000AC
:100090000DA400000DA400000DA400000DA400009C
:1000A000018400000D8400000DA400000DA40000D8
:1000B0000DA400000DA400000DA400000DA400007C
:1000C0000DA400000DA400000DA400000DA400006C
:1000D0000DA400000DA400000DA400000DA400005C
:1000E0000DA400000DA400000DA400000DA400004C
:1000F0000DA400005DC800000DA4000089C9000027
:100100000DA4000099AD00000DA400000DA4000096
:100110000DA400000DA400000DA400000DA400001B
:100120000DA400000DA400000DA400000DA400000B
:100130000DA400000DA400000DA400000DA40000FB
:100140000DA400000DA400000DA400000DA40000EB
:1001500015C6000029C600003DC6000051C60000BB
:100160000DA40000B5B000000DA400000DA4000017
:100170000DA400000DA400000DA400000DA40000BB
:100180000DA400000DA400000DA400000DA40000AB
:100190000DA400000DA400000DA400000DA400009B
:1001A0000DA400000DA400000DA400000DA400008B
:1001B0000DA400000DA400000DA40000564B4CF24D
:1001C000205210B51A804DF628121A8000BF00BFC9
:1001D0000AF020F9514B4FF010621A60504A9A60B1
:1001E000504ADA60504A136813F4807304D14F49BF
:1001F0000B604FF4A85313604D4B1A78110703D5C9
:100200001A7842F008021A704A4B4B492A221A7097
:100210004A4A4B4B8B4204D252F8040F43F8040B6A
:10022000F8E7484B484900228B4202D243F8042B9E
:10023000FAE74649464A002352F8230041F82300D2
:1002400001336F2BF8D1434B434A802103F8011B44
:100250009342FBD1414B3D4A1A60414B8A221A70AE
:10026000A3F5805324225A70A0221A709A7992071B
:10027000FCD59A79D406FCD43A4A937903F00C035E
:10028000082B384BF9D103221A7140225A719A79FE
:100290009006FCD5334A9179324B4906FBD5324A58
:1002A000324911600221516020221A709A7902F0BD
:1002B0000C020C2AFAD12E4B2E4A1A602E4B2F4AD2
:1002C0001A6000225A60072243F8042C2C4AC3F813
:1002D0000C2D62B60AF028FC144B1B68DA0705D512
:1002E00028480AF0F5F9284B284A1A60284B1B7851
:1002F0005B0609D5244C254B22689A4204D121483B
:100300000AF0E6F9002323600DF0FEFD0AF088F8FC
:100310000CF016FAFEE700BF0E20054030800440C6
:10032000823F04000100002B10D0034014D0034092
:1003300002D0074000E007401C9BFF1F2C0E01006D
:100340004088FF1F1C9BFF1F08A3FF1F0082FF1F89
:100350000000000000E400E05FE400E008ED00E0E1
:100360000050064000400640448004400000030165
:1003700004800440C010050014E000E0FF76010096
:1003800000002020A9A4A65E1CE00340A5C3945A47
:1003900000F00740FFFFFFFFFFFFFFFFFFFFFFFF32
:1003A000FFFFFFFFFFFFFFFFFFFFFFFFFFFFFFFF5D
:1003B000FFFFFFFFFFFFFFFFFFFFFFFFFFFFFFFF4D
:1003C000FFFFFFFFFFFFFFFFFFFFFFFFFFFFFFFF3D
:1003D000FFFFFFFFFFFFFFFFFFFFFFFFFFFFFFFF2D
:1003E000FFFFFFFFFFFFFFFFFFFFFFFFFFFFFFFF1D
:1003F000FFFFFFFFFFFFFFFFFFFFFFFFFFFFFFFF0D
:10040000FFFFFFFFFFFFFFFFFFFFFFFFDEF9FFFF23
:1004100010B5054C237833B9044B13B10448AFF33E
:1004200000800123237010BD1C9BFF1F00000000F3
:10043000300E0100084B10B51BB108490848AFF356
:1004400000800848036803B910BD074B002BFBD0A0
:10045000BDE81040184700BF00000000209BFF1FB0
:10046000300E01001C9BFF1F0000000038B5044641
:10047000104621700A491D460DF028FB01464FF039
:100480007E500DF0D7FB07490DF020FBE560606062
:10049000256165610AF0D8FAE061204638BD00BFE9
:1004A000DB0FC9400024744938B50446104621705A
:1004B00009491D460DF00AFB01464FF07E500DF034
:1004C000B9FB06490DF002FBE560606025616561DE
:1004D0000AF0BAFAE06138BDDB0FC9400024744964
:1004E00038B503780446032B20D8DFE803F01A1848
:1004F0001002C16840690DF0DFF90D4905466068DA
:100500000DF098FB014628460DF094FB38BD0849D4
:1005100040680DF08FFBE1680DF0D8FA38BDC06877
:1005200038BDC16840690DF0C7F938BD002038BD3D
:100530000024744970B504460E460AF085FA054653
:10054000E069281A0DF06EFAE3682361E5616661DF
:10055000A061014660680DF06DFB0146A060104887
:100560000DF068FB0CF03EFE0CF0DEFA0DF050F9D9
:10057000054601464FF07E500DF09EF961690DF081
:10058000A5FA2169064628460DF0A0FA0146304634
:100590000DF094F9E0602046BDE87040FFF7A0BF81
:1005A000000080BF38B50E201C4C09F0E5FD218805
:1005B0001B4B884205461A881DDA0023511AB1F5F3
:1005C000805FAABF1B03C3EB03330131142093FBED
:1005D000F1F10AF08FF8134B1988F1B923889D4285
:1005E00010DAC3F57F630F33282091FBF3F1BDE8E8
:1005F00038400AF07FB89042D4BFC1EB0003C1EB92
:100600000203DBE740F6FF718D42D4BFC3EB050167
:10061000C3EB0101C1EB0131E3E738BDFA9BFF1FDA
:10062000A09DFF1F4C9DFF1F10B504460BF0D0FF8F
:10063000204610BD70B44C88A04220D9012301335C
:10064000DBB21CB2660031F8144084421D46F6D37A
:10065000A04211D005F10045013D965B31F815101F
:1006600032F81530401AF21A00FB02F0641A90FBBF
:10067000F4F4E01870BC7047905B70BC70470226C1
:100680000125E5E700280CDA064A434282FB0320F5
:10069000DA17C2EB600000EB4000A3EB8000C0F172
:1006A0000C007047ABAAAA2A2DE9F0470C2009F0EC
:1006B0002FFD0C200AF01CF9A04914200AF028F99B
:1006C0009F49A04807F0A2FB022103200AF0B6F9D7
:1006D000022104200AF0B2F9022105200AF0AEF945
:1006E000022106200AF0AAF901210A200AF0A6F93F
:1006F000012109200AF0A2F901210D200AF09EF93A
:10070000012128200AF09AF9012114200AF096F913
:10071000012116200AF092F9172001210AF08EF922
:1007200004200AF07DF9002833D005200AF078F97A
:100730000446002834D000242046834D287004F05D
:1007400039FF2D780DBB204606F048FB7F4B8049D2
:100750001B88804C098821707F4A804EA3F5AF71B9
:1007600040F23A7303FB01F382FB0312DB17A3EBA6
:100770006213323301210D2033600AF04BF95D2101
:10078000774807F0EDFE90B9FEE7BDE8F04707F0C7
:1007900051BA06200AF044F90028C6D10124CCE75A
:1007A00003200AF03DF9B0FA80F04009C5E75C216A
:1007B0006C4807F0D5FE00B9FEE75B216A4807F0F8
:1007C000CFFE00B9FEE729460D200AF023F9674A5B
:1007D00067481268DFF8E8A1DFF8A091654EDFF8FE
:1007E000E481654F00230121FFF75EFE0123C9F874
:1007F00000503560C8F800508AF8003004250F20FA
:100800000AF036FBD8F8003003440E20C8F8003058
:1008100009F0B2FCD9F800309AF800200344C9F876
:1008200000301520002A78D009F0A6FC336818445F
:10083000306005F0010080F0010003F0D1FD3B883D
:10084000002B14BF4B20FA200AF020F9013DD6D12D
:10085000D8F80030D9F80020484930683D88DFF8E2
:1008600068E1474F002BB8BF0333002AB8BF0332FB
:1008700092100A604349444A098812880028B8BF88
:1008800003309B10801030605E1A19443E60CEF831
:1008900000103E4F3E4E3F49C8F80030C2EB000EFC
:1008A0000244C7F800E032600B605DB94FF4FA70A3
:1008B00003F0A6FD03F090FD05F072F94FF4AF6070
:1008C0000AF0E4F8344B012504201D600AF0A8F872
:1008D00010B9324B20701D70314B1B881C2B23D05C
:1008E000304C04F1C805232009F046FC44F8040FFD
:1008F00001200AF0CBF8A542F5D12B4A2B4B1078FA
:10090000187006F075F903F063FD45F6BF522849EB
:100910002848BDE8F0470BF011BE11200AF0A8FAF4
:1009200033681844306084E7234B18880028D7D0F8
:10093000224BC0B2197806F0A3F8D1E7001B374666
:10094000801A06002490FF1F719BFF1F9C9DFF1FB4
:10095000109DFF1FC49BFF1FB5814E1BDC89FF1F2D
:10096000709BFF1FF89BFF1F9C9BFF1F3C89FF1F75
:10097000149DFF1F389BFF1F429DFF1F509BFF1FB1
:10098000689DFF1FEE89FF1F4489FF1F909BFF1F7B
:10099000C89BFF1FB09DFF1F709DFF1F5F9BFF1F28
:1009A000769DFF1F049CFF1FFC9CFF1FE19CFF1F07
:1009B000A5050000949DFF1FCC9BFF1F889BFF1F78
:1009C0005C9DFF1F649DFF1FE49CFF1FF0B40E8819
:1009D00086420DD203F10043013B31F813508542AA
:1009E00002D9F0BCFFF726BE32F81300F0BC704706
:1009F0001088F0BC704700BF094B1B880C2B09D82E
:100A0000084A80B252F8232028B143F6FE73984278
:100A100003D9108C7047108870470349FFF70ABE4E
:100A20006C9BFF1F24F000000CF10000374A38498E
:100A30001088384AF8B5384B12881B68834248DB67
:100A40009342A8BF134698420B60C8BF002342DD03
:100A5000101AB0F5804FAABF9B03C3EB833301305C
:100A600093FBF0F0FFF7C8FF2C4B2D4F1C883B6821
:100A7000C0F3C61505FB04F47F2CA8BF7F249D425C
:100A8000064608D0274B1B88002B38D1264B1B88E5
:100A9000002B30D13D60254D2B689E4205D0214B67
:100AA0001B885A1F032A1DD92E60214D2B689C429A
:100AB0000ED0204B188848B11A4B1F4A1B88D35CB4
:100AC000834203D0C0B2E1B205F0DAFF2C60F8BD7A
:100AD000F8BD034608609A42D4BFC0EB0203C0EBE6
:100AE0000303B5E7144AD05C2030C0B206F07F01A2
:100AF00005F0C6FFD8E7284606F036F8CAE70E4AE2
:100B00002946D05C05F0BCFFC0E700BFFA9BFF1F81
:100B1000409BFF1FA09DFF1F489DFF1F549BFF1F71
:100B2000A49BFF1F389DFF1FF29BFF1FA89DFF1F67
:100B3000F49BFF1F7A9DFF1FE089FF1F2DE9F04FF7
:100B4000012089B00AF094F9AF4B186000200AF038
:100B50008FF9AE4BAE4A1B8810600C2B00F03B8126
:100B6000AC4BAD4A19880093AC4B52F8214000229F
:100B70001A70AB4BAB4D1B88AB4A2E88013B32F948
:100B80001370002E5CD0A94BA94A1B88A949127882
:100B9000013B31F91380002A40F0DF8011200AF078
:100BA00067F9A54B0193D3F800A00646B24540F380
:100BB000DF80A24BDFF8A4921B88A14A012BD9F851
:100BC0000030B2F800B09F4A02922046C8EB0308FA
:100BD00000F09A820CF026FF029A52F82B100CF0CB
:100BE00075FF014600200CF067FE0DF035F9CAEBE9
:100BF0000802B045B8BFB0469042CAEB080880F280
:100C0000968200FB0888013298FBF2F08E4BDFF8E9
:100C100050820293D8F80030034403EBD3735B1087
:100C2000C8F800302B88012B12D1884BDFF834B282
:100C30000393874BDBF8005004934FF0000A47E022
:100C40007D4B0193DFF814927F4BDFF814820293FF
:100C50007E4B03931D460F200AF00AF92B68984239
:100C6000824641DA754A1288012A00F01D82744AD0
:100C700005931288734D049220460CF0D3FE049A1B
:100C8000DFF8E0B155F82210DBF800500CF01EFF41
:100C9000014600200CF010FE0DF0DEF8EF1B059B66
:100CA0005745A7EB0302B8BF5746FF1A9042BABF99
:100CB000013200FB0777474397FBF2F7D8F8002093
:100CC000634B0493BB1803EBD3735B10C8F800307D
:100CD000604B1B88013B032B00F2B082DFE813F06E
:100CE0006301A901C4008601594B04931B68984213
:100CF00040F3C281514A1288012A00F0A682504A6C
:100D0000079311884F4A0691204605920CF08AFEFF
:100D1000059A0699DFF84CB152F82110DBF8005023
:100D20000CF0D4FE0DF098F8079B2F445745A7EB25
:100D30000302A8BF5746FF1AD8F800309042BABF46
:100D400000FB07770132474397FBF2F73B4403EB85
:100D5000D3735B10C8F80030BAE7152009F00CFA1D
:100D6000354B0193D3F800A00646B2453FF721AFBB
:100D7000354B0293D3F800A0B24580F289812F4B06
:100D8000DFF8D8901B882E4A012BD9F80030B2F832
:100D900000B02C4A03922046984400F070820CF078
:100DA00041FE039A52F82B100CF090FE0DF054F80F
:100DB000B045CAEB0802A8BFB046CAEB080890428B
:100DC000B6BF00FB088800FB08F8013298FBF2F080
:100DD000DFF88C801EE7204B1B78002B3FF4C0AE61
:100DE0000C4B0D4A198800930C4B52F8210001223C
:100DF0001A700CF017FE4FF07C510CF067FE0DF0EE
:100E00002BF80446B5E600BF989BFF1F769DFF1F99
:100E1000BC9DFF1F9E9BFF1FA489FF1F469BFF1FBA
:100E2000EC89FF1FEA9CFF1F58F200003C8AFF1F5D
:100E30005C9DFF1FE8F00000909BFF1FE09BFF1FE1
:100E4000689BFF1F70F20000C89BFF1F689DFF1F7B
:100E5000E49CFF1F7889FF1F5E9BFF1F389BFF1FCD
:100E6000809DFF1F649DFF1F28460CF0DBFDB249EB
:100E70000CF02CFE054650460CF0D4FDAF490CF0AA
:100E800025FE014628460CF019FD0CF0E5FF05464D
:100E9000CBF80050D9F800000CF0C4FDA6490CF0C6
:100EA00015FE074630460CF0BDFDA4490CF00EFEC1
:100EB000014638460CF002FD0CF0CEFFC9F80000E8
:100EC0009F4AA04B168819889F4AA04B12681B881E
:100ED0009F4FC6EB050E3544039EC6F800E0461A48
:100EE000084404990D6001990E6002993E880860DB
:100EF0009A4280F289810025C3EB060E954974451C
:100F00000F6880F27681611C9F4205FB01F50EF1AE
:100F1000010E95FBFEF5C0F2BE81BE42A8BF3E4663
:100F2000F61A01FB06F494FBFEF49A4200F33681B4
:100F3000BB42C0F23381884C20680CF073FD8749B6
:100F40000CF0C4FD86490CF0B9FC0CF085FFA0F54F
:100F5000FF531C3B082B98BF4FF40050D8F80030CB
:100F6000184400282060C0F24281B0F5804F80F222
:100F700052817C4B1B781BB1B0F5005F40F0538170
:100F8000794D2B78002B40F05481784D20682B68E8
:100F9000714C984204D080B205F050FE23682B605B
:100FA00009B0BDE8F08F28460CF03CFD70490CF00C
:100FB0008DFD054650460CF035FD6E490CF086FD62
:100FC000014628460CF07AFC0CF046FF0546CBF8AB
:100FD0000050D9F800000CF025FD65490CF076FDB5
:100FE000074630460CF01EFD62495FE728460CF0CC
:100FF00019FD5A490CF06AFD054650460CF012FDE9
:101000005D490CF063FD014628460CF057FC0CF0DE
:1010100023FF0546CBF80050D9F800000CF002FD84
:101020004E490CF053FD074630460CF0FBFC52498C
:101030003CE728460CF0F6FC50490CF047FD05460D
:1010400050460CF0EFFC4E490CF040FD014628469E
:101050000CF034FC0CF000FF0546CBF80050D9F83A
:1010600000000CF0DFFC45490CF030FD074630462F
:101070000CF0D8FC424919E7D8F80030DFF810B17D
:1010800003EBD3735B10DBF80050C8F800301FE6A9
:10109000DFF80081DFF80091D8F8003003EBD3735C
:1010A0005B10C8F80030BDE5364A06931188364A11
:1010B000059120460492DFF8D8B00CF0B3FC049AF6
:1010C0000599DBF8005052F821100CF0FFFC0CF0F1
:1010D000C3FEEF1B069B5745A7EB0302B8BF57465D
:1010E000FF1AD8F800309042BABF013200FB0777F0
:1010F000474397FBF2F73B4403EBD373234A049235
:101100005B10C8F80030E3E50CF08CFC029A52F852
:101110002B100CF0DBFC0CF09FFECAEB0802B04574
:10112000B8BFB0468242CAEB08083FF76AAD00FB81
:1011300008F898FBF2F069E5CDCC4C3FCDCC4C3EA5
:10114000EE89FF1F4489FF1F989BFF1F469DFF1FCD
:10115000809BFF1FBC9DFF1FD889FF1F9A99193FD5
:10116000CDCC4C45779EFF1FF09BFF1F3889FF1F9A
:101170003333733FCDCC4C3DCDCCCC3E6666663F21
:10118000CDCCCC3D689BFF1F70F20000E49CFF1F9C
:10119000649DFF1F809DFF1F389BFF1F009B1B88C6
:1011A000002B3FF4C8AE2B1B002BB8BF5B42092BB2
:1011B00047DD05F500500130001B0CF033FC3B49C6
:1011C0003B4C0CF083FC054620680CF02BFC3949A5
:1011D0000CF07CFC014628460CF070FB0CF03CFE49
:1011E000D8F80030184400282060BFF6BEAE0022B8
:1011F00013E09F4205FB04F5B8BF002195FBFEF507
:101200004BDA91FBFEF490E6B242D4BFC3EB020589
:10121000C3EB060570E643F6FF72274B22601B788E
:10122000002B3FF4ADAE03F0D7F8244B01221A7027
:10123000ABE603F0CDF800232B70A6E6D9F800004A
:101240003EE64FF400501A4C88E61D491D4A0693AD
:1012500020460D8805920CF0E5FB059ADFF868B092
:1012600052F82510DBF800500CF030FC014600204D
:101270000CF022FB0CF0F0FD2F44069B56E50CF021
:10128000D1FB039A52F82B100CF020FC01460020F1
:101290000CF012FB8AE51E4642E6B742D4BFC3EB10
:1012A0000701C3EB060104FB01F1AAE7CDCCCC3E5C
:1012B000D889FF1F9A99193F779EFF1FF09BFF1F48
:1012C000689BFF1F70F20000649DFF1F38B5114C32
:1012D0002320257808F050FF0F4A42F82500131FFD
:1012E00002F1C400002253F8041F83420A44FAD1D9
:1012F00023780A4907480A4C0133DBB2322B81FBC1
:10130000025108BF0023D217C2EB211203702260E2
:1013100038BD00BF569BFF1F089CFF1F1F85EB5168
:10132000609DFF1F2DE9F0479F4CA04D206882B0C3
:101330000CF078FB9E490CF0C9FB0646102009F022
:1013400097FD0CF06FFB9B490CF0C0FB31460CF095
:10135000B5FA0CF081FD2B882060192B00F0CA80B3
:101360001A2B00F0F5801E2B00F0FB8001252E4685
:10137000914A1188002900F09180904B904A1B8877
:101380001288834240F3DD800020D31A8B42C6BF0F
:1013900001FB00000133484390FBF3F3894A1360DB
:1013A000894F388848B9894B1B8833B9884A1178E6
:1013B00001B1137002B0BDE8F087DFF80082216848
:1013C000B8F80030784A8B426EDCDFF804E29EF811
:1013D0000090B9F1000F2FD14FF0010C04288EF8C6
:1013E00000C029D1002D40F07181784B1888002869
:1013F000E0D0002EDED02368B8F80040704AA34247
:10140000128880F23E810023141B7E2C714DD5BFC3
:10141000C3EB8313C3EBC3135B00013493FBF4F4FE
:101420002B680134A34203D0C0B2E1B205F028FB1F
:101430002C6002B0BDE8F087012800F0D5800228BA
:1014400000F0A9800328D0D1634B1B88092BCCD096
:10145000002DCAD02368B8F80050594AAB42128810
:1014600080F25C810023551B7E2DDFF874A1D5BF6F
:10147000C3EB8313C3EBC3135B00013593FBF5F59B
:10148000DAF800300135AB4203D0E9B24A2005F06A
:10149000F7FACAF80050A8E70D460E461E2B7FF457
:1014A0007FAF00214D4F64E0494B1A78002A81D06C
:1014B000002401281C7062D0022840F0E980002D31
:1014C00063D0474D2B68002B5FD00420214605F0E8
:1014D000D7FA3E4B2C60188800283FF46BAF002EE3
:1014E0003FF468AFC0B2002105F0CAFA394B0022C0
:1014F0001A605FE7394F3B4E3A7872B13349098839
:1015000059B196F800E0964542D0C8B27F2105F067
:10151000B7FA3A782B8832700AE03178914237D0A6
:101520002A4B0021187805F0ABFA3A782B883270F4
:10153000214A11880029AFD000251E2B2E4618D035
:101540001BE08242D4BFC3EB0200C3EB00001CE7E8
:10155000224F3A78002A0BBF0125002500260126DC
:1015600006E71E4F144B3D781988B5FA85F56D09CD
:1015700000263B78002B3FF411AF2068FDE625B133
:10158000174D2B68002B40F09A80104B1888A3E76A
:1015900000252E46ECE6002D3FF427AFDFF840A0F3
:1015A000074ADAF800304AE08C9BFF1F769DFF1F48
:1015B0009A99193FCDCCCC3EA49DFF1FF49CFF1FF0
:1015C000EE9CFF1F009CFF1F969BFF1F889DFF1F27
:1015D0007D9DFF1F749BFF1F389DFF1F5E9BFF1F9C
:1015E000049CFF1F5B9BFF1F002D3FF4FEAE534A80
:1015F00010888842D4BFC3EB0009C3EB0109C31AAA
:101600007E2B40F38280C9EBC91103F1010991FBE4
:10161000F9F909F10109DFF82CA1DAF800304B459E
:1016200006D05FFA89F10120019205F029FA019AAA
:101630003888CAF8009002287FF404AF4B4621682E
:10164000B8F800901088494558DA0022C9EB000923
:10165000B9F17E0FD3BFC2EB8212C2EBC21209F105
:101660000109520092FBF9F909F10109994504D0E9
:101670005FFA89F1042005F003FA3888CAF800906F
:10168000E0E69342D4BFC4EB0303C4EB0203BBE622
:10169000032828D12A4B1B88092B3FF476AF002D55
:1016A0003FF473AF274D2B68002B3FF46EAF4A20F9
:1016B000214605F0E5F9244B2C6018880CE72146FB
:1016C00005F0DEF9204B2C60188805E740207F21CB
:1016D000019205F0D5F93888019A012825D0022811
:1016E0007FF4B0AE5AE704287FF44FAF002D3FF4EB
:1016F0004CAF2146402005F0C3F946E78142D4BFF4
:10170000C9EB0102C9EB0002A0E7C9EB89194FEA56
:10171000490999FBF3F909F101097CE79342D4BF28
:10172000C5EB0303C5EB02039DE61168B8F8003072
:10173000024A99421088FFF662AF5AE7EE9CFF1FFB
:10174000389DFF1F049CFF1F889DFF1F08B50F4B8E
:101750001B88022B0FD0032B12D0042B03D00C4B71
:1017600001221A7008BD7F21092005F089F9084B74
:1017700001221A7008BD7F21412005F081F9EEE7B2
:101780004021092005F07CF9E9E700BFFE9BFF1F1F
:10179000B79BFF1F38B51C4B1B881D2B26D01B4B3E
:1017A0001B88012B25D01A4A1A4B14881B681A4A29
:1017B000A342128818DB9342D4BFC4EB0303C4EBEB
:1017C0000203141B7F2CC6BFDB010134C3EBC31320
:1017D00093FBF4F4114D2B689C4203D0E1B2052039
:1017E00005F04EF92C6038BD0023EAE70C4B1C884D
:1017F000F0E70C4B0C4A0D491B6812680C689B1AE9
:101800001C1B84F30704E5E7769DFF1FEA9CFF1F7E
:10181000B29BFF1F4C9BFF1F749DFF1F909DFF1FDE
:10182000889BFF1FB09DFF1F4089FF1FF89CFF1F73
:1018300010B50F4C23685BB90E4B1B88022B11D0DF
:10184000033B012B09D90C4A00231370236010BD00
:101850000021052005F014F9EEE70021092005F02C
:101860000FF9F0E70021412005F00AF9EBE700BF8E
:10187000909DFF1FFE9BFF1FB79BFF1F08B5274BC7
:101880001B78ABB1152008F077FC254A254B128850
:1018900018601D2A15D0244A1288EAB1012A25D0E1
:1018A000224B1B78002B34D0BDE80840FFF7C0BFA7
:1018B000112009F0DDFA1A4A1A4B128818601D2A05
:1018C000E9D11B4B1B78002BEAD0184B1B780BB3CC
:1018D000BDE80840FFF75EBF164A1288002ADFD035
:1018E000154A1B6812889A42DADCEEE70F2009F0ED
:1018F000BFFA104B114A1B88106033B1104B114ACC
:101900001B6812689B1A9842DFDD084B1B78002B7E
:10191000CAD108BDFFF71AFFDAE700BF5C9DFF1FC1
:10192000769DFF1F4C9BFF1FEA9CFF1FB79BFF1F6D
:101930005E9BFF1FFE9BFF1FB29BFF1FF89CFF1FBC
:10194000B09DFF1F4089FF1F2DE9F04FDFF818B34E
:101950009BF80060012E93B000F02182C0F0F3816B
:10196000022E00F0BF809948994B9A4DDFF8ECE2C7
:10197000994A9A499A4F9B4C009400789A4C1B784C
:101980002D789EF800E01278097897F800A0DFF82B
:10199000DCC2DFF8DC82DFF8DC920194012E934C8C
:1019A00094BF0136002622708BF80060904C914E57
:1019B00023703070904C914E21703570904C914E48
:1019C00084F800A03270BEF1000F40F0F1808E4C20
:1019D00024880D2C00F09181DFF888E2002426464F
:1019E0008EF80040A3462BB1874B1C88002C40F09A
:1019F00091812346854C248803EB0B0E002C40F08C
:101A00003B81834B834C1B7899F8009024780133F9
:101A1000A3EB4903002C40F08081019C2478C4EBA7
:101A2000030B002C40F039820023DFF82C927A4C13
:101A300099F800902478C3EB0B03A3EB49032B44E4
:101A4000181A002C00F07D81B5FA85F56D099CF817
:101A500000300544ED1A002B00F0718119F10000EF
:101A600018BF0120009C98F8003027786B4C281A8A
:101A7000C31AA3EB47030B449B1A2178684C694AAD
:101A80002568A3EB4A034FF00C0A1AFB01331360DD
:101A9000654A66481288664900680988C2EBC20236
:101AA00002446448194450F822200C398E44724490
:101AB0000EB161490B60AA4200F01B815F4B604888
:101AC00019680591059901601B6806935D48069B9E
:101AD000008822605B1A834284BF5B4B1A6013B09C
:101AE000BDE8F08F594F06AE0025E9B2584806F020
:101AF000FBFC57F8043B0135C01A0C2D46F8040BCB
:101B0000F3D1544B079FB3F800C00E9B0D9E0F9D61
:101B10001098354C01946345ACBF4FF0000E4FF068
:101B2000010EBC45D4BF00270127B445D4BF002611
:101B30000126AC45D4BF4FF000084FF00108119BBF
:101B400084F800808445444C4449324ADFF82491AB
:101B50001770D4BF4FF0000A4FF0010A9C45099B53
:101B600084F800A01B4C81F800E0D4BF00250125BB
:101B70009C450A9B2570154C154F174A89F8006043
:101B8000D4BF00200120164E144920709C45D4BFBC
:101B900000230123134C96F800A03B7012780978BB
:101BA0009BF80060DFF8C4C0DFF8C4800094F5E65D
:101BB0002B4E2C4CB6F800B00126BBF1180F267046
:101BC00040F2B9804FF0000B0DE700BFB59BFF1F3F
:101BD000B69BFF1FB49BFF1F359DFF1F349DFF1F4A
:101BE000369DFF1F799DFF1F849DFF1FC19DFF1F15
:101BF000C39DFF1FC29DFF1FC59DFF1FC49DFF1FEB
:101C00007C9DFF1FC69DFF1FC89DFF1F449BFF1F9C
:101C1000F089FF1FB49DFF1F9E9DFF1FE99CFF1FC2
:101C2000AC9BFF1F3C9DFF1F6C9DFF1F009CFF1F77
:101C3000589BFF1F98F20000849BFF1F949EFF1F7C
:101C4000D09BFF1F869DFF1FB89DFF1F4889FF1F68
:101C5000F89BFF1F9C9DFF1F8C9DFF1FC79DFF1FB3
:101C6000769DFF1F5E9BFF1FE09CFF1FC09DFF1F17
:101C7000789DFF1F8B9DFF1F012C00F07981022CA6
:101C800000F0DA81032C9E4B00F00D811D78009B43
:101C90009CF800B0197899F800209A4B019C98F8AC
:101CA000008093F800C02778A5EB4B05A1EB8104D9
:101CB000C2EB8273C8EB05012144C2EB83028B188F
:101CC00003EB4C0303EB8A0A27B18F4B1B78002BE5
:101CD00040F04E8201238D4A8D4C12788D49256843
:101CE000C2F10602534402EB420203EB82030B6093
:101CF000CEE68949894B0968E6E6002B3FF46CAED5
:101D0000874E884FB6F800B00126BBF1180F3E7021
:101D100011D9F346A4F10D036CE6019C2478B9F1C6
:101D2000000F40F09E80013BC4EB030B002C3FF4FE
:101D30007BAE4B4679E6ABF10C0B012653E6184619
:101D400090E6254683E6784F06AE0025E9B277484F
:101D500006F0CAFB57F8043B0135C01A062D46F8B9
:101D6000040BF3D1724A0B991288684B0020914200
:101D70001870C0F283800A998A4240F3DA816D4874
:101D80006D4A6E4990F800A012780978DFF8D4C146
:101D9000DFF8D48105201870694B009351E0694F3A
:101DA00006AE0025E9B2684806F09EFB57F8043BF2
:101DB0000135C01A0C2D46F8040BF3D15C4B099C7D
:101DC00018880A9F4F4B0E9ADFF89C81DFF894C168
:101DD00006A962C98442ACBF4FF000094FF0010967
:101DE000B842D4BF00270127B042D4BF0026012645
:101DF00083F80090A842524B0093D4BF00250125E0
:101E000088421D70D4BF002101214B4B0D9C88F8E6
:101E100000609042D4BF002201221A70109B474EEE
:101E2000444D8CF80070A042D4BF4FF0000A4FF030
:101E3000010A9842317085F800A019DC002343485C
:101E40000370434E4348444B444D454C96F800E0E4
:101E500000781B782D789BF80060DFF810910194D2
:101E60009CE5002C40F07B8103F1FF3B2346DCE541
:101E70000F9B9842D4BF00230123E0E72E4A2F494D
:101E80002C481D702E4B1278097890F800A0DFF8CE
:101E9000D4C0DFF8D4800093D3E7B9F1000F3FF44A
:101EA000C3AD0123C1E51978009B9CF800C01A78E6
:101EB00098F8008099F80030124D019C2D78247814
:101EC000A1EB4C01C8EB0108A2EB8202C3EB8371CA
:101ED0004244C3EB8103134403EB450303EB8A0A3B
:101EE000002C40F049810120084B0A4A1B78084C1D
:101EF00082440C2111FB03A313602568C8E500BFD1
:101F0000F089FF1F9E9DFF1F8C9DFF1FE99CFF1FF7
:101F1000AC9BFF1F3C9DFF1FD09BFF1F949EFF1F8C
:101F2000769DFF1F5E9BFF1F248AFF1F709BFF1F74
:101F30009C9DFF1F369DFF1F359DFF1F349DFF1F7A
:101F4000799DFF1FF489FF1F9C9BFF1F829BFF1F32
:101F5000C79DFF1FB59BFF1FB69BFF1FB49BFF1FB5
:101F6000849DFF1FC09DFF1F789DFF1F8B9DFF1F3E
:101F7000AD4BDFF8E4B21F7899F800309BF8009081
:101F8000029307F1010BABEB43031F46B9F1000FBE
:101F900040F0B380019C94F800B0C9EB0703CBEB91
:101FA00003030193BBF1000F40F0BB805B469F4CE5
:101FB000DFF88C92247803942746019C99F80090CE
:101FC000E31AA3EB49032B44181A002F00F0A48056
:101FD000B5FA85F464099CF800300444E41A1BB196
:101FE00019F1000318BF0123009898F800500078F9
:101FF000E31A5B1BA3EB40030B449B1A029AA3EB6F
:102000004A03002A40F09280BBF1000F40F0C280EA
:102010005B4400287ED1BAF1000F0CBF00226FF0A4
:102020000902834883490078834C1A440C2313FB2C
:1020300000230B6025682BE5019C804B24780194DC
:10204000009CDFF814B227787D4C98F80080247843
:1020500000949CF800C099F800909BF800B09DF89F
:10206000044083F806805A72DFF8F0819DF8002062
:1020700083F805C0DA709C7083F800901D71DF71E1
:10208000197283F80AA083F801B04FF0000C012206
:1020900000236A4F194645464C4607E0022A09D0FC
:1020A0000B2B0BD017F8014F15F8012F944203F1B9
:1020B0000103F3D101310B2BC9B2F3D10A2907D89F
:1020C0000CF1010CBCF1110F4CD018F80B2FDFE70D
:1020D000554A5C4B1478554953F82C20544B0978D9
:1020E0001B78544D01342244101A08440C22524CDF
:1020F00012FB03032B602568CAE4029B002B44D02B
:10210000019B93F800B0BBF1000F07D17B1E019338
:102110005B464CE7002284E7039C5CE7CBEB0703BC
:102120000193029B003318BF012340E74FF0000BDF
:102130006EE709998A4235DC08998A4242DD4248B5
:10214000424A434990F800A012780978DFF810C19C
:10215000DFF81081032018703E4B009371E6C4EB4A
:10216000030B9EE6344C334B25681D602B468FE4F1
:10217000031C18BF0123AEE5314B1B78002B3FF445
:10218000B2AE003018BF0120AEE6019BA14693F825
:1021900000B002E7B9F1000F0CBF4FF0000B4FF099
:1021A000090B35E72848294A294990F800A01278F8
:1021B0000978DFF8ACC0DFF8AC8004201870254B3C
:1021C00000933EE607998A420FDD1F481F4A2049C7
:1021D00090F800A012780978DFF884C0DFF88480D6
:1021E000022018701B4B00932BE606998A42174A6F
:1021F00017490DDD1448127890F800A00978DFF82F
:1022000060C0DFF8608001201870124B009318E660
:102210000D4B127893F800A00E4B0978DFF840C000
:10222000DFF8408000930CE6F089FF1F9E9DFF1FA2
:10223000E99CFF1F3C9DFF1FAC9BFF1FD49BFF1F12
:102240008C9DFF1FBCEF0000369DFF1F359DFF1FBB
:10225000349DFF1F799DFF1FB49DFF1F30F10000CB
:10226000C09DFF1F789DFF1F2DE9F04F2E4B1B785F
:102270008BB0002B53D10E2007F07EFF0BF0D2FB6A
:1022800001462A482A4C2B4DFEF754F92748FEF701
:1022900027F90BF0E1FD80F30C002060FFF754FB01
:1022A0002E68012E5AD0022E00F08782032E00F0F5
:1022B0009783214C2368214A214E0993099B177863
:1022C0003068204C07210122181A11FB0722904286
:1022D000236000F26D821C4E32689A1A0D2A00F2B9
:1022E00060821A4E32689A1A132A00F25582184EEA
:1022F00032689A1A252A00F23C82164D2A689B1AE7
:10230000502B00F2F581144B1B88012B00F00D823D
:1023100004F04AFC04F078FA0BB0BDE8F08F05F049
:1023200015FB0BB0BDE8F08F719BFF1F149DFF1FC5
:10233000489DFF1F709DFF1F949EFF1FE29CFF1F83
:10234000F09CFF1F0C9DFF1FE89BFF1FBC9BFF1F06
:10235000C09BFF1F009DFF1F4C9DFF1FDFF80083E8
:102360009A4AB8F800001378834204D0C3B21846E2
:10237000137004F055FBDFF8E492954AB9F8003089
:102380001178994204D0934F3978002940F098870A
:10239000914A23681288914C9A42C0F2EE80904A8A
:1023A0001278002A40F0E980DFF8B8A2BAF80030CD
:1023B00023B98C4B1B88002B00F042858A4A8B4B3B
:1023C00011881B888A4A0B4412685B109342894A21
:1023D000126880F2B78400219342B4BF01230B46F8
:1023E00004910093ACBF4FF0010B8B4605910E207A
:1023F00007F0C2FE804B814A1B68176803930133C4
:10240000A7F25232002B8446029240F36A87802B57
:10241000A8BF80237A4A7B4912780191002A00F0F4
:10242000B6800978914200F0B280B9F80010DFF868
:102430002CE2994201F061816649AEF80030724B9E
:102440004FF0010E81F800E01978DFF81CE2019BE3
:102450008EF800101A70009B002B00F00781BAF86C
:102460000030002B00F00281684B1B685A1C002AC8
:1024700040F33B87802A00F33787654E65496648FD
:102480003688098800683144B0EB610FC1F20982D7
:10249000A3F148020F2A02D8473BA8F800300E20CB
:1024A00007F06AFE6FF454731F44874202DC5B4BF3
:1024B00000221A705A4B1B88002B00F03B84594BAA
:1024C000594A1B781178994240D0002B3ED0574989
:1024D0000E78002E00F0EE87554991F800C0BCF14F
:1024E000000F40F0E587534F0097534F5348029732
:1024F000504F007887F800C04F4F4FF0010E87F81B
:1025000000C081F800E0002841F089814C49097839
:10251000002901F04A804B4903910E4609780029B1
:1025200041F040804848444F0078397001210297BB
:10253000317058B13F483E49009000200870009922
:10254000029F0870039901263E70087013703F4B7C
:102550001B88A3F11B02012A40F28D861D2B7FF4FC
:10256000A9AE394F3B78002B41F00C81384E3378BF
:10257000002B40F0958433709CE62168354A069123
:1025800006983549106002220B602A600CE71E494C
:10259000DFF8D4E0097800293FF459AF9EF8000035
:1025A00081423FF454AF03984B2841F352801833D3
:1025B000802BB9F80000A8BF802398423FF447AFB2
:1025C0002648038003480123037040E7E19CFF1F76
:1025D000C49BFF1F5F9BFF1FFA9BFF1F949EFF1F63
:1025E0006A9BFF1FEE9BFF1F809BFF1F469DFF1FE7
:1025F000989BFF1FBC9DFF1F849BFF1F509BFF1FCD
:10260000AC9DFF1FA89BFF1FAD9DFF1F3C9DFF1FA3
:10261000F49CFF1FEE9CFF1F8C9BFF1FE89CFF1F7D
:102620004E9DFF1F829BFF1F5A9BFF1FC49DFF1FD4
:10263000449DFF1F8A9DFF1FFC9BFF1FC59DFF1F21
:10264000C19DFF1F3C9BFF1F5E9BFF1F769DFF1FD1
:102650005B9BFF1FB89BFF1F089DFF1F109DFF1F67
:10266000FC9CFF1FB09BFF1FA99BFF1F029B9C456B
:10267000BFF615AF8E4B1B88002B3FF410AFBBF19C
:10268000000F7FF4F1AE8B4B1B881BB1059B002B19
:102690007FF4EAAE049B002B3FF401AF864B1A781F
:1026A000002A7FF4FCAEDFF8888298F800600122EF
:1026B0001A70002E40F09183804B1B78002B01F0A4
:1026C00032817F4B1B78002B01F043817D4B1B78BF
:1026D000002B7FF4E4AE7C4B1B78002B3FF4DFAE85
:1026E000B9F8003079490A3BA9F800300A70D6E6FB
:1026F00002F0A8FF764B1B7873B9764B1B785BB959
:10270000754B1B7843B9754B1B782BB9744B1B78F1
:1027100013B901F05DFE01E001F066FE23682B6055
:10272000704B1B88012B7FF4F3AD6F4A6F4B116820
:102730006F481A78A1F118032A2101FB03F1016007
:10274000002A00F0E1826B4A1368994200F37C830F
:1027500080F2868368480068D0F17F0048BF03306C
:10276000801001301B1A994200F37A8313601946D6
:10277000CCE2FEF7ABFD614B1B881B3B9BB2022BEF
:1027800005D85F4B1B7813B12B68012B01D001F0EA
:1027900049FE23683360B0E5FFF770F823683360C3
:1027A000A5E5FEF7CBF9FEF7BDFD2368336098E59C
:1027B000FEF73CF9236833608DE5524A266812889B
:1027C000B24204DB464B1B78002B00F064834E4C76
:1027D0004E48236807934E4B079900681B88091AD7
:1027E000994200F2AB80002B00F0A880494B198879
:1027F00000293FF45FAD484B48481B680088B3424E
:10280000B8BF33469A4241F34580454B1A60DFF822
:10281000248188F80010344FFEF708F938687F28C3
:1028200040F342863F4B7F3883FB0032C317C3EB34
:10283000620303EB4303A0EB830073303A4B019335
:102840001B883860002B40F04A87234B00931B788D
:10285000002B00F07384354E3378002B00F06E842B
:10286000DFF8D490DFF8BCA04FF0000B0CE003F1D0
:102870007300C0B298F8001004F02AF933780BF115
:10288000010B5B4540F35A843B6859F8040F184428
:10289000A0F17F038AFB0321DA17C2EB610202EB8E
:1028A00042027F28A3EB8203E1DCFDF7EBFEE0E7C9
:1028B000EE9BFF1F049DFF1FE89CFF1FC19DFF1F94
:1028C000C29DFF1FC39DFF1FC49DFF1F5F9BFF1F76
:1028D000FC9BFF1F449DFF1F8A9DFF1F3C9BFF1F0A
:1028E0006A9BFF1F4C9DFF1FB89DFF1FB79BFF1FDB
:1028F000E49BFF1F649BFF1F909DFF1F769DFF1FA2
:102900005E9BFF1FFA9BFF1F949EFF1FB89BFF1F3C
:10291000EC9BFF1F5C9BFF1F089DFF1FA09DFF1FDF
:10292000409BFF1FABAAAA2A949BFF1FA089FF1FF1
:10293000E99CFF1FE29BFF1F7889FF1F554B5649FB
:102940001B6808885549B342B8BF33469A4200F322
:102950008982534E09888342A8BF03463360002909
:102960007FF455AF9A42C8BF0B4640F38282801A6B
:10297000B0F5804FAABF9B03C3EB8333013093FBB9
:10298000F0F0FEF739F8C0F3C6100BF04BF8454BEA
:10299000064618880BF046F84349074630460BF0C8
:1029A00095F8014638460BF091F831460AF086FF5B
:1029B0004FF07E5106460BF027FA002840F05F8763
:1029C0003A4930460BF03EFA002840F01C8730466A
:1029D0000BF068FAC0B2DFF8F48088F800001AE75C
:1029E000334B26681988B14274DD324B1B78002BBB
:1029F00070D1DFF8DC9099F800007F2840F3BE86A4
:102A0000A3F155337F3803F1004383FB0032C31732
:102A1000C3EB620303EB4303A0EB83007330264B4D
:102A200001931B88C0B289F80000002B40F0078793
:102A3000224B00931B78002B00F06785204E3378E3
:102A4000002B00F062851F4FDFF87C804FF0000AFA
:102A50000AE003F17300C0B204F062F833780AF1BF
:102A6000010A534540F3518557F8043F99F8000097
:102A70001844A0F17F0388FB0321DA17C2EB61023F
:102A800002EB42027F28A3EB8203E2DCFDF7FAFDB2
:102A9000E1E700BF089DFF1FA09DFF1F5C9BFF1F7C
:102AA000409BFF1F489BFF1FCDCCCC3D0000FE424A
:102AB000FA9BFF1F6A9BFF1F949BFF1F8A9DFF1FAE
:102AC000A089FF1F7889FF1FABAAAA2AE29BFF1FDC
:102AD000409DFF1FA24F38687F2840F3D181A14B52
:102AE0007F3883FB0032C317C3EB620303EB43035E
:102AF000A0EB83007330DFF8B49299F800A0824510
:102B000000F02882984B1B88002B43D1974A9848A5
:102B100012680088914205DC8242D4BFC1EB0203F7
:102B2000C1EB0003411AB1F5804FA6BF9B030131F1
:102B3000C3EB833393FBF1F0FDF75EFFC0F3C610E8
:102B40000AF070FF8B4B064618880AF06BFF8A4923
:102B5000804630460AF0BAFF014640460AF0B6FF0A
:102B600031460AF0ABFE4FF07E5106460BF04CF9B1
:102B7000002840F06186814930460BF063F9002857
:102B800040F0308630460BF08DF9C0B2DFF820827D
:102B900088F80000BAF17F0F40F381847148AAF1F0
:102BA0007F0A80FB0A304FEAEA73C3EB600000EB58
:102BB0004000AAEB80007330714B00931B78C0B2C9
:102BC00089F80000002B40F0E1836E4B03931B78E3
:102BD000002B40F0AE856C4B02931B78002B40F02D
:102BE00051866A4B0193029B1B78002B3AD0684BAD
:102BF0001B88182B17D099F800201344A3F1180054
:102C00007F2840F3F285574A973B82FB0321DA176E
:102C1000C2EB610202EB4202A3EB820303F17300F9
:102C2000C0B203F07DFF5B4A5B4B127833F8123081
:102C3000182B17D099F800201344A3F118007F280F
:102C400040F3DD85474A973B82FB0321DA17C2EB4D
:102C5000610202EB4202A3EB820303F17300C0B2F4
:102C600003F05EFF009B1B78002B00F0AE84019BFD
:102C7000464E1988002900F0558538687F2840F3B2
:102C80005083384B7F3883FB0032C317C3EB62039A
:102C900003EB4303A0EB830073303860002940F05E
:102CA000E984009B1B78002B00F05F813B4E33785A
:102CB000002B00F05A81DFF8FCA0DFF8F4804FF021
:102CC000000B0CE003F17300C0B298F8001003F0A1
:102CD000FFFE33780BF1010B5B4540F346813B6807
:102CE0005AF8040F1F4A1844A0F17F0382FB032106
:102CF000DA17C2EB610202EB42027F28A3EB8203E8
:102D0000E0DCFDF7BFFCDFE7254B1960254B1B68B6
:102D1000A92202FB03F3002BBCBF03F57F533F3313
:102D20009B13543B194481F30C01282007F0E2FC6B
:102D3000FFF7EEBA144E1C481149124A3370037063
:102D40000B7003E493424FF0000B80F29C80012350
:102D5000CDF800B0CDF814B00493FFF748BB00BF26
:102D6000B89DFF1FABAAAA2A5C9BFF1F409BFF1FB9
:102D7000A09DFF1F489BFF1FCDCCCC3D0000FE4215
:102D80008A9DFF1F3C9BFF1FFC9BFF1F949BFF1F07
:102D9000789BFF1FA29BFF1F549DFF1FA089FF1F51
:102DA000649BFF1FD889FF1F449DFF1F409DFF1F8D
:102DB000E29BFF1F7889FF1F924B1B78002B7FF44B
:102DC0006EAB039B904A243B83F34703D9B25B204D
:102DD000136003F055FE98F80060032E30D1DFF841
:102DE000808298F80030002B40F03686874F3B7881
:102DF000002B40F02486834E3378002B40F012865F
:102E0000834B1B78002B40F00086824A1380824B54
:102E10001B78002B40F0EC85804B7F221A8098F8BD
:102E200000306BB93B785BB933784BB97C4A7F2172
:102E30000720138003F024FE7F210B2003F020FEE7
:102E4000784B1F68FFF72BBB77480068D0F17F00F5
:102E500048BF033003EBA00301339942BFF686ACB1
:102E6000116053E7714B09881A6000297FF4CFACD9
:102E700013469842D4BFC2EB0003C2EB030376E5CE
:102E8000FDF700FC37E60123CDF810B0CDF800B017
:102E90000593FFF7ACBA01232B60654CFFF70ABA24
:102EA000644B6A20198803F06FFF3B783370FFF79B
:102EB00001BA614B1B78002B3AD0604B1B88182B52
:102EC00017D099F800201344A3F118007F2840F38D
:102ED000ED845B4A973B82FB0321DA17C2EB610268
:102EE00002EB4202A3EB820303F17300C0B203F0D2
:102EF00017FE544A544B127833F81230182B17D05F
:102F000099F800201344A3F118007F2840F3D284DD
:102F10004B4A973B82FB0321DA17C2EB610202EBBB
:102F20004202A3EB820303F17300C0B203F0F8FD89
:102F3000019B1B88002B00F08C84444B1B78002BDA
:102F400040F08184424B394A1988266800200123C9
:102F500010602B60B142364CBFF6ACA922683D4BE5
:102F60000892089A1A60FFF7A5B9039B1B78002BFB
:102F70007AD03B68A3F10C007F2840F3F2833048FD
:102F80008B3B80FB0320DA17C2EB600000EB4000B4
:102F9000A3EB800303F17300DFF8C080C0B298F8A0
:102FA000001003F095FD009B1B78002B5CD02A4E8F
:102FB0003378002B58D0DFF8ACA04FF0000B0BE0BB
:102FC00003F17300C0B298F8001003F081FD33786C
:102FD0000BF1010B5B4547DD3B685AF8040F184ABB
:102FE0001844A0F18B0382FB0321DA17C2EB6102C4
:102FF0000C3802EB42027F28A3EB8203E0DCFDF7F2
:1030000041FBDFE7C49DFF1F7C9BFF1FC39DFF1F8C
:10301000C29DFF1FF29BFF1FC59DFF1F5C9BFF1FF3
:10302000389DFF1F509BFF1F909DFF1F409BFF1F60
:10303000949EFF1F889BFF1FFC9BFF1F789BFF1F19
:10304000ABAAAA2AA29BFF1F549DFF1F449DFF1FEE
:10305000FA9BFF1F549EFF1FA089FF1FE29BFF1FCB
:10306000C19DFF1F7889FF1F029B1B78002B3AD060
:10307000AD4B1A88182A18D03B681344A3F11800E6
:103080007F2840F3B683A94A973B82FB0321DA17D6
:10309000C2EB610202EB4202A3EB820303F1730075
:1030A000A34BC0B2197803F013FDA2490B78022B91
:1030B00000F253830133DBB20B701A469E4830F89E
:1030C0001260182E40F090820422032B03F10106B7
:1030D000F3B208BF002330F81360182E40F083824B
:1030E000013AF2D10B70019B1B88002B00F0CB82C0
:1030F000009B1B783BB9039B1B7823B9029B1B7871
:10310000002B00F0E0838D4B1B78002B00F0D68065
:103110008B490B78082B00F2D1808A483A68006806
:10312000894E0133DBB25F1E101A46F827000B7080
:10313000864B2668198889F800200BE77F4B1B789F
:10314000002B40F0C1823B68814A1278002A45D0AA
:10315000A3F10C007F2840F30A83744A8B3B82FB67
:103160000321DA17C2EB610202EB4202A3EB8203F6
:1031700003F17300C0B298F8001003F0A9FC009BA3
:103180001B7853B36E4E33783BB3DFF8FC91DFF816
:103190009CA14FF0000B0BE003F17300C0B298F854
:1031A000001003F095FC33780BF1010B5B4514DD47
:1031B0003B6859F8040F1844A0F18B038AFB0321E4
:1031C000DA17C2EB61020C3802EB42027F28A3EB54
:1031D0008203E1DCFDF756FAE0E73B685D4A1278CE
:1031E000002A3DD0504A1288182A18D01344A3F15F
:1031F00018007F2840F30D834C4A973B82FB032144
:10320000DA17C2EB610202EB4202A3EB820303F185
:103210007300C0B298F8001003F05AFC3B684549AF
:103220000A78022A00F2A6820132D2B20A70164649
:10323000414830F816E0BEF1180F40F0F081042646
:10324000032A02F1010E5FFA8EF208BF002230F865
:1032500012E0BEF1180F40F0E181013EF0D10A709A
:10326000019A1288002A00F041823B4903220B7028
:103270002A60FFF71FB8394F3B78002B3FF476A93F
:10328000374E307801F01EF9364B1B78002B00F0DA
:10329000918233887E2B00F28D82334A013310886D
:1032A00099B23180002800F09582C9B2C0B22F4E89
:1032B00003F0E6FB3B783370FEF7FCBF3A6837E774
:1032C000DBB21846137003F0B9FB294B1B491A46B1
:1032D0001F4B184600230B703B7013700370FFF7F1
:1032E00057B80123FFF796B880262249224B234A7C
:1032F00009881B8812680B44B2EB630FBFF6CFA896
:10330000164B1B78002B40F0FE81B9F800301C4AA8
:10331000B3423FF4C4A81B4B168001221A70FFF77A
:10332000BEB8FDF7AFF9B8E4789BFF1FABAAAA2A95
:10333000E29BFF1FA29BFF1F549DFF1F449DFF1F89
:10334000A089FF1F609BFF1F7C89FF1FFA9BFF1F47
:103350003C9BFF1FFC9BFF1F409DFF1F5E9BFF1FB1
:10336000889BFF1FC69DFF1FCC9BFF1F5B9BFF1F02
:103370008A9DFF1FEE9CFF1FF49CFF1F8C9BFF1F6D
:10338000109DFF1F5F9BFF1F7889FF1FC14B01939B
:103390001B88002B40F06C83BF4B0393BF4B029301
:1033A000BF4E33786BB3DFF81483DFF8F8A24FF029
:1033B000000B09E003F17300C0B203F0B1FB3378F6
:1033C0000BF1010B5B451CDD58F8043F99F8000038
:1033D0001844A0F17F038AFB0321DA17C2EB6102D4
:1033E00002EB42027F28A3EB8203E3DCFDF74AF9FC
:1033F000E2E7AA4B029303F093FB009B1B78002BA0
:10340000CED1039B1B78002B3FF4EDAB99F8003035
:10341000A3F10C007F2840F3A781A2488B3B80FBDF
:103420000320DA17C2EB600000EB4000A3EB80033F
:1034300003F17300C0B203F073FB009B1B78002BF9
:1034400000F08081964E3378002B00F06582DFF823
:103450006C82DFF850A24FF0000B0AE003F173001A
:10346000C0B203F05DFB33780BF1010B5B457FF7D6
:10347000BAAB58F8043F99F800001844A0F18B0348
:103480008AFB0321DA17C2EB61020C3802EB42021D
:103490007F28A3EB8203E1DCFDF7F4F8E0E7504678
:1034A000FDF7F0F8FFF788BBFDF7ECF8FFF7C6B9BA
:1034B000002008707C49087840B17C490091097867
:1034C000002900F0A981009F00213970784909780E
:1034D00000297FF420A8002E67D1002865D1754E01
:1034E000724F96F800E06C4E03966C4E02966A4E50
:1034F00071493070694E0097087038703070BEF1B5
:10350000000F7FF41AA8FFF721B8634B1B78002B3C
:103510003FF4CFAC99F80030A3F10C007F2840F3C2
:10352000C281604A8B3B82FB0321DA17C2EB610246
:1035300002EB4202A3EB820303F17300C0B203F07B
:10354000EFFA009B1B78002B3FF4B3AC544E33785A
:10355000002B3FF4AEAC594FDFF848814FF0000A22
:103560000AE003F17300C0B203F0DAFA33780AF12B
:10357000010A53457FF79DAC57F8043F99F80000C6
:103580001844A0F18B0388FB0321DA17C2EB610218
:103590000C3802EB42027F28A3EB8203E1DCFDF74B
:1035A00071F8E0E703980021017042490978002989
:1035B0003EF4CCAF394902910978002900F08881A6
:1035C000029800210170FEF7C1BF039B1B78002BFE
:1035D0007FF44DAB029B1B78002B7FF448AB019B23
:1035E0001988FFF74ABB0B703B681E44A6F1180010
:1035F0007F2840F301812B4B973E83FB0632F31764
:10360000C3EB620303EB4303A6EB830606F17300EF
:103610002B4BC0B2197803F05BFA64E50A7073446F
:10362000A3F118007F2840F3F1801E4A973B82FBEC
:103630000321DA17C2EB610202EB4202A3EB820321
:1036400003F17300C0B298F8001003F041FA3B6830
:1036500006E6243B002BB9F8000040F32F81984286
:103660003EF4F5AE9BB21748A9F800300123037071
:10367000FEF7EDBEDFF84880C0B298F8001003F006
:1036800027FAFFF70EBB0E4B3878197803F020FAB3
:103690002EE500BF949BFF1F3C9BFF1FFC9BFF1F61
:1036A000A089FF1FABAAAA2AC59DFF1F8A9DFF1FE5
:1036B000C19DFF1F5E9BFF1F449DFF1F7889FF1F59
:1036C000E29BFF1F5F9BFF1F7F21402003F0D8F983
:1036D000B349B44A3B680B600021117034E5C0B2B5
:1036E00098F8001003F0F4F9FFF7AFB8D8B298F8E3
:1036F000001003F0EDF93B68B7E5AB4BDFF8ECE207
:103700001978FEF7A4BE4B2E40F3A9801836802E00
:10371000B9F80030A54AA8BF8026B3427FF4FBADBC
:10372000FEF7BDBE99F8000003F0FAF93188FFF703
:10373000A4BA9F4B01931B88002B7FF45AAE9D4B7C
:10374000029363E6029B1B78002B7FF450AA039B35
:103750001B78002B7FF48BAA41E7002213460A70E6
:10376000ACE4FCF78FFF17E4FCF78CFF62E6FCF794
:1037700089FFFFE4002216460A7059E5FCF782FF34
:10378000FFF74DB98C4E307800F09CFE8B4B1B78C8
:103790001BB133887E2B40F2A780894B1B7823B165
:1037A0003388854A002B40F0AB80864E3B783370DF
:1037B000FEF780BD824B1B78002BF6D033887E4A03
:1037C000002BF2D08049013B088899B21180002873
:1037D0007FF46BADC8B27B4E03F0C6F93B78337013
:1037E000FEF768BD7F20FFF7D1B9FCF74BFFFFF76D
:1037F00017BAFCF747FF53E4FCF744FF08E7FCF770
:1038000041FFFFF72CBA7F20FFF7E5B8FCF73AFF3E
:1038100018E7FCF737FFFCE4664F6C4902974FF05E
:10382000000C81F800C0009F02994FF0010E87F84C
:1038300000E081F800C049E60120FFF7A7B903F0D6
:103840006FF9FFF7F5B80021402003F019F9FFF7F1
:1038500079BB99F8000003F063F9FFF76EBB243ED3
:10386000002EB9F800303ADDB3423EF418AEB6B2DD
:10387000574BA9F8006001221A70FEF710BE012014
:10388000FFF7A9B84A4B01931B88002B7FF4B3AD17
:10389000FFF7A9B94F4A8342A8BF03461360FEF75A
:1038A000B6BF16462CE5FCF7EDFE47E6FCF7EAFE50
:1038B000FFF71CBBFCF7E6FEFFF737BB01283EF421
:1038C000C6AD0123CFE699F8000003F029F91AE408
:1038D0004148009041483D490390FEF72EBE012B20
:1038E0003EF4DDAD0126C3E701339BB23380D9B28C
:1038F0000520344E03F0C4F83B783370FEF7DABC91
:10390000013B9BB2D9B205202E4E138003F0B8F8CC
:103910003B783370FEF7CEBC029B1B78002B7FF404
:1039200066A9FFF7A4B92E4B1B782BB32D4B1B7840
:10393000002B7EF4B4AD2C4B1B78002B3EF4AFADC6
:10394000B9F8003022490A33A9F800300A70FEF7AE
:10395000A6BD244B1B78002B7EF4A1AD224B1B7817
:10396000002B3EF49CADB9F800301949013BA9F891
:1039700000300A70FEF793BD1A4B1B78002B7FF4C2
:103980001BAA194B1B78002B3EF489ADB9F8003007
:103990000F490133A9F800300A70FEF780BD00BF5F
:1039A000609BFF1FA089FF1FAD9DFF1F109DFF1F84
:1039B000949BFF1FFC9BFF1F889BFF1FC69DFF1F43
:1039C000C59DFF1F5B9BFF1FCC9BFF1F449DFF1FDF
:1039D0005F9BFF1F409BFF1F8A9DFF1F3C9BFF1F9C
:1039E000C29DFF1FC39DFF1FC49DFF1FA99BFF1FFB
:1039F000224B00227F2107201A8003F041F87F210B
:103A00000B2003F03DF8FFF70ABA1D4B01227F217E
:103A100007201A8003F034F87F210B2003F030F8E0
:103A2000FFF7F5B9174B04227F2107201A8003F016
:103A300027F800210B2003F023F8FFF7E1B9114B21
:103A400002227F2107201A8003F01AF87F210B2021
:103A500003F016F8FFF7CFB90A4B002107201E80AC
:103A600003F00EF87F210B2003F00AF8FFF7BEB930
:103A7000054B0393054B0293BDE400BF5C9BFF1F06
:103A8000F29BFF1F389DFF1F3C9BFF1FFC9BFF1FEE
:103A900038B506F00DFC0E4804F0BEFC0D4804F0ED
:103AA000BBFC0D4804F0B8FC00234FF07E5201210E
:103AB0000A48FCF7DBFC0A4B0A4A0B498024002524
:103AC0001C7118461D60BDE838400AF00BBA00BFF3
:103AD000709BFF1F9C9BFF1FF89BFF1F149DFF1FE8
:103AE000949DFF1F1C89FF1F2906000043682A20A0
:103AF000198803F049B900BF10B504462220636855
:103B0000198803F041F9E36824201988BDE81040C2
:103B100003F03AB910B504460A206368198803F027
:103B200033F9E3680C201988BDE8104003F02CB984
:103B300010B5044606206368198803F025F9E36888
:103B400008201988BDE8104003F01EB910B50446DE
:103B500002206368198803F017F9E36804201988C4
:103B6000BDE8104003F010B970B50E4C84B01225BA
:103B70000422012306460390029320468DE8240088
:103B80001423102105F040FE062209230293039618
:103B90000195204600921423102105F035FE04B053
:103BA00070BD00BFEC9DFF1F2DE9F041224D82B09A
:103BB000012602B284B20092284601967823192188
:103BC00005F068FD04F10C0212B28DE844002846AD
:103BD000A7197823192104F1020805F05BFD3FB213
:103BE0000FFA88F819233A46284619460196CDF867
:103BF000008005F04FFD78233A4628461946CDF857
:103C00000080019604F10A070B3405F043FD3FB232
:103C100024B278233A46284619468DE8500005F02C
:103C200039FD192300943A4601962846194605F0B5
:103C300031FD02B0BDE8F081EC9DFF1F2DE9F041A0
:103C40001E4682B01446002A6AD0099B4D4A00EBFA
:103C5000C305012C6F8929896868A7EB010382FBE2
:103C600003E21A444FEAE373C3EBA21302887BD04A
:103C7000042C38D112FA83F3994203DC9F4239466F
:103C8000A8BF1946089A0180B6F90030BDF9208016
:103C90003D48971D4FF0000E3FB21946424600972F
:103CA000CDF804E005F0F6FC29896A896B68521AA0
:103CB0001B885C2AA3EB010359DD03EB43030132AC
:103CC000C3EB431393FBF2F303F11B0213B2012086
:103CD000328019464246019000972B4805F0DAFCE5
:103CE0002A4B00221A702A4B022CB3F9001045D03F
:103CF000082C31D100221A8091422DD0089AB6F9B1
:103D0000003021480632012412B200921946019473
:103D1000BDF9202005F0BEFC204602B0BDE8F081D0
:103D20001C4D1D4A2B681268CB1A93420F4617D9B7
:103D3000164A338811781448012918BF01241470D9
:103D4000089A06321BB212B28DE814001946BDF96A
:103D5000202005F09FFC2F60012002B0BDE8F0811B
:103D6000204602B0BDE8F0819BB2D31A84E75C2103
:103D700001FB03F393FBF2F21B32A7E74A1C12B2DA
:103D80001A80B9E7C94216B2EC9DFF1F769EFF1F4D
:103D9000D49DFF1F549EFF1F3CFF000030B583B031
:103DA00000230C4605B2009326225B231C210C48FD
:103DB00005F0C0F9294601232622094804F0D6FC63
:103DC000002C24B205DB214601232622044804F0FE
:103DD000CDFC044A044B15801C8003B030BD00BFED
:103DE000EC9DFF1F3E8AFF1F408AFF1FF0B59B4CD2
:103DF000237883B01BB19A4B4FF6FF721A80994B10
:103E0000B3F90030C3B9984A954B1068B3F9002054
:103E100080F30C005B2303FB00F000131C30824294
:103E20005ED04FF0FF31FFF7B9FF904805F0E6F99B
:103E30000023237003B0F0BD012B36D0022B6ED0CF
:103E4000032B53D0042BF3D1252200258DE8240029
:103E500076231C218548864E864F05F01BFC17E013
:103E6000B0F5AF7FA8BF4FF4AF70323803FB00F35B
:103E700087FB0321DB17C3EB61111C3109B201235E
:103E80001D442522794804F071FC0C2D00F084803B
:103E9000E9B2794804F028FB56F8042B801A31283F
:103EA0004FF05B03DCDC1C21E9E7744B1A68B2F5C8
:103EB0002F7F32DB41F25C239342A8BF1346A3F568
:103EC0002F735B226E4802FB03F380FB0320DB179A
:103ED000C3EBA0201C30624BB3F900308342A0D169
:103EE000684BB3F9003001339BD1A1E7664B1B68E7
:103EF000B3F5FA7F11DBB3F57A6FA8BF4FF47A639D
:103F0000A3F5FA7261485B2303FB02F380FB0320F5
:103F1000DB17C3EB20201C30DDE71C20DBE75C4B0C
:103F20001B68B3F5FA7F33DBB3F57A6FA8BF4FF4A4
:103F30007A63A3F5FA7255485B2303FB02F380FB17
:103F40000320DB17C3EB20201C30524B1B68B3F55A
:103F5000FA7F1FDBB3F57A6FA8BF4FF47A63A3F53E
:103F6000FA724A495B2303FB02F381FB0321DB174F
:103F7000C3EB21211C313A4BB3F9003083427FF46B
:103F800052AF404BB3F900308B427FF44CAF4FE758
:103F90001C20DAE71C21EEE7262200258DE824000C
:103FA00076231C2131483C4E324F05F073FB16E05E
:103FB000B0F5AF7FA8BF4FF4AF70323803FB00F30A
:103FC00087FB0321DB17C3EB61111C3109B201230D
:103FD0001D442622254804F0C9FB0C2D0CD0E9B263
:103FE0002E4804F081FA56F8042B801A31284FF03D
:103FF0005B03DDDC1C21EAE7272200258DE8240095
:1040000076231C211948264E1A4F05F043FB17E072
:10401000B0F5AF7FA8BF4FF4AF70323803FB00F3A9
:1040200087FB0321DB17C3EB61111C3109B20123AC
:104030001D4427220D4804F099FB062D3FF4F5AEF0
:10404000E9B2184804F050FA56F8042B801A3128C7
:104050004FF05B03DCDC1C21E9E700BFCA9DFF1FBA
:104060003E8AFF1FD09DFF1F489DFF1FEC9DFF1F35
:10407000F489FF1F4B48371B9C9BFF1F4C9BFF1F66
:10408000D3058541408AFF1F8C9BFF1F011FB8127B
:10409000989BFF1FBC9DFF1F4889FF1FF89BFF1FB8
:1040A000248AFF1F709BFF1F2DE9F04FDFF8F0926D
:1040B000B84CB9F900504E7854F8255087B00290AA
:1040C000039306B10E78DFF800B3002A35D19BF8D0
:1040D0000030002B31D1B04FB7F90000002800F0BC
:1040E000CE80012800F02481012032233246019045
:1040F00000930299A94B2846FFF7A0FD002604462D
:10410000B7F90030022B40F3F48000233B80B9F96B
:104110000030A34A002BC0F2F880042BC4BF002358
:104120001380039B002B40F0F680002E0CBF20462E
:104130004FF0FF3007B0BDE8F08F9A4C964FEB6818
:104140002A6804934FF0000820460592A7F80080E3
:104150008BF8008004F046FF1120FFF725FD4FF09B
:10416000010A192328212046CDF804A00091242219
:10417000194605F08FFA782328212422CDF804A0CF
:1041800000912046194605F085FA5146204605F073
:104190000BFEDDF814A0022319222382E28150468F
:1041A0000AF06EFC51460246204608F05BFA2046B3
:1041B00008F06EFA142303227B4923822046A4F8D8
:1041C0000E8008F04FFA204608F062FA232323827B
:1041D00003227649A4F80E80204608F043FA2046D0
:1041E00008F056FA049B002B73D10123704A18463D
:1041F0001370FFF7B9FC28896B896C68191A5C2960
:1042000022885CDC131A5C2202FB03F292FBF1F3BE
:104210001B33684A6348138001241BB21A221946D3
:104220008DE81400142205F035FA049BDBB1298ACD
:104230006B8AEC68581A5C2822886FDD521A02EBF0
:104240004202C2EB4212431C92FBF3F31B33534A6C
:1042500054481380012438221BB28DE814001946FB
:10426000322205F017FA544A544BB7F900000121E5
:1042700011704FF6FF721A8000287FF432AFDFF81A
:104280004C814F4AD8F8003002991268CB1A9342F9
:104290004CD9474B1A78012A18BF01201870FFF734
:1042A00063FC029BC8F800300124012E4DD0042E7F
:1042B00058D0022E5FD0082E63D0002620E7121AB5
:1042C00002EB4202C2EB42124B1C92FBF3F31B3394
:1042D0009FE72F20FFF768FC322303223949A4F817
:1042E0000E802046238208F0BDF9204608F0D0F960
:1042F0007BE77FF40CAFEB68002B3FF406AFB9F916
:104300000030274A002BBFF608AF04231380039B1D
:10431000002B3FF40AAFFFF769FD06E7511A5C2254
:1043200002FB01F292FBF0F31B3390E70446BCE77B
:10433000002414238DE81800324602991D4B2846AC
:10434000FFF77CFC26460446DAE6B9F800308BF825
:1043500000600133A9F800306B6983B1002628465C
:104360009847CDE6B9F800300122013BA9F80030AA
:104370008BF80020F0E701233B800026C7E61E46AD
:10438000BEE66B6900223A804FF0FF36002BE6D183
:10439000BDE600BF448AFF1FD49DFF1FCE9DFF1FB7
:1043A000D09DFF1FEC9DFF1FE4F30000E8F3000029
:1043B000769EFF1FCC9DFF1FCA9DFF1F3E8AFF1FD9
:1043C0003CFF0000ECF30000D29DFF1F549EFF1F36
:1043D00001210D2006F01EBB00210D2006F01ABBA6
:1043E00001460D2006F016BB08B50D2006F018FB9F
:1043F000B0FA80F149090D20BDE8084006F00ABB7B
:1044000010B5002144080D2006F004FB204606F0FC
:104410003DFB0D20012106F0FDFA2046BDE81040CD
:1044200006F034BB08B5214A214B12881868824235
:1044300034DA204B1B88991A8342A8BF0346B1F592
:10444000F87FA3EB020321DAC3EB031303EB43135F
:1044500093FBF1F105310A2006F04CF9164B19785F
:10446000F1B1164B16491B6883F30703C3EB031323
:1044700003EB431381FB03211944DB17C3EBA111A9
:1044800005310920BDE8084006F034B9C3EB4313F9
:104490001B01013193FBF1F10531DCE70021DAE783
:1044A0000920BDE8084006F025B900BFFA9BFF1FB0
:1044B000409BFF1FA09DFF1FB79BFF1F909DFF1FED
:1044C000090402817F2838B5A8BF7F200D4D4FF425
:1044D000FA7303FB00F485FB04232344E117C1EBCB
:1044E000A3110A2006F006F9A4F578400C3885FBE4
:1044F00000310144C017A0EBA111BDE838400920EC
:1045000006F0F8B809040281024B4E20198802F027
:104510003BBC00BF949BFF1F024B4420198802F054
:1045200033BC00BF789BFF1F024B1020198802F09C
:104530002BBC00BFFC9CFF1F024B2C20198802F0F3
:1045400023BC00BF6C9BFF1F024B1E20198802F08A
:104550001BBC00BF689BFF1FC3680E20198802F0B8
:1045600013BC00BF024B2820198802F00DBC00BF0D
:10457000509DFF1F024B6420198802F005BC00BF4C
:104580004C9DFF1F024B5A20198802F0FDBB00BF53
:10459000549BFF1F024B1620198802F0F5BB00BF89
:1045A0005C9BFF1F024B2E20198802F0EDBB00BF61
:1045B000EC9BFF1F024B3020198802F0E5BB00BFC7
:1045C000489BFF1F024B1820198802F0DDBB00BF7B
:1045D000FE9BFF1F024B1A20198802F0D5BB00BFBB
:1045E0009E9BFF1F024B1C20198802F0CDBB00BF11
:1045F000969BFF1F024B6620198802F0C5BB00BFC7
:10460000889DFF1F024B7220198802F0BDBB00BFBE
:10461000A49DFF1F024B2020198802F0B5BB00BFEC
:10462000869DFF1F024B3220198802F0ADBB00BFF0
:10463000769DFF1F024B6820198802F0A5BB00BFC2
:10464000CC9BFF1F024B6C20198802F09DBB00BF62
:10465000449BFF1F024B6E20198802F095BB00BFE0
:10466000C89DFF1F024B5220198802F08DBB00BF6E
:104670007889FF1F024B5020198802F085BB00BFCC
:10468000EC89FF1F024B5420198802F07DBB00BF4C
:10469000EE89FF1F024B5C20198802F075BB00BF3A
:1046A0003C8AFF1F024B5E20198802F06DBB00BFE1
:1046B0004489FF1F024B6020198802F065BB00BFD0
:1046C000EA9CFF1F024B5620198802F05DBB00BF19
:1046D000E09BFF1F38B5094D4624204602F06EFBD3
:1046E00035F8021B00B28842204601D002F04CFB94
:1046F0000234A4B24E2CF0D138BD00BF549DFF1F30
:10470000064B074A10B41C88064B0846002C14BF01
:1047100011461946042210BC0AF070BAB09BFF1F64
:10472000E8FA0000ECFA0000064B074A10B41C88B7
:10473000064B0846002C14BF11461946042210BC33
:104740000AF05CBAEE9BFF1FE8FA0000ECFA0000EA
:10475000064B074A10B41C88064B0846002C14BFB1
:1047600011461946042210BC0AF048BA4E9DFF1F9C
:10477000E8FA0000ECFA0000064B074A10B41C8867
:10478000064B0846002C14BF11461946042210BCE3
:104790000AF034BA429DFF1FE8FA0000ECFA00006C
:1047A000064B074A10B41C88064B0846002C14BF61
:1047B00011461946042210BC0AF020BAF29BFF1FD2
:1047C000E8FA0000ECFA0000F0B52B4E2B4FDFF8B2
:1047D000C4E005460FCE87B06C460FC496E80300D0
:1047E0003B68274A274F44F8040B40F6CC308342FD
:1047F000C8BF3A46BEF800602180012E1188927829
:10480000ADF80D108DF80F202AD032D340F6CA0231
:10481000022E18BF00229A4226DCA3F698031A49FA
:104820001A4AC3EB031381FB03011944DB17C3EBE3
:104830006123243382FB0321DA17C2EBA10202EBCE
:104840008201A3EB4103303330328DF813308DF801
:1048500011206946284616220AF0D0F907B0F0BDAB
:1048600040F698029A42D8DD094B1868CDF811003D
:10487000EFE740F6FC02CEE700FB0000609DFF1F63
:10488000F4FA0000F0FA00003B773B986766666632
:10489000F8FA0000DE9CFF1FF8B5174C174E22787F
:1048A000174D33782F888E46003218BF01220146FB
:1048B0007046FFF7F9FB002398423370237015DB35
:1048C00014BF012000202B889F420ED040F23A7284
:1048D000A3F5AF730B490C4C02FB03F381FB0312EE
:1048E000DB17A3EB621332332360F8BD07490122C3
:1048F00018460A702270E6E7E88AFF1FE59DFF1F51
:104900009C9DFF1FB5814E1BDC89FF1F6C9EFF1F06
:10491000014B187802F0D0B9509EFF1F014B187858
:1049200002F0E4B9FC8FFF1F134BB3F9003030B530
:1049300083EAE374A4EBE374002BA0B218DB012339
:1049400000E0134603EB830252009442F9DA0B4D68
:1049500090FBF3F285FB03E403FB1200DB1730321C
:10496000D3EBA40380B201F8012BF1D10B7030BD61
:104970002D230B700131E2E7FC8FFF1F676666662F
:10498000144BB3F9003070B583EAE375A5EBE3751A
:10499000002BACB21ADB012300E0034603EB8300DB
:1049A00040008542F9DA0C4E94FBF3F086FB03E5F8
:1049B00003FB1044DB173030D3EBA503A4B201F89E
:1049C000010BF1D105480B70106070BD2D230B70E9
:1049D0000131E0E7549BFF1F6766666618FB000025
:1049E000134BB3F9003030B583EAE374A4EBE374FE
:1049F000002BA0B218DB012300E0134603EB830277
:104A000052009442F9DA0B4D90FBF3F285FB03E47C
:104A100003FB1200DB173032D3EBA40380B201F8A2
:104A2000012BF1D10B7030BD2D230B700131E2E76A
:104A30007889FF1F67666666134BB3F9003030B59F
:104A400083EAE374A4EBE374002BA0B218DB012328
:104A500000E0134603EB830252009442F9DA0B4D57
:104A600090FBF3F285FB03E403FB1200DB1730320B
:104A7000D3EBA40380B201F8012BF1D10B7030BD50
:104A80002D230B700131E2E7EC89FF1F6766666634
:104A9000134BB3F9003030B583EAE374A4EBE3744D
:104AA000002BA0B218DB012300E0134603EB8302C6
:104AB00052009442F9DA0B4D90FBF3F285FB03E4CC
:104AC00003FB1200DB173032D3EBA40380B201F8F2
:104AD000012BF1D10B7030BD2D230B700131E2E7BA
:104AE000EE89FF1F67666666134BB3F9003030B579
:104AF00083EAE374A4EBE374002BA0B218DB012378
:104B000000E0134603EB830252009442F9DA0B4DA6
:104B100090FBF3F285FB03E403FB1200DB1730325A
:104B2000D3EBA40380B201F8012BF1D10B7030BD9F
:104B30002D230B700131E2E73C8AFF1F6766666632
:104B4000134BB3F9003030B583EAE374A4EBE3749C
:104B5000002BA0B218DB012300E0134603EB830215
:104B600052009442F9DA0B4D90FBF3F285FB03E41B
:104B700003FB1200DB173032D3EBA40380B201F841
:104B8000012BF1D10B7030BD2D230B700131E2E709
:104B90004489FF1F67666666054B1B881BB9054B7A
:104BA000186808607047044B18680860704700BFB9
:104BB000949BFF1F20FB00001CFB0000164B1B8872
:104BC0000BB31BB230B583EAE374A4EBE374002BA0
:104BD000A0B21CDB012300E0134603EB830252006A
:104BE0009442F9DA0D4D90FBF3F285FB03E403FBED
:104BF0001200DB173032D3EBA40380B201F8012B93
:104C0000F1D10B7030BD064B1868086070472D233A
:104C10000B700131DEE700BF689BFF1F67666666A9
:104C2000ECFA0000164B1B880BB31BB230B583EABD
:104C3000E374A4EBE374002BA0B21CDB012300E0BF
:104C4000134603EB830252009442F9DA0D4D90FBB8
:104C5000F3F285FB03E403FB1200DB173032D3EBE6
:104C6000A40380B201F8012BF1D10B7030BD064BCB
:104C70001868086070472D230B700131DEE700BF14
:104C80007A9DFF1F67666666ECFA0000164B1B886C
:104C90000BB31BB230B583EAE374A4EBE374002BCF
:104CA000A0B21CDB012300E0134603EB8302520099
:104CB0009442F9DA0D4D90FBF3F285FB03E403FB1C
:104CC0001200DB173032D3EBA40380B201F8012BC2
:104CD000F1D10B7030BD064B1868086070472D236A
:104CE0000B700131DEE700BF5C9BFF1F67666666E5
:104CF00024FB0000174B1B881BB31BB270B583EA63
:104D0000E375A5EBE375002BACB21EDB012300E0DD
:104D1000034603EB830040008542F9DA0E4E94FB14
:104D2000F3F086FB03E503FB1044DB173030D3EBD5
:104D3000A503A4B201F8010BF1D108480B70106073
:104D400070BD074B1868086070472D230B70013148
:104D5000DCE700BFEC9BFF1F67666666FCFA00009D
:104D6000ECFA0000164B1B880BB31BB230B583EA7C
:104D7000E374A4EBE374002BA0B21CDB012300E07E
:104D8000134603EB830252009442F9DA0D4D90FB77
:104D9000F3F285FB03E403FB1200DB173032D3EBA5
:104DA000A40380B201F8012BF1D10B7030BD064B8A
:104DB0001868086070472D230B700131DEE700BFD3
:104DC000489BFF1F67666666ECFA0000164B1B885F
:104DD0000BB31BB230B583EAE374A4EBE374002B8E
:104DE000A0B21CDB012300E0134603EB8302520058
:104DF0009442F9DA0D4D90FBF3F285FB03E403FBDB
:104E00001200DB173032D3EBA40380B201F8012B80
:104E1000F1D10B7030BD064B1868086070472D2328
:104E20000B700131DEE700BF889DFF1F6766666675
:104E3000ECFA0000164B1B880BB31BB230B583EAAB
:104E4000E374A4EBE374002BA0B21CDB012300E0AD
:104E5000134603EB830252009442F9DA0D4D90FBA6
:104E6000F3F285FB03E403FB1200DB173032D3EBD4
:104E7000A40380B201F8012BF1D10B7030BD064BB9
:104E80001868086070472D230B700131DEE700BF02
:104E9000A49DFF1F67666666ECFA0000174B1B882F
:104EA0001BB31BB270B583EAE375A5EBE375002B6A
:104EB000ACB21EDB012300E0034603EB830040009D
:104EC0008542F9DA0E4E94FBF3F086FB03E503FB13
:104ED0001044DB173030D3EBA503A4B201F8010B6B
:104EE000F1D108480B70106070BD074B186808605E
:104EF00070472D230B700131DCE700BF869DFF1F3B
:104F00006766666628FB0000ECFA0000074B1B880A
:104F1000022B06D0012B0CBF054B064B186808600E
:104F20007047054B18680860704700BFEA9CFF1F78
:104F300030FB000034FB00002CFB0000054B1B88FD
:104F40001BB1054B186808607047044B186808606F
:104F5000704700BFE09BFF1F3CFB000038FB0000D8
:104F600008B5702001F02AFF044B1988884204D04C
:104F70007020BDE8084001F007BF08BDDE9CFF1FA0
:104F800008B5742001F01AFF044B1988884204D038
:104F90007420BDE8084001F0F7BE08BD6C9DFF1FFE
:104FA00038B5FCF7D1FC0D4B1B7833B90C4B1020F6
:104FB000198801F0E9FE012038BD0A4D0A4C2B7812
:104FC0002288B3FA83F382F008025B09114642207B
:104FD0002B70228001F0D8FE002038BD5E9BFF1FA1
:104FE000FC9CFF1FE29CFF1FA29DFF1F184B1A880D
:104FF00052B3184A128830B50A80B3F90030002B3A
:1050000083EAE374A4EBE374BCBF2D238B70A0B2DE
:10501000ACBF02310331012300E0134603EB8302EE
:1050200052009442F9DA0C4D90FBF3F285FB03E455
:1050300003FB1200DB173032D3EBA40380B201F87C
:10504000012BF1D10B7030BD044B1868086070471C
:105050009E9BFF1F40FB000067666666ECFA00003F
:1050600010B40A4B0A4C0A4693E8030083B0238825
:1050700002AC04E9030004EB8303104653F8081C58
:10508000052203B010BC09F0B9BD00BF74F40000E4
:105090004C9DFF1F30B40A4B0A4D0C4693E80700A5
:1050A00084B02B8804AD05E9070005EB8303204697
:1050B00053F80C1C042204B030BC09F09FBD00BFA3
:1050C0007CF40000DE9CFF1FF0B40C4D0C4F0E462C
:1050D0000FCD8CB001AC0FC40FCD0FC495E8070005
:1050E0003B8884E807000CAA02EB8303304653F8A0
:1050F0002C1C04220CB0F0BC09F080BD88F4000028
:10510000389DFF1FF0B40A4D0A4F0E460FCD86B0F2
:1051100001AC0FC42A683B88226006AA02EB830315
:10512000304653F8141C042206B0F0BC09F066BDEA
:10513000B4F40000FE9BFF1FF0B40A4D0A4F0E4668
:105140000FCD86B001AC0FC42A683B88226006AA46
:1051500002EB8303304653F8141C0C2206B0F0BC5B
:1051600009F04CBDC8F40000969BFF1FF0B40A4D37
:105170000A4F0E460FCD86B001AC0FC42A683B889B
:10518000226006AA02EB8303304653F8141C042263
:1051900006B0F0BC09F032BDDCF400006C9DFF1FCE
:1051A000164B1B880BB31BB283EAE370A0EBE370D2
:1051B000002B30B584B21DDB012300E0134603EB66
:1051C000830252009042F9DA0D4894FBF3F280FB1F
:1051D00003E503FB1244DB173032D3EBA503A4B283
:1051E00001F8012BF1D10B7030BD084604220549AE
:1051F00009F004BD2D230B700131DDE7CC9BFF1FAF
:105200006766666644FB0000F0B40A4D0A4F0E461E
:105210000FCD86B001AC0FC42A683B88226006AA75
:1052200002EB8303304653F8141C042206B0F0BC92
:1052300009F0E4BCF0F40000449BFF1F70B53C4D46
:105240002B780646002B35D11C4673780BB92046C7
:1052500070BDFCF779FB374A374B38481278317804
:105260001B78007802EB43034A1E03EB80030E2AEF
:10527000EDD801A050F822F0E152000003530000E5
:105280004F520000E15200004F5200004F52000008
:105290004F520000CF5200004F5200004F5200000A
:1052A0004F5200004F5200004F5200004F5200007A
:1052B000CB520000AE21224803F048FC204803F006
:1052C00091FE00232B700124BFE705F0F1FEAF2112
:1052D0001B4803F03BFC1B4A012313702B70B6E7FD
:1052E00083B91948038804294FF6FF7103F1FF328F
:1052F0000CBF01230B46134403F07F0301330380EB
:105300000FE073B1013B114A32F813304BB10E4E2E
:105310000F481049104A33800123002606700B7095
:105320001370084A0221012311702B70204670BDB2
:10533000E88AFF1F8B9DFF1F849DFF1F8C9DFF1F11
:10534000EC9DFF1F6C9EFF1F109DFF1FD09CFF1F39
:10535000C49BFF1F5F9BFF1F789EFF1F10B5064B6E
:10536000064C1A882046012101F0FCFC21884220CD
:10537000BDE8104001F008BDB09BFF1FA29DFF1FBC
:1053800010B5064B064C1A882046022101F0EAFCB3
:1053900021884220BDE8104001F0F6BCEE9BFF1FC3
:1053A000A29DFF1F10B5064B064C1A88204605210A
:1053B00001F0D8FC21884220BDE8104001F0E4BC97
:1053C0004E9DFF1FA29DFF1F10B5064B064C1A886D
:1053D0002046002101F0C6FC21884220BDE8104093
:1053E00001F0D2BC429DFF1FA29DFF1F08B51220F5
:1053F00001F0E4FC054B1988884206D0122001F028
:10540000C3FCBDE8084001F0D7BB08BD389DFF1FB5
:1054100008B5582001F0D2FC054B1988884206D007
:10542000582001F0B1FCBDE8084001F0C5BB08BD43
:105430007A9DFF1F08B5142001F0C0FC054B1988A8
:10544000884206D0142001F09FFCBDE8084001F01E
:10545000B3BB08BDF29BFF1FF0B480EAE075A5EB7B
:10546000E0750028ACB21FDB1DBF2B230B704E1C58
:105470000E46012300E0134603EB830252009542DF
:10548000F9DA0B4F94FBF3F287FB030503FB12449D
:10549000DB173032D3EBA503A4B206F8012BF1D110
:1054A00033700846F0BC70472D230B704E1CE0E7AC
:1054B00067666666084B188828B10D2807D00D3836
:1054C00000B2FFF7C9BF054A106808607047044A78
:1054D00010680860704700BFC89DFF1FECFA00000D
:1054E00048FB0000174B18880C2813D0192815D03A
:1054F0001A2817D01B2819D01C281BD01D281DD0F6
:105500001E2803D00C3800B2FFF7A6BF0E4A106861
:10551000086070470D4A1068086070470C4A1068B0
:10552000086070470B4A1068086070470A4A1068A4
:1055300008607047094A106808607047084A106898
:1055400008607047769DFF1F64FB00004CFB000065
:1055500050FB000054FB000058FB00005CFB000007
:1055600060FB0000034B1888A0EB8000400000B2F5
:10557000FFF772BF509EFF1F024B1888033800B21E
:10558000FFF76ABF509DFF1F024B18880C3800B20E
:10559000FFF762BF589BFF1F024B1888183800B2F4
:1055A000FFF75ABF789BFF1FC3681888183800B2EE
:1055B000FFF752BF30B5134C85B001252B463C2276
:1055C00002212046009503F037FB204603F00AFD38
:1055D00000224021802320460191009311460A4B6E
:1055E000029504F0ADF9204603F008FE074808498B
:1055F000084A0023036083800B608B8013609380D4
:1056000005B030BDEC9DFF1F90F60000D89DFF1F38
:10561000709EFF1F5C9EFF1F10B500EBC00000F1E5
:105620000F02D2B293B284B09C1E981C3D2303910A
:105630008DE819003921024804F0E6F804B010BDE5
:10564000EC9DFF1F014B01221A707047E59DFF1F63
:10565000F0B585B0634C644B0293644A0192042315
:105660000093634E634B644F644D2046402280217B
:1056700003F0EAF82046624A6249634C08F032FCC3
:10568000B761624FF761624FAF61624FEF61624F86
:10569000A7616248624FE761624F87616249634F69
:1056A000C761634F8F61634A634FCF61634F9761F7
:1056B000634B644FD761644F9F61644E644FDF61F9
:1056C000644FB761644D654FF761654FAF61654CDD
:1056D000654FEF61654F6648A761664FE761664FAA
:1056E00066498761664FC761664F674A8F61674F3A
:1056F000CF61674F674B9761674FD761674F684EC0
:105700009F61684FDF61684F684DB761684FF7610F
:10571000684F694CAF61694FEF61694FA761694894
:10572000694FE761694F876169496A4FC7616A4F8D
:105730008F616A4A6A4FCF616A4F97616A4B6B4FBC
:10574000D7616B4F9F616B4E6B4FDF616B4FB761E2
:105750006B4D6C4FF7616C4FAF616C4C6C4FEF61F0
:105760006C4FA7616C486D4FE7616D4F87616D4964
:105770006D4FC7616D4F8F616D4A6E4FCF616E4F38
:105780006E4B97616E4FD7616E4F6F4E9F616F4F3B
:10579000DF616F4F6F4DB7616F4FF7616F4F704CA7
:1057A000AF61704F70487149EF61714F714DA761E2
:1057B000E561714F714D724CDFF8E8E1714A724B4F
:1057C0008761C5618C61714EC1F81CE0704F714DED
:1057D000714C724872499761D5619C61D861B16022
:1057E00005B0F0BDEC9DFF1FA0860100801A0600E9
:1057F0004C8DFF1F2490FF1F89550000808EFF1FD6
:105800001C89FF1FA1880000F08DFF1F5945000073
:105810007955000065450000014700002C8CFF1FF2
:105820005D53000029470000E08CFF1F81530000FA
:10583000514700000090FF1FA55300006150000079
:10584000988CFF1F7545000079470000288DFF1FC9
:10585000C953000065550000048DFF1F1149000069
:10586000294900005C8EFF1F1D4900009550000073
:10587000E48BFF1F614F0000C9500000E88EFF1F3E
:10588000ED530000254C0000748CFF1F11540000E4
:1058900081490000A08BFF1F85450000A147000043
:1058A000548FFF1F355400008D4C0000508CFF1F9B
:1058B00095450000F54C0000708DFF1FA5450000C8
:1058C000654D0000108BFF1FB5450000055100001D
:1058D000BC8CFF1FC5450000ED4F0000388EFF1F38
:1058E000D545000039510000D88FFF1FE545000065
:1058F000CD4D0000CC8DFF1FF5450000354E00005A
:10590000348BFF1F054600006D5100000C8FFF1FF8
:10591000814F00009D4E0000148EFF1F15460000B1
:10592000E5540000588BFF1F25460000A1510000E0
:10593000EC8AFF1F3546000009520000588AFF1FFD
:1059400045460000B5540000A88FFF1F55460000D3
:10595000E1490000088CFF1F65460000394A00003D
:10596000C48AFF1F754600007C8BFF1FA48EFF1F9B
:10597000914A000085460000E94A00009546000073
:10598000414B0000A08AFF1F7C8AFF1FCC8FFF1FA6
:105990000D4F0000B54600003D4F0000C546000019
:1059A000555F0000A5460000F0B5461C83B00D46CB
:1059B0000127032336B22AB2044631468DE8880017
:1059C0002448ADB203F0B6FE0C23AA1C12B2009319
:1059D0000197052321B21F4803F0ACFE1E4A1F4B5E
:1059E00012881B68BA422AD023D3022A10D11C4C39
:1059F000A3F6CA0384FB03241C44DB17C3EB241463
:105A00000A2CA8BF0A2424EAE474A2B223B202E05A
:105A100000231A461C460D35AA1A01200093019056
:105A200012B2314603230B4803F002FE204603B0B6
:105A3000F0BD0C4CA3F6FC0384FB0324DDE7084C0B
:105A4000A3F6980384FB03241C44DB17C3EBE40494
:105A5000D6E700BFEC9DFF1FDE9CFF1F609DFF1F70
:105A6000898888881F85EB512DE9F0438FB283B078
:105A7000DFF84C80BD1D461D2DB204B236B24FF08A
:105A800001090AB22346314640460095CDF80490FC
:105A900003F000FE2A463346214640468DE82002A8
:105AA00003F0F8FD07F10C020095334612B22146CF
:105AB000CDF80490404603F0EDFD03B0BDE8F0835F
:105AC000EC9DFF1F2DE9F04F804685B0002959D18C
:105AD0000121314804F068F9304998F8062098F817
:105AE000083011F80290994525DADFF8ACB04FEA9A
:105AF00089064D460C244FF0000AD8F80C309B590B
:105B00005F68ABF810403846ABF80EA008F0B8FF5D
:105B100039460246204806F0A5FD1F4806F0B8FDAC
:105B200098F8083001350934AB42A4B206F10406F6
:105B300001DD422CE1D1B9F1000F13D109F10609C1
:105B400099450CDA3C2301213B22039102930093F7
:105B5000019239233F223A210F4803F055FE05B048
:105B6000BDE8F08F0F2301213B22039102930093A4
:105B7000019239230C223A21074803F045FE98F898
:105B80000830DBE700213423009301913F230C22EE
:105B9000014803F04DFD9BE7EC9DFF1F709EFF1F2A
:105BA00038B50F4C012320461946A3826382552540
:105BB00004F0FAF83423204602220A492382E581C0
:105BC00006F050FD20460522074906F04BFD204611
:105BD00006F05EFD2046BDE8384003F00FBB00BF75
:105BE000EC9DFF1F68FB00006CFB0000F8B50F4642
:105BF000064608F045FF00EB40008400AFB338468E
:105C000008F03EFF00EB4000400023185B10194DE8
:105C100003F16002121A4FF0280E01212846C3F149
:105C20006004EA81A5F810E004F0BEF8384608F0F8
:105C300027FF39460246284606F014FD284606F09E
:105C400027FD02210B4804F0AFF8212330462B82B8
:105C5000EC8108F015FF31460246064806F002FDC9
:105C60000448BDE8F84006F013BD6410C4F16004B8
:105C7000004DE6E7EC9DFF1F10B50D4B1B5C51F886
:105C80002340237884B013B1012004B010BD04AACE
:105C900001A942F8103D2046A3699847A38A9B07B3
:105CA000F2D401A80099FFF7A1FF012004B010BDB4
:105CB000D89DFF1F2DE9F04F304DDFF8D0B0DFF851
:105CC000C8A00FCD91B003AC0FC40FCD0FC40FCD42
:105CD0000FC42B6823600025A8462F462E4600E0FF
:105CE0009846BAF8003026495BF82320DFF8A090E8
:105CF00011232846FAF76AFE00EBC00300EB83008D
:105D0000204B83FB00340444C017C0EB6434C4F15F
:105D10003C00C6F13C0207F14101012600B208F146
:105D2000410300901BB2019612B209B2484603F03B
:105D3000B1FC08EB060305F211153C2B2646ADB26B
:105D40004746CDD16B22342300214846A9F80E20C6
:105D5000A9F8103004F028F80B4B1B8810AA02EBAE
:105D6000830353F8344C204608F08AFE214602464D
:105D7000484611B0BDE8F04F06F074BC04F50000D1
:105D80000CF10000090002806C9BFF1F24F0000052
:105D9000EC9DFF1F214B70B5B3F9003083EAE3742B
:105DA000A4EBE374002B82B0A1B22FDB68466D46F2
:105DB000012300E0134603EB830252009442F9DA18
:105DC000174E91FBF3F286FB03E403FB1211DB1782
:105DD0003032D3EBA40389B205F8012BF1D1194677
:105DE0002B70FFF703FF0F4B1B786BB10E4C01219B
:105DF000204603F0D9FF74253323204601220B49A6
:105E0000E581238206F02EFC02B070BD2D238DF8B3
:105E100000300DF101056846CAE700BFFC9CFF1F7A
:105E200067666666E29CFF1FEC9DFF1FFCFE00009C
:105E300070B5404E404D82B0304603F0D3F82B7819
:105E4000D3B93C4C0621204603F0AEFF2B78012B42
:105E500038D9022B4FF003024FF00A030CBF374929
:105E60003749E3812046238206F0FCFB204602B03E
:105E7000BDE8704006F00CBC324B1A7801210523B6
:105E8000002A33D1019100931146304603F052FCB1
:105E90002D4B1A78002A34D0052301220192009359
:105EA00000220A21234803F0C3FB284B1A78002A5A
:105EB00033D1012105230191009314211D4803F0E2
:105EC00039FCBEE7224B1988092930D963298CBFD8
:105ED0000A221F220A231748F281338206F028FC87
:105EE000144802B0BDE8704006F0D2BB0022019118
:105EF00000931146304603F09BFB134B1A78002A9F
:105F0000CAD105230121019100930A21094803F018
:105F100011FC0E4B1A78002ACBD0012205230192E6
:105F2000009300221421034803F082FB89E730220A
:105F3000D0E700BFEC9DFF1F789EFF1F74FB0000A1
:105F400078FB00008B9DFF1F849DFF1F8C9DFF1F12
:105F5000109DFF1F2DE9F047714E307848B9714B05
:105F60001B6899425FD3704A012313703370BDE8F8
:105F7000F0876E4D6B4F0C46284603F033F804F65D
:105F8000AC5331240022EC810124114628462A8298
:105F9000AC826C823B60327003F006FF05226449DC
:105FA000644E284606F05EFB102728464FF00C088A
:105FB00006F06EFB0B226049EF812846A5F81080A1
:105FC00006F050FB5D490522284606F04BFB2846AB
:105FD00006F05EFB5A4BEF811A68A2F69803C3EBFA
:105FE000031386FB03161E44DB17C3EB662640F63D
:105FF000CC3320219A42298206F124064FF0220157
:106000004FF0040011DCFFF7CFFC4E4BB3F80090CB
:106010008246B9F1000F30D0B9F1010F4DD0B9F17E
:10602000020F47D02046BDE8F087FFF71DFD464927
:106030000922284606F016FB4449EF8181FB06370A
:10604000F317C3EBA7072A23394628462B8206F00D
:106050006FFB22463E49284606F004FB07EB87010A
:10606000A6EB4101284606F063FB22462846394943
:1060700006F0F8FA2046BDE8F08737493A46284648
:1060800006F0F0FA284606F003FB2A232B8251463D
:10609000EF8128462D4F06F04BFB07222F4928465B
:1060A00006F0E0FAF31787FB0627C3EBA70739468C
:1060B0002846CCE742462A49E1E742462949234C93
:1060C000284606F0CFFA284606F0E2FA2A232B8269
:1060D00051462846EF8106F02BFB07221F49284630
:1060E00006F0C0FAF31784FB0624C3EBA404214690
:1060F000284606F01DFB4A461549284606F0B2FA26
:1061000004EB8401A6EB4101284606F011FB4A4648
:106110002846104906F0A6FA4846BDE8F08700BFB9
:10612000E88AFF1F589EFF1F6C9EFF1FEC9DFF1FFC
:106130007CFB00003B773B9884FB00006CFB00007D
:10614000609DFF1FDE9CFF1F90FB00006766666678
:1061500070000100E0FF00009CFB0000B0FB0000AD
:10616000C8FB0000B8FB00002DE9F041744C227818
:10617000002A05460F4614BF4FF001084FF00008F3
:106180004ED1704E3368CB1AB3F5FA6F04D86B78E2
:10619000A3B94046BDE8F0816B4B6C486C49DFF811
:1061A000CCE11A70012303700988237026208EF831
:1061B000002000F0E9FD6B78002BEAD03760FBF798
:1061C000C3FB644A644B6549127828781B780978C8
:1061D00002EB4303421E03EB81030E2AD9D801A12F
:1061E00051F822F0D16200009D620000936100002E
:1061F000D162000093610000936100009361000090
:1062000085620000936100003B6200009361000022
:106210009361000093610000936100003762000009
:10622000AF214F48474E02F091FCFFF701FE0023DB
:1062300037602370ABE704F03BFF494C204602F087
:10624000D1FE2046022103F0AFFD23250F23238238
:1062500005224449E581204606F004FA204606F06E
:1062600017FA1E230522404923822046E58106F0C5
:10627000F9F9204606F00CFA204602F0BFFF00F0C4
:10628000A7FC86E7394D2B78012B50D9304B2620BF
:10629000198800F079FD00232B707AE7002B3FF47A
:1062A00078AF013B324A32F81330002B3FF471AF24
:1062B000274C304825492D4A23804FF00108002300
:1062C000037081F8008082F80080FFF7B1FD60E77D
:1062D00093B1013B264A32F8131019B31C4B254DDC
:1062E0001A4C224A19800026012326202E70237082
:1062F000137000F049FD15E0154C1E4922880B7003
:1063000004284FF6FF7002F1FF310CBF0122024654
:106310000A440E4E154D02F07F0201320121228007
:1063200031702B70FFF784FD4FF0010831E706490B
:10633000064A01230020087013702370A6E700BFEF
:10634000E88AFF1F689EFF1F6C9EFF1F5F9BFF1F59
:10635000109DFF1F8B9DFF1F849DFF1F8C9DFF1FA6
:10636000EC9DFF1FD8FB0000E0FB0000789EFF1FA4
:10637000D09CFF1FC49BFF1F2DE9F04FAE4E4FF086
:106380000109A6F81490A6F81290838813EA09046C
:106390008BB005460F46934640F0AB80DFF8C482D1
:1063A00098F80030002B7BD1AA79A44CA35CA3B948
:1063B000DFF8B4A279781AF8029039B33B78013B40
:1063C000072B00F2B280DFE813F0EF005101B000BC
:1063D0006B01B000B000B000E7007E78002E00F046
:1063E000C580013BE868397850F82360F0684B1E9F
:1063F0000788072B00F2A380DFE813F07001590132
:10640000A1006A01A100A100A1009B008C4E33688D
:10641000C3EB0B03B3F5967F72D98A4B187801282A
:106420001ABF012018701970874B18BF0146985C7D
:10643000C0EB0900C0B2FFF7EFF80124C6F800B0C6
:10644000AB889B076DD57B78002B6AD0FBF77CFA75
:106450007E4B7F4A7F481B78127839780078022576
:1064600015FB02330A2903EB800300F049810C2954
:1064700057D1002B55D003F11900774E774A013BD5
:106480000021400080B226F813100123157088F80F
:10649000003000F079FC724B032220461A702CE089
:1064A000304602F09FFD3046494603F07DFCF48102
:1064B0003482AB88580725D42C68204608F0E0FACF
:1064C00021460246304606F0CDF8304606F0E0F8A8
:1064D000092201238DE80C0000217F23564803F098
:1064E000D9F800212846FFF7EDFA002388F800309C
:1064F0005AE783681146384698470BB0BDE8F08FDD
:106500000846FAE72B6804A8984704A808F0B8FAE8
:1065100004A90246304606F0A5F8304606F0B8F861
:10652000D6E720460BB0BDE8F08F00240AF80290B1
:1065300086E70023A3543046F3699847F068078044
:10654000002425223C238DE81400412118223A48DA
:1065500003F06EF8E968A879FFF78EFB394A384BEB
:106560001470C3F800B00BB0BDE8F08F34490B686D
:10657000C3EB0B03B3F5967F40F2E080314FC1F8D7
:1065800000B03C78012C00F0AF800123E9683B703B
:106590001046FFF771FBB0E7304BE9791970012322
:1065A00088F800300024C1E72B7A013B4B45BCDD65
:1065B00009F10104E4B2A145B7D0234E16F802B0A8
:1065C000CBEB0900C0B20021FFF726F82B7A052B90
:1065D000D9461BD9CBEB0402042A40F3A980A4F1CD
:1065E000040BBBF1000FC0F2AD80063B5B45A8BFBA
:1065F0005B465FFA83F9AA791348B15C994205D0EA
:1066000000F8029001212846FFF75CFAC9EB04006C
:10661000C0B201210B4EFEF7FFFF00213423019190
:1066200000930B223170044840233F21A14602F021
:10663000FFFF0124AA7979E7EC9DFF1F5C9EFF1FF5
:10664000549EFF1F769EFF1F709EFF1F8B9DFF1F96
:10665000849DFF1F8C9DFF1FD09CFF1F6C9EFF1F02
:10666000789EFF1FE88AFF1FD89DFF1F0FFA89F34E
:10667000E9685D4851F823B0036804935B499BF8CF
:10668000003004980860002B6CD0012B7FF44DAFD4
:1066900057499BF8080088F800300870002445E747
:1066A000B9F1000F4CD009F1FF34E4B283E7B38AAB
:1066B00003F004039BB2002B3FF43CAF336A9847CE
:1066C00000283FF43BAFAB79F0680022E25436E794
:1066D000738ABB4240D90137BFB230E7338ABB422D
:1066E00034D2013FBFB22AE725238DE84800414854
:1066F0003E703C231822412102F09AFF2046FCE61E
:10670000002B3FF40EAF3C4A3C4E1188384A03F14F
:106710001900013B400080B226F81310012388F8CD
:106720000030157000F030FB354B20461D70E4E65C
:10673000002A3FF75AAF04F1FF3B52E73046DCE650
:106740004C46F3E64FF000094B4654E7B38AD907AD
:106750007FF5F5AE778AF2E6B38ADA077FF5EFAE1A
:10676000378AECE627490393885CC0EB090009F1FE
:10677000010EC0B2012104F802E0FEF74DFF039BB9
:10678000DBF808B0019334231A4800930B2240230E
:106790003F2102F04DFF012434230B228DE8180025
:1067A0003F214023134802F0C5FF2146114803F062
:1067B000FBFA584608F064F9A0EB800000F15F0393
:1067C0000F22F3813282584608F05AF959460246A0
:1067D000084805F047FF074805F05AFFE968A8791F
:1067E000FFF74AFAAA79A1E6949EFF1F549EFF1F65
:1067F0006C9EFF1FEC9DFF1F109DFF1FD09CFF1F75
:10680000789EFF1F709EFF1F2DE9F047DFF808926A
:106810006D4B99F800601B68DFF800A282B000366B
:1068200001934FF0030018BF0126019F9AF80080E2
:1068300004F0F6F80546042004F0F2F804460520BA
:1068400004F0EEF8800040EA4404062004F0E8F882
:106850002C4364B25D4944EAC0000A7880F00F031B
:10686000DBB29A425A4A3CD01760002259480B705A
:1068700003788DF800808DF8012053B3564A1268D2
:106880004EF66021BA1A8A4219D8022B59D0012B30
:106890005FD0062B48D0032B63D0042B69D0052B87
:1068A00077D0072B7DD0082B00F08380092B68D090
:1068B00016B14A4802F0A2FC02B0BDE8F087484A8F
:1068C000484C00230121237003701360938089F8E2
:1068D00000103A4669464448FFF74EFD3043C6B2C1
:1068E000E6E71268BA1A1E2A6BD99AF8002093427A
:1068F00022D0394C3D488AF80030012B276082EACB
:10690000030207609846B1D0042BAFD13748006826
:10691000381AB0F5C87FA9D9354C2068381A322802
:10692000A4D927601A46A1E73A4669463148FFF7DD
:1069300023FD3043C6B2BBE7012B4FF00002E3D189
:10694000E4E73A4669462C48FFF716FD3043C6B2E5
:10695000AEE73A4669462948FFF70EFD3043C6B216
:10696000A6E73A4669462648FFF706FD3043C6B219
:106970009EE73A4669462348FFF7FEFC3043C6B21D
:1069800096E73A4669462048FFF7F6FC3043C6B220
:106990008EE73A4669461D48FFF7EEFC3043C6B223
:1069A00086E73A4669461A48FFF7E6FC3043C6B226
:1069B0007EE73A4669461748FFF7DEFC3043C6B229
:1069C00076E7002252E700BF949EFF1F799EFF1FCB
:1069D000E09DFF1F6C9EFF1F649EFF1FEC9DFF1F2D
:1069E0005C9EFF1F779EFF1F3CF600007C9EFF1FF2
:1069F000E89DFF1F90FA000000F6000060F500001F
:106A000044F5000094F5000050F50000A4F50000E6
:106A1000E4F50000CC8FFF1FE88AFF1FE49DFF1FF5
:106A200028B11028044BA8BF102018607047024BF3
:106A300001201860704700BF809EFF1F38B50F4DC2
:106A40002B78013B01381B02C4B203F470632004AD
:106A500043F4404343F00C0300F4FE00184305F0F8
:106A600045F92868013860F03F00C0B204F06EF9C3
:106A70002046BDE8384004F069B900BF809EFF1F82
:106A800070B5124D2B78013B1B0203F47063064670
:106A900043F430430806320400F0FE4043F00B0399
:106AA000034302F4FE0018430C4605F01FF9286862
:106AB000013860F04F00C0B204F048F9304604F0ED
:106AC00045F92046BDE8704004F040B9809EFF1FA4
:106AD00070B5124D2B78013B1B0203F47063064620
:106AE00043F410430806320400F0FE4043F009036B
:106AF000034302F4FE0018430C4605F0F7F828683B
:106B0000013860F06F00C0B204F020F9304604F0A4
:106B10001DF92046BDE8704004F018B9809EFF1FA3
:106B200038B5104D2B78013B1B0203F4706304460B
:106B300043F41043000443F0090300F4FE0018433B
:106B400005F0D4F82868013860F06F00C0B204F096
:106B5000FDF8204604F0FAF80020BDE8384004F0C3
:106B6000F5B800BF809EFF1F38B50E4D2B78013B56
:106B70001B0203F47063044643F45043000443F0E3
:106B80000D0300F4FE00184305F0B0F82868013842
:106B900060F02F00C0B204F0D9F82046BDE83840BC
:106BA00004F0D4B8809EFF1F08B5002005F068F9F6
:106BB0000028FAD108BD00BF08B564210720FFF7FF
:106BC0005FFF7F210B20BDE80840FFF759BF00BFE2
:106BD00010B500217B20FFF753FF0024E0B2FFF740
:106BE0009FFF0134022003F051FF802CF6D110BD2D
:106BF00010B504464FF4406004F058F804F0B0F8C3
:106C00002CB1102C044BA8BF10241C6010BD024BEB
:106C100001241C6010BD00BF809EFF1F10B50446FC
:106C200041F0E00004F092F804F07F0004F08EF8E8
:106C3000C4F3C610BDE8104004F088B838B5134D51
:106C40002B78044641F6FF72A0F50050824203F112
:106C5000FF33A8BF02461B0202F5005203F4706323
:106C6000100443F4604343F00E0300F4FE005204AA
:106C7000184302F0FE42104305F038F82968013944
:106C80002046C9B2BDE83840FFF7C8BF809EFF1F4D
:106C900038B504460D46F02004F058F835B12544C7
:106CA00014F8010B04F052F8AC42F9D1F720BDE81A
:106CB000384004F04BB800BF00B50B4B83B0024620
:106CC000998818680090032AADF8041002D903B01F
:106CD0005DF804FB684606218DF80520FFF7D8FF14
:106CE00003B05DF804FB00BFA0FF000000B50B4B34
:106CF000024683B0186899880090131F4C2BADF89A
:106D0000041002D903B05DF804FB684606218DF833
:106D10000520FFF7BDFF03B05DF804FBA8FF0000EE
:106D2000030203F4FE43C0F3C6101843704700BFCC
:106D300003784078DB0103F47E5300F07F001843B2
:106D4000704700BF82B002AA114642F8040D00202D
:106D500012F8013B03F07F03914243EA0020F7D190
:106D600002B07047003210B403884FF0010404FAF7
:106D700001F418BF012202FA01F123EA04020A43D6
:106D8000028010BC704700BF70B5CEB20C460546FD
:106D900003F0D6FA864203D03146284603F0EAFAD9
:106DA0000135284603F0CCFA240A844205D0214656
:106DB0002846BDE8704003F0DDBA70BD38B5054621
:106DC00003F0BEFA4FF0000460F30704681C03F000
:106DD000B7FA60F30F24A0B238BD00BFF8B504467F
:106DE0000020FFF7EBFF002C00F0CD834FF4AF61E4
:106DF0000220FFF7C9FF4FF47A610420FFF7C4FFB8
:106E00004FF496610620FFF7BFFF4FF4FA610820A8
:106E1000FFF7BAFF4FF4AF610A20FFF7B5FF40F666
:106E2000FC010C20FFF7B0FF4FF496612220FFF722
:106E3000ABFF4FF416612420FFF7A6FF7D212A2027
:106E4000FFF7A2FF0C210E20FFF79EFF012110206B
:106E5000FFF79AFF02211220FFF796FF002114206E
:106E6000FFF792FF00211620FFF78EFF0221182066
:106E7000FFF78AFF01211A20FFF786FF02211C205D
:106E8000FFF782FF04211E20FFF77EFF1421202040
:106E9000FFF77AFF01212620FFF776FF0321282044
:106EA000FFF772FF04212C20FFF76EFF0F212E2029
:106EB000FFF76AFF00213020FFF766FF0C21322028
:106EC000FFF762FF00213420FFF75EFF002136202C
:106ED000FFF75AFF00213820FFF756FF00213A2024
:106EE000FFF752FF00213C20FFF74EFF00213E201C
:106EF000FFF74AFF00214020FFF746FF0021422014
:106F0000FFF742FF1F214420FFF73EFF13214620D9
:106F1000FFF73AFF0E214820FFF736FF11214A20E4
:106F2000FFF732FF0A214C20FFF72EFF00214E20F1
:106F3000FFF72AFF06215020FFF726FF02215220EB
:106F4000FFF722FF0C215420FFF71EFF00215620DF
:106F5000FFF71AFF00215820FFF716FF01215A20E2
:106F6000FFF712FF03215C20FFF70EFF0A215E20CE
:106F7000FFF70AFF00216020FFF706FF04216220CF
:106F8000FFF702FF01216420FFF7FEFE00216620CB
:106F9000FFF7FAFE0B216820FFF7F6FE7F216A203B
:106FA000FFF7F2FE00216C20FFF7EEFE00216E20BD
:106FB000FFF7EAFE00217020FFF7E6FE00217220B5
:106FC000FFF7E2FE00217420FFF7DEFE2321002000
:106FD000FFF7DAFE0220FFF7F1FEB0F5805F03460F
:106FE00080F01184D24A04201380FFF7E7FEB0F549
:106FF000805F034680F0FE83CE4A06201380FFF7B1
:10700000DDFEA0F52F739BB2B3F57A6F024606D969
:1070100040F628210620FFF7B7FE40F62822C64B8F
:1070200008201A80FFF7CAFEA0F52F739BB2B3F5B4
:107030007A6F024606D940F6E4410820FFF7A4FE25
:1070400040F6E442BD4B0A201A80FFF7B7FEA0F5D8
:10705000FA739BB240F6AC518B42024606D94FF40C
:10706000AF610A20FFF790FE4FF4AF62B44B0C20E3
:107070001A80FFF7A3FEA0F5FA739BB240F6AC515D
:107080008B42024606D940F6FC010C20FFF77CFE3D
:1070900040F6FC02AB4B0E201A80FFF78FFE18283B
:1070A000034600F2A183A84A10201380FFF786FE52
:1070B000431E9BB20F2B024604D901211020FFF77B
:1070C00063FE0122A14B12201A80FFF777FE0A28E7
:1070D000034600F283839E4A14201380FFF76EFE5E
:1070E0000128034604D900211420FFF74DFE002398
:1070F000984A16201380FFF761FE7F28034600F2AE
:107100006783954A18201380FFF758FE042803462A
:1071100000F25883914A1A201380FFF74FFE0C2883
:10712000034600F249838E4A1C201380FFF746FE77
:107130000428034600F23A838A4A1E201380FFF790
:107140003DFE0928034600F22B83874A2020138046
:10715000FFF734FE4628034600F21C83834A2220B0
:107160001380FFF72BFEA0F5FA739BB240F6AC51EB
:107170008B42024606D94FF496612220FFF704FEA7
:107180004FF496627A4B24201A80FFF717FEA0F581
:10719000FA739BB240F6AC518B42024606D94FF4CB
:1071A00016612420FFF7F0FD4FF41662714B262084
:1071B0001A80FFF703FE7F28034600F2E5826E4A3D
:1071C00028201380FFF7FAFD0628034600F2D68236
:1071D0006A4A2A201380FFF7F1FDA0F132039BB227
:1071E000B3F5967F024604D97D212A20FFF7CCFD16
:1071F0007D22634B2C201A80FFF7E0FD0C2803460C
:1072000000F2B6825F4A2E201380FFF7D7FD1E28BA
:10721000034600F2A7825C4A30201380FFF7CEFDC0
:107220000928034600F26382584A32201380FFF790
:10723000C5FD1E28034600F25482554A34201380AF
:10724000FFF7BCFD7F28034600F24582514C3620F3
:107250002380FFF7B3FD7F28034600F236823820F3
:107260006380FFF7ABFD7F28034600F228823A20B7
:10727000A380FFF7A3FD7F28034600F21A823C207B
:10728000E380FFF79BFD7F28034600F20C823E203F
:107290002381FFF793FD7F28034600F2FE81402003
:1072A0006381FFF78BFD7F28034600F2F0814220C7
:1072B000A381FFF783FD384D28804420FFF77EFD32
:1072C0003028034600F2DD81344A46201380FFF760
:1072D00075FD3028034600F2CE81314C48202380D2
:1072E000FFF76CFD3028034600F2BF814A2063801F
:1072F000FFF764FD3028034600F2B1814C20A380E3
:10730000FFF75CFD3028034600F2A3814E20E380A6
:10731000FFF754FD0128034604D900214E20FFF752
:1073200033FD00231F4A50201380FFF747FD3BE049
:10733000FA9BFF1FA09DFF1FB29BFF1F749DFF1FA5
:10734000469DFF1F809BFF1F589BFF1FFC9CFF1F3C
:10735000389DFF1FF29BFF1F5C9BFF1FFE9BFF1FC3
:107360009E9BFF1F969BFF1F689BFF1F869DFF1F15
:10737000F49CFF1FEE9CFF1F109DFF1F509DFF1FE1
:107380009C9DFF1F6C9BFF1FEC9BFF1F489BFF1FDB
:10739000769DFF1FD09CFF1FA29DFF1F789BFF1FA4
:1073A000549DFF1F949BFF1F431E9BB20B2B024655
:1073B00004D906215020FFF7E7FC0622CF4B5220CC
:1073C0001A80FFF7FBFC0428034600F23C81CC4AFC
:1073D00054201380FFF7F2FC431E9BB21D2B024684
:1073E00004D90C215420FFF7CFFC0C22C54B5620AA
:1073F0001A80FFF7E3FC0128034604D90021562038
:10740000FFF7C2FC0023C04A58201380FFF7D6FCC8
:107410007F28034600F21181BC4A5A201380FFF7EF
:10742000CDFC431E9BB2092B024604D901215A20F0
:10743000FFF7AAFC0122B64B5C201A80FFF7BEFCC6
:10744000431E9BB2102B024604D903215C20FFF798
:107450009BFC0322AF4B5E201A80FFF7AFFC431E5C
:107460009BB21D2B024604D90A215E20FFF78CFC3B
:107470000A22A94B60201A80FFF7A0FC02280346CD
:1074800000F2D580A54A64201380FFF797FC0128FD
:10749000034604D901216420FFF776FC0123A04AAA
:1074A00062201380FFF78AFCC31E9BB2012B0246A9
:1074B00004D904216220FFF767FC0422994B66205F
:1074C0001A80FFF77BFC7F28034600F2AA80964AC9
:1074D00068201380FFF772FC7F28034600F29B8030
:1074E000924A6A201380FFF769FC7F28034600F266
:1074F0008C808F4A6C201380FFF760FC04280346C1
:107500007DD88C4A6E201380FFF758FC192803465B
:107510006FD8894A70201380FFF750FC0228034679
:1075200061D8864A72201380FFF748FC062803467C
:1075300053D8834A74201380FFF740FC042846D8B0
:107540002B88DFF81CE27F4F7F4A804D804E814CB4
:10755000814903F0010CAEF800C0C3F3400EA7F858
:1075600000E0C3F380071780C3F3C0077B4A2F7086
:10757000C3F30017C3F34015C3F38013378025808E
:107580000B801080F8BD4FF6FF7398423FF42EAC8D
:1075900023283FF41FAD17287FF628AC19287FF663
:1075A00091AC1B287FF6AEAC1C283FF4C3AC1E2860
:1075B0007FF6C8AC1F283FF4CDAC20283FF4E6ACE2
:1075C00021283FF4EFAC22287FF400ADF2E47420D0
:1075D0000021FFF7D9FB0020B2E700217220FFF75E
:1075E000D3FB0023A5E700217020FFF7CDFB00238C
:1075F00097E700216E20FFF7C7FB002389E70021F2
:107600006C20FFF7C1FB00237BE77F216A20FFF797
:10761000BBFB7F236DE70B216820FFF7B5FB0B2336
:107620005EE700216620FFF7AFFB00234FE7002154
:107630006020FFF7A9FB002324E700215820FFF773
:10764000A3FB0023E8E602215220FFF79DFB022363
:10765000BDE60A214C20FFF797FB0A2356E61121CD
:107660004A20FFF791FB112348E60E214820FFF73F
:107670008BFB0E233AE613214620FFF785FB1323ED
:107680002BE61F214420FFF77FFB1F231CE6002170
:107690004020FFF779FB002309E600213E20FFF799
:1076A00073FB0023FBE500213C20FFF76DFB00236B
:1076B000EDE500213A20FFF767FB0023DFE500211D
:1076C0003820FFF761FB0023D1E500213620FFF7CA
:1076D0005BFB0023C3E500213420FFF755FB0023AB
:1076E000B4E50C213220FFF74FFB0C23A5E5002168
:1076F0003020FFF749FB002396E500BFEC89FF1F10
:107700007889FF1FEE89FF1FE09BFF1F7A9DFF1FF7
:10771000549BFF1F3C8AFF1F4489FF1FEA9CFF1FE9
:107720004C9DFF1FA09BFF1F889DFF1FCC9BFF1F31
:10773000889BFF1F449BFF1FC89DFF1FDE9CFF1FF0
:10774000A49DFF1FB09BFF1FEE9BFF1FE29CFF1F2E
:10775000EC9CFF1F4E9DFF1F049DFF1F6C9DFF1F94
:10776000429DFF1F0F212E20FFF70EFB0F2352E536
:1077700004212C20FFF708FB042343E503212820E4
:10778000FFF702FB032323E501212620FFF7FCFA84
:10779000012314E514212020FFF7F6FA1423DDE479
:1077A00004211E20FFF7F0FA0423CEE402211C205E
:1077B000FFF7EAFA0223BFE401211A20FFF7E4FAF7
:1077C0000123B0E402211820FFF7DEFA0223A1E42E
:1077D00000211620FFF7D8FA002392E4022112209C
:1077E000FFF7D2FA022376E40C210E20FFF7CCFA41
:1077F0000C2358E44FF47A610420FFF7C5FA4FF4E4
:107800007A63FFF7F9BB4FF4AF610220FFF7BCFAD0
:107810004FF4AF63FFF7E6BBF8B5872006F09CFB9B
:10782000204B214A054603CB1368C5F803001A0C08
:107830007620C5F807102B80AA70FFF771FA2E4644
:10784000002426F80B0FA0B2FFF7B8FAFFF768FA8A
:107850000234762C26F8020FF5D16C1E05F1820653
:107860004FF0FF3014F8013F082758400F4B40F30A
:1078700000017A1E0B4012F0FF0783EA5000F5D199
:10788000B442EFD1C043FFF75DFA3A46C5F8830032
:107890008721284604F078FA2846BDE8F84006F02B
:1078A00063BB00BFB4FF0000B0FF00002083B8ED51
:1078B000F0B50E4B0E4C054693E8070085B02468E2
:1078C0002E88AD7801AB83E80700270C184600220C
:1078D0000B21ADF804408DF80670ADF80C608DF802
:1078E0000E5004F051FA05B0F0BD00BFC0FF00001B
:1078F000B0FF0000F0B5124B124D1E68124F0FCDB5
:1079000087B06C460FC495E8030044F8040B386850
:107910003B79CDF80D00320C232021808DF8022018
:107920008DF81130ADF80060FFF7FAF90022ADF8DC
:107930000B001221684604F027FA07B0F0BD00BF23
:10794000B0FF0000CCFF00006CFB0000002004F042
:1079500097BA00BF02F0ACBC70B5104C82B00025E5
:107960004023064629462046009301958023202285
:1079700001F05EFE0123202230462282A382638230
:10798000E58107F07DF831460246204604F06AFEA4
:10799000204602B0BDE8704001F030BCEC9DFF1FF6
:1079A000F0B5862983B075D90546441E00F18206DC
:1079B0004FF0FF3014F8012F08275040404A40F3A1
:1079C00000017B1E0A4013F0FF0782EA5000F5D148
:1079D000B442EFD1C043FFF7B5F90146D5F88300B3
:1079E0000190019A914202D0B2F17F2F0BD105F1A3
:1079F0000B00FFF79DF976280BD03248FFF7ACFF5C
:107A0000002003B0F0BD3048FFF7A6FF384603B0B2
:107A1000F0BD05F10D00FFF78BF9232840D10024BC
:107A200040F6AC5613E004281AD0062821D00828C6
:107A30001FD00A2828D00C2822D1A1F5FA7292B2C0
:107A4000B24201D8FFF7A0F90234762C0ED004F12F
:107A50000D002844FFF76CF9022C0146A0B2E2D1D8
:107A6000B1F5805FEED30234762CF0D1012003B063
:107A7000F0BDA1F52F7292B2B2F57A6FE4D8E1E7CA
:107A8000222801D0242811D1A1F5FA7292B2B24273
:107A9000DAD8D7E70D48FFF75FFF002003B0F0BD4D
:107AA0000B48FFF759FF002003B0F0BD2A28C9D1C9
:107AB000A1F1320292B2B2F5967FC5D8C2E700BFFB
:107AC0002083B8ED10000100FCFF0000E4FF00007F
:107AD0002400010003290CD970B5461C82B005466C
:107AE0000C46304603222A4907F038F810B102B09C
:107AF00070BD70470B2C05D905222649281D07F0BB
:107B00002DF840B12448FFF727FF244802B0BDE814
:107B10007040FFF7CDBE05F10901032201A807F06F
:107B20006DF801A803221E4907F018F8D8B1032206
:107B30001C4901A807F012F808B301A803221A494A
:107B400007F00CF8B0B91948FFF706FFA11E89B27B
:107B50003046FFF725FF0028C9D0154802B0BDE820
:107B60007040FFF7F9BE1348FFF7F6FEFFF754FE2B
:107B70001148F3E71148FFF7EFFE1148C6E7114837
:107B8000FFF7EAFE02B0BDE87040FFF7B3BE00BFEA
:107B9000B0FF00003C00010044000100580001005B
:107BA0005C000100840001009C000100A0000100B5
:107BB000B40001006000010074000100C800010071
:107BC000DC000100880001002DE9F043174D2B680F
:107BD00083B081460F469046F3B1154E34880A199A
:107BE00092B218461146328006F034FD28603A46BB
:107BF0004946204402F0E0F8B8F1000F09D031887E
:107C00002868FFF767FF286806F0AEF900232B60AD
:107C1000338003B0BDE8F083054E01930846318000
:107C200006F09AF9019B28601C46E0E7889EFF1F3A
:107C3000849EFF1F10B51D4C4FF4FA70FCF7E0FB5B
:107C4000204601F0CFF90023194601222046E381A6
:107C50002382A282628202F0A7F80B2214492046F6
:107C600004F000FD204604F013FD0F2211492046C8
:107C700004F0F8FC204604F00BFD0F4907222046D3
:107C800004F0F0FC204604F003FD204601F0B6FAB3
:107C90000A4B0B4A1A604FF4FA70FCF7B1FBFFF77E
:107CA00029FE0848BDE81040FFF756BEEC9DFF1FB7
:107CB000E0000100EC000100FC00010020A0FF1F1B
:107CC000C97B0000040101000020704790F83920B2
:107CD00090F83800101A704790F8383090F8392032
:107CE0009A4205D95A1C034480F83820187E704700
:107CF0004FF0FF30704700BF90F8383090F83920CF
:107D00009A4286BF1B18187E4FF0FF30704700BFA5
:107D1000704700BF38B50546B0F85E0090B195F8E1
:107D20005D301446C3F1210294420CD805F13B00AA
:107D30001844224602F040F895F85D30234485F857
:107D40005D30204638BD012014462871EEE700BFA3
:107D5000B0F85E306BB190F85D30202B07D8C218B8
:107D6000013380F85D30012082F83B107047012319
:107D700003710020704700BF0023426980F838304B
:107D800080F8393080F85C3080F85D3080F85E3003
:107D900080F85F3006CA30B40D68046943662A4330
:107DA00083660A60A370426990F8613016491468CE
:107DB00013441D7A5B7B01EBC5051B026D6803F460
:107DC000E06343F064032B6090F8623013449D7CC1
:107DD000DB7D01EBC5011B02496803F4E06343F05E
:107DE00064030B6021685368194205D00369272298
:107DF0005A70036904229A71036920225A71036937
:107E000080229A7030BC7047280C010043690CCB6B
:107E100012681A420CD0094B99420AD9084B994270
:107E2000036994BF1A220D225A70036904229A71C1
:107E30007047036927225A70F7E700BF7F1A0600D0
:107E40003F420F0010B50269D378DBB2D906044671
:107E50003DD510215806D17038D503F0040303F046
:107E6000FF02002B51D03D49626E00230B7084F855
:107E70005D30002A5BD0904794F85D30002B56D0DF
:107E80002369D0229A70236994F83B201A712369E0
:107E9000012284F85C200222DA7010BD304B84F895
:107EA00060009C424AD02F4B9C4252D094F839102B
:107EB00013791F29DBB207D82848007820B1601851
:107EC000013184F8391003760223D37010BD5906AE
:107ED000C3D4917801F0100101F0FF000029DDD03A
:107EE00013F001031ED194F85C1094F85D008842F1
:107EF00081BF4B1C091984F85C3091F83B30137139
:107F00002369D0229A702269DEE7236984F8392038
:107F1000C0229A702369114A197901211170022235
:107F2000DA7010BDC023937022691379CCE7012267
:107F3000002384F85D2084F83B30A1E7626994F85F
:107F40006130094913440322187A02F001FB2269C7
:107F5000ACE7626994F861300449F3E78C9EFF1F37
:107F60002490FF1F9090FF1FCD7F0000D97F00005D
:107F70000369DB7803F0200373B190F860300133BC
:107F8000DBB2012B80F860301AD9426990F8613079
:107F90001344187A02F058BB70B5426903F0FF052C
:107FA00090F8613013440446187A02F04DFBA36E3A
:107FB0005BB184F8385094F83900BDE87040184738
:107FC00090F85F30002BE0D0704770BD0148FFF79C
:107FD000CFBF00BF2490FF1F0148FFF7C9BF00BFFC
:107FE0009090FF1F2DE9F047374FDFF8E0903B6896
:107FF000026982B006460093DDF800800021A025CA
:10800000D3789B065BD53B680193019BC8EB0303C8
:108010000F2BF5D949B1102BF2D0002090703369A5
:1080200080229A7002B0BDE8F087726996F86130DC
:1080300013440521187A02F001FD726996F8613047
:108040001344012193F812A0504602F0F7FC0924D2
:108050000021504602F0DEFC2B46013BFDD1012100
:10806000504602F0D7FC2B46013BFDD1013CEFD13D
:10807000706996F8611001444FF4A0720C7A4B7B42
:1080800009EBC4011B02496803F4E06343F0640395
:108090000B6096F862300344997CDB7D09EBC101EB
:1080A0001B02496803F4E06343F064030B60013A88
:1080B000FDD13269D3789B064FF00101A3D4012092
:1080C00002B0BDE8F08700BF949EFF1F280C01009E
:1080D000F0B503691222DA700269937803F0200385
:1080E00085B004460D46002B5ED0B42393703C4906
:1080F00022690B680093009E05E00B680193019BC9
:108100009B1B042B42D8D37803F0200303F0FF001D
:10811000002BF2D094F85D30002B31D04FF0000EE0
:108120004FF0020C04EB0E0393F83B3013710B6815
:108130000393039F206907E09B060DD50B6802930C
:10814000029BDB1B052B28D8C378DBB203F00202AD
:1081500002F0FF06002AEFD080F803C02669F3780A
:10816000DBB2DF0632462DD49F062BD5DB0731D498
:108170000EF1010E94F85D305FFA8EFE7345D1D892
:1081800000201DBB002384F85E3004E0907023695A
:1081900080229A70042005B0F0BD86702369802289
:1081A00004209A7005B0F0BD03F0FF06FFF71AFF38
:1081B00010B9042005B0F0BD236984F85F60B022D7
:1081C0009A7094E78023B3700420DAE7266980234D
:1081D000B370D7E7BEF1000F0CBF02200320F6E713
:1081E000949EFF1F2DE9F04106690025122780F8B3
:1081F000385080F83950F770D0F810C09CF802E081
:108200000EF0200E88B00446884615461E46BEF184
:10821000000F49D0B4238CF80230784B21691A68DA
:108220000092DDF800E006E01A6801920198CEEBBA
:108230000000042830D8C87800F0200000F0FF07C4
:108240000028F1D04FEA480242F00102D2B20A718E
:108250001A680292DDF808E0206906E01A680392C5
:108260000399CEEB010105292AD8C17801F002015A
:1082700001F0FF070029F1D04FF0020C80F803C095
:108280002269D17811F0110722D12DBB002E0CBF2D
:10829000A0238023937003E08F70236980229A705B
:1082A000384608B0BDE8F0810EF0FF07FFF79AFEF0
:1082B0000028F5D0236984F85F70B0229A70ACE78B
:1082C00087702369802238469A7008B0BDE8F08133
:1082D000802393700027E3E7012D75D0A0219170D2
:1082E00021690A79BE4667464FF0A80C1A680492C5
:1082F000049805E01A680592059A121A052A4AD8C8
:10830000CA7802F0020202F0FF08002AF2D0CF7011
:108310002169CA78D2B212F0100F08465AD19206DB
:1083200058D5013DEDB2012D49D0BEF11F0F3BD90B
:108330000A79012DDAD11A680692069D05E01A68BD
:108340000792079A521B052A46D8C27802F0020209
:1083500002F0FF01002AF2D00223C3702269D37811
:10836000DBB2D9063AD49B0634D5B023BEF11F0F39
:1083700093703FD8226904EB0E0312791A760EF13E
:10838000010E5FFA8EFE16B1236980229A7084F87E
:1083900039E0774684E781F80280236980229A7069
:1083A000774684F839E07BE704EB0E0291F804800D
:1083B00082F818800EF1010E5FFA8EFEB9E781F89F
:1083C00002C021690846B0E7A82191702069BE4625
:1083D0000279B0E7774663E78170DEE71021A023DA
:1083E000D170013BFDD12269937803F0F703774602
:1083F000937055E723691B79C5E700BF949EFF1F63
:108400000148FFF71FBD00BF2490FF1F0148FFF781
:1084100019BD00BF9090FF1F704700BF38B5144CC6
:10842000037801225B000546204684F83B3084F83F
:108430005E2084F85D20FFF78BFC20460021FFF7CB
:1084400047FE0B4C2978012320461A46FFF7CAFE47
:108450000128F6D194F8383094F839209A4205D999
:10846000E218013384F83830107E38BDFF2038BD63
:108470002490FF1F38B51B4C037801225B00054692
:10848000204684F83B3084F85E2084F85D20FFF7B6
:108490005FFC20460021FFF71BFE124C2978204686
:1084A00001230222FFF79EFE0228F6D194F838201D
:1084B00094F839108A420FD2531CDBB2A0189942AB
:1084C00084F83830007E0AD9234402321B7E84F8B7
:1084D000382040EA032038BD4FF6FF7038BD40F425
:1084E0007F4038BD2490FF1F0C2901D90020704720
:1084F0000231490001F0FE01FFF7BCBF70B50C4C22
:108500000378164601255B00204684F83B3084F84A
:108510005E5084F85D50FFF71BFC31462046FFF7A4
:1085200017FC29462046BDE87040FFF7D1BD00BFCB
:108530002490FF1FF8B505460F46164641242146F4
:108540003A462846FFF7DAFF611C0234C9B23246C8
:108550002846E4B2FFF7D2FF592CF0D1F8BD00BF96
:1085600038B504460D463548FFF706FC63228021E6
:1085700020462570FFF7C2FF012002F087FA20464F
:1085800000225E21FFF7BAFF20465D21FFF746FF7C
:10859000242801D0002038BD204606220C21FFF7F8
:1085A000C9FF204601222B21FFF7A8FF2046012208
:1085B0002C21FFF7A3FF20460E222D21FFF79EFF5F
:1085C000204600222E21FFF799FF204601222F216D
:1085D000FFF794FF204605223021FFF78FFF20464A
:1085E00001223121FFF78AFF204600223221FFF7C6
:1085F00085FF204600223321FFF780FF204600221E
:108600003421FFF77BFF204600223521FFF776FF5C
:10861000204600225B21FFF771FF204610225C21DB
:10862000FFF76CFF204620225D21FFF767FF204601
:108630008F225E21FFF762FF012038BD2490FF1FCB
:1086400010B4047F4160022CC26002D010BC03F061
:1086500087BE836810BC184790E80C00F0B41C6813
:1086600059682568164F174E29432160164D174942
:108670001760D66015611160417A154A5C180A319D
:1086800094F8244053F8215002EBC40149680D606E
:10869000017A5C1803EB8101247ECD6902EBC401F1
:1086A00049680D60817A581803EB810390F8300017
:1086B000596B02EBC002F0BC53681960704700BFF1
:1086C00001401F00011000380110007800001F80D9
:1086D000280C0100704700BFF0B50C1EBDF81460F7
:1086E00034DBB0F906701919B942C4BF3B1B1BB289
:1086F000002BA6461CDD002A1146B8BFD11D02F092
:108700000705CC10826A012007FB04E1A840012E76
:108710000A44C0B21ED00CD3022E09D1013B12FA7A
:1087200083F3013A12F8011F41409A421170F9D1C6
:10873000F0BDC043013B12FA83F3C0B2013A12F814
:10874000011F014093421170F9D1F0BD23441BB2C7
:108750000024C6E7013B12FA83F3013A12F8011F25
:1087600001439A421170F9D1F0BD00BF00291EDB10
:1087700030B4B0F90A408C4218DD002A16DBB0F99B
:108780000C40944212DD047E022C54D0032C4CD0B9
:10879000012C06D15140C4884A405140013C611A25
:1087A00009B2012B2DD017D3022B01D030BC70475A
:1087B000002AB0F90630856A1446B8BFD41D44F3C8
:1087C000CF0404FB031102F007026B5C012000FAE6
:1087D00002F25A406A54E9E7002AB0F90630856A85
:1087E0001446B8BFD41D44F3CF0404FB031102F0B8
:1087F00007026B5C012000FA02F223EA02026A54CB
:10880000D4E7002AB0F90630856A1446B8BFD41DF3
:1088100044F3CF0404FB031102F007026B5C012058
:1088200000FA02F21A436A54C0E70489013C641A50
:10883000114622B2B5E7C5880489013D013C691A99
:10884000A21A09B212B2ACE72DE9F041079E9DF9D8
:108850001880089D04461F4600F0BCFF0D4B0E48D3
:108860000E4984F83380FF22002F08BF1F4684F88A
:108870002F20002384F8302084F8312084F832201F
:1088800020606665A565676221662362A362204653
:10889000BDE8F0812490FF1F900101000110013814
:1088A00010B50446806A034B236008B105F05CFBF9
:1088B000204610BD90010100F8B5436ADBB190F885
:1088C0002C200125AA4083F83B2083F85E5083F8D2
:1088D0005D500446406A03680E461B6800219847B5
:1088E000606A036831461B6898472946606ABDE89C
:1088F000F840FFF7EDBBC26BC56C1368046A23EA4E
:10890000050313604CB122684FF00043D3625163FA
:10891000D36A002BFCDA936BF8BD836B466B08259A
:10892000802410E03768426C3A4332601F68826CE2
:108930003A431A601A68876C013D22EA07024FEA3F
:1089400054041A6007D02142ECD13268476C22EA05
:1089500007023260EAE7F8BD70B50446406A0D468A
:1089600000282BD0616DFFF751FA002D20460CBF77
:10897000A621A721FFF7A0FF606A20B1A16DBDE885
:108980007040FFF743BA216C226D0868236A0243E6
:108990000A6093B1DA7A82B1D00703D5224A996985
:1089A0001160DA7A910703D5204AD9691160DA7A21
:1089B000520702D51E4A1B6A136070BD236A002B42
:1089C0002BD0D97A226EE1B172B6D97ACE0706D50C
:1089D0001848D9680668314099610160D97A8807DA
:1089E00006D51548196906683140D9610160D97A00
:1089F0004E0705D511485969066831401962016072
:108A000062B61B68D968914207D00D4818600D49BD
:108A1000DA6042F0804018611960226C216D1368A1
:108A200023EA01031360A0E700E100E004E100E0B5
:108A300008E100E080E100E084E100E088E100E09E
:108A400001403F0000003F80436A2DE9F0410546A8
:108A50000E469046002B3ED090F82C100124A140E9
:108A600083F83B1083F85E4083F85D40406A0368FA
:108A700000211B6808F1FF379847FFB2B8F1000FDB
:108A800023D03744A046013E686A16F8011F0368E8
:108A90001B6898470134B742E4B216D0202CF3D1BA
:108AA0000121686AFFF714FB95F82C206B6A5200CD
:108AB00083F83B2083F85E8083F85D80686A0368F2
:108AC00000211B6898470124DEE7686A0121BDE8A0
:108AD000F041FFF7FDBAC26BC16C136823EA0103D2
:108AE00006EB080413604FF00048A6420ED02B6A34
:108AF00016F801EB63B11A68C2F82C80C2F834E0B2
:108B0000D36A002BFCDAA642936BF0D1BDE8F0816A
:108B1000AB6BD5F834C008208021DCF800206F6CE6
:108B20001EEA010F14BF3A43BA43CCF800201A687A
:108B3000AF6C3A431A601A68AF6C013822EA070238
:108B40004FEA51011A60E8D1CFE700BF70B5044683
:108B5000406A0D46002828D0616DFFF757F920467E
:108B60002946FFF7A9FE606A20B1A16DBDE87040FB
:108B7000FFF74CB9216C226D0868236A02430A6032
:108B800093B1DA7A82B1D00703D5234A996911608B
:108B9000DA7A910703D5214AD9691160DA7A520746
:108BA00002D51F4A1B6A136070BD236A002B2BD0AD
:108BB000D97A226EE1B172B6D97ACE0706D51948B4
:108BC000D9680668314099610160D97A880706D56D
:108BD0001548196906683140D9610160D97A4E0794
:108BE00005D512485969066831401962016062B6BC
:108BF0001B68D968914207D00D4818600D49DA60AA
:108C000042F0804018611960226C216D136823EADC
:108C100001031360A3E700BF00E100E004E100E00E
:108C200008E100E080E100E084E100E088E100E0AC
:108C300001403F0000003F802DE9F041044686B02E
:108C4000806A9DF830801E460F461546B4F90830FC
:108C5000002800F04B81DA1D48BF03F10E02B4F981
:108C60000630D21003FB02F2002105F0A1FCB4F99A
:108C70000820202A00F3A780B4F90610A74B012092
:108C8000203A733902EBD27201EBD1714FF0200E12
:108C9000029073208DE8014042F34F0241F34F01EF
:108CA000204600F04DFE606A84F82D70002800F028
:108CB0005181002D40F09F80B4F90830202B14BF63
:108CC0003D253C2584F82C50B8F1000F40F09A80E7
:108CD00006B394F93300002818DBC0B2012101F07B
:108CE000ADFE012194F8330001F094FE012001F063
:108CF000CDFE002194F8330001F08CFE0A2001F033
:108D0000C5FE012194F8330001F084FE606A00285A
:108D100000F09880616DFFF779F8042280492046C1
:108D2000FFF792FE217A0139C9B22046FFF7C4FD50
:108D30007C4904222046FFF787FE94F92D30012B51
:108D400014BF142110212046FFF7B6FD04227649F6
:108D50002046FFF779FEB4F906308F22802B84F885
:108D60005C2000F0A580602B00F0B1800225DA21A4
:108D70002046FFF7A1FD29462046FFF79DFD8121F2
:108D80002046FFF799FD94F85C102046FFF794FD0C
:108D9000D9212046FFF790FD94F92D30012B14BF07
:108DA000F12122212046FFF787FD204606225F4958
:108DB000FFF74AFE606A58B3A16DFFF727F801205C
:108DC00006B0BDE8F081B4F90610594B0120403AD5
:108DD00052394FF0400E029002EBD272522001EB5A
:108DE000D1718DE8014042F34F0241F34F0120461B
:108DF00000F0A6FD57E76DB284F82C50B8F1000FD3
:108E00003FF466AFFEF7B8FF002E3FF47FAF60E798
:108E1000216C226D0868236A02430A6073B1DA7A12
:108E200062B1D00703D5434A99691160DA7A910794
:108E30006FD4520702D5404A1B6A1360012006B066
:108E4000BDE8F081236A002B2BD0D97A226EE1B1E4
:108E500072B6D97ACF0706D53848D968056829404F
:108E600099610160D97A8E0706D535481969056878
:108E70002940D9610160D97A4D0705D53148596932
:108E8000056829401962016062B61B68D968914281
:108E900007D02D4818602D49DA6042F080401861F3
:108EA0001960226C216D136823EA0103136034E713
:108EB000B4F90830402B7FF459AF94F92D30012BD1
:108EC00014BFCF239F2384F85C3012254FE7B4F9F9
:108ED0000830102B7FF44AAF94F92D30012B14BFCA
:108EE000AF23102384F85C30022540E7DA1D48BF29
:108EF00003F10E02B4F90630D21003FB02F2104661
:108F0000059205F029F8A06200283FF459AF059AB0
:108F1000AAE60F4AD9691160DA7A8AE7E00101000E
:108F2000C0030100C4030100C8030100CC03010019
:108F3000D403010000E100E008E100E080E100E08E
:108F400084E100E088E100E001403F0000003F8054
:108F500004E100E0012194F83100214F01F06EFDA1
:108F600094F83200012101F069FD94F9312094F95F
:108F7000323057F83220E26357F83330206A2364E6
:108F80000125E56425651A682A431A6048B1B8F1DD
:108F9000000F3FF439AFFFF75FFB002E3FF4B6AE92
:108FA00097E6294694F82F0001F048FD294694F8E9
:108FB000300001F043FD94F92F2094F9303057F838
:108FC0003220626357F833306564A5641A68A3637E
:108FD00022F001021A60002E3FF498AE79E600BF3D
:108FE000280C0100B0F90820D31D48BF02F10E0380
:108FF000B0F90620806ADB1002FB03F2002105F0C5
:10900000D7BA00BFF0B50029BDF814502EDBB0F977
:109010000660B1422ADA002A59DBB0F9087014461A
:109020001C44BC42C4BFBB1A1BB2002B1EDDD2B213
:10903000D408D0F828E016FB041112F00702DBB2C6
:109040000EEB010421D0C2F10807FAB2374F934268
:10905000BF5C0CD2C3EB020CFF2646FA0CF6012DC6
:1090600007EA06073FD005D3022D36D0F0BD012D0B
:1090700039D030D21EF8016026EA07070EF80170D9
:109080009342F3D3B0F906100C449A1AD2B2072ACD
:1090900010D9022D36D0002D14BFFF26002613460E
:1090A0002670083BB0F90610DBB2072B0C44F7D84A
:1090B00002F00702002AD9D01D4B012D9B5C1DD068
:1090C00017D3022DD2D1227853402370F0BD134420
:1090D0001BB20022A1E7022D25D11EF801607740C6
:1090E0000EF80170CCE71EF8016037430EF80170EE
:1090F000C6E7227822EA03032370F0BD22781343E7
:109100002370F0BD11462378DB4323700839B0F992
:109110000630C9B207291C44F5D812F00702A5D0C1
:10912000034B9B5CCFE73444AFE700BF80010100F5
:109130007001010070B4047EBDF80C50022C18D0F0
:10914000032C1FD0012C0BD0002A03DBB0F9084000
:10915000944201DC70BC7047039570BCFFF7BCBA49
:10916000C4880395013CA41A0A4621B270BCFFF7DB
:1091700049BF0689C488013E641AB21AE41A12B2C1
:1091800021B2E1E704890395E41A641A114622B278
:1091900070BCFFF737BF00BF70B4057EBDF80C6030
:1091A000022D1AD0032D12D0012D03D0039670BCCE
:1091B000FFF728BFC488E41AA41A0A4621B2002A7D
:1091C00003DBB0F90840944213DC70BC704704899B
:1091D000013C641A114622B2F1E7C488058903965E
:1091E000013CAD1AED1A621A11B22AB270BCFFF737
:1091F00009BF039670BCFFF76FBA00BF2DE9F843B3
:109200000446406A002863D0616DFEF7FFFD052229
:1092100074492046FFF718FCA1790139C9B22046EC
:10922000FFF74AFBB4F90820E588A66AD31D48BFBA
:1092300002F10E03DB10626A15FB03F51FFA85F8D5
:10924000002A7BD094F82C300125AB4082F83B30CB
:1092500082F85E5082F85D50606A036840211B68A6
:1092600008F1FF379847BFB2B8F1000F23D0374459
:10927000A846013E606A16F8011F03681B689847FC
:109280000135B742EDB216D0202DF3D10121606A2D
:10929000FEF71EFF94F82C20636A520083F83B20EF
:1092A00083F85E8083F85D80606A036840211B68F4
:1092B00098470125DEE70121606AFEF709FF606A31
:1092C000002800F08D80A16DBDE8F843FEF79EBD3B
:1092D000236A002B2BD0D97A226EE1B172B6D97AEB
:1092E000CE0706D54048D9680568294099610160D4
:1092F000D97A8D0706D53D48196905682940D96195
:109300000160D97A480705D5394859690568294067
:109310001962016062B61B68D968914207D035486E
:1093200018603549DA6042F0804018611960226C9B
:10933000216D136823EA0103136068E7E26BE36CB5
:109340001168276A0B4306EB080913604FF0004EC3
:109350004E450DD016F801CB2FB33A68C2F82CE079
:10936000C2F834C0D36A002BFCDA4E45936BF1D1BE
:10937000226C236D11680B43136097B1FB7A83B1A4
:10938000D90703D51D4BBA691A60FB7A9A0703D532
:109390001B4BFA691A60FB7A5B0702D5194B3A6AD4
:1093A0001A60BDE8F883A36BD4F8348008208021CC
:1093B000D8F80020656C1CEA010F14BF2A43AA43A9
:1093C000C8F800201A68A56C2A431A601A68A56CB0
:1093D000013822EA05024FEA51011A60E8D1B7E7E5
:1093E000276AC5E77801010080E100E084E100E040
:1093F00088E100E001403F0000003F8000E100E024
:1094000004E100E008E100E02DE9F04F85B0994665
:10941000BDF93870BDF83CA0BB1AC1EB090B002B9D
:10942000B8BF5B42BBF1000FB8BFCBF1000B5B458F
:109430000D4616460093804648DC4D453A46334675
:109440004CDC194613460A46C5EB09019B1A89B242
:10945000002B0CB2B8BF5B4204EBD474BE42ACBF6D
:109460004FF0FF3201224D45039102924FEA64040E
:1094700029DC9BB201930DE0D8F80070BF69B847B2
:10948000019BE41AA3B21CB20135002C2DB211DBF2
:10949000A94518DB009B5B452A46534631464046AA
:1094A000EADCD8F800205346976929463246404600
:1094B000B847E5E7029A1644039AA94502EB03046C
:1094C00036B224B2E6DA05B0BDE8F08F4A462B4644
:1094D000B94635464D4517461E46B2DD304629464B
:1094E0003E464D4607468946AEE700BF10B40468C5
:1094F0002469A44610BC604730B40468BDF8085025
:109500000295A46BA44630BC604700BF30B4046829
:10951000BDF808500295E46BA44630BC604700BF1C
:1095200070B40468BDF90C60BDF810500396049542
:10953000246CA44670BC6047704700BF10B582B071
:10954000B0F90C2001910168009200220C6CB0F976
:109550000A301146A04702B010BD00BF704700BFDF
:1095600001F003010129017606D0032904D0C28845
:1095700003894281838170470289C3884281838144
:10958000704700BF2DE9F0410568134E6F6986B042
:10959000B7420446BDF8308010D1013B13441BB2E2
:1095A0000093CDF804800B46AD6A2046A847236897
:1095B000DB6AB3420AD106B0BDE8F081059304929C
:1095C0000391B84703A925680EC9E6E7204606B00F
:1095D000BDE8F041184700BF399500002DE9F04182
:1095E0000568124E6F6986B0B7420446BDF83080F8
:1095F0000FD1013BCDF804800B4400921BB2AD6A41
:109600002046A8472368DB6AB3420AD106B0BDE80A
:10961000F081059304920391B84703A925680EC908
:10962000E7E7204606B0BDE8F0411847399500004D
:109630002DE9F04F0568DFF858B06F6985B05F45D8
:109640000646BDF93890BDF83CA00C46904615D1B1
:109650001F19BC420CDACDF800A0214601342D6A56
:109660004B464246304624B2A847BC423568F2DB3E
:10967000EB6A5B4507D105B0BDE8F08F0393B847AF
:109680003568039BE4E7304605B0BDE8F04F184766
:10969000399500002DE9F04387B099420546BDF9A0
:1096A0003840BDF83C6025D0A24212D00768DFF8F0
:1096B0008080D7F81490C14532D18DE850002846FB
:1096C000BC6AA0472B68DB6A434524D107B0BDE8DC
:1096D000F083994202DD08461946034628680E9633
:1096E000C46B01335B1A1BB22846A44607B0BDE821
:1096F000F0436047A24202DD134622461C4628681A
:109700000E96631C846B9B1A1BB22846A44607B0B6
:10971000BDE8F0436047284607B0BDE8F04318476E
:10972000059304920391C84703A92F680EC9C4E7A3
:10973000399500002DE9F04FD0F800E0DFF8909067
:10974000DEF814B083B0CB450446BDF93080BDF8D7
:1097500034A00D4617461E4631D1CDF800A0DEF8E4
:1097600024B0294633463A462046D8472368CDF8E8
:1097700000A008F1FF323A44D3F824B0294612B2CF
:1097800033462046D8472368CDF800A02946D3F8B1
:1097900020B03A4643462046D8472068CDF800A07E
:1097A000711E29444346056A09B23A462046A84735
:1097B0002368DB6A4B4506D103B0BDE8F08FD8477C
:1097C000D4F800E0C9E7204603B0BDE8F04F1847E1
:1097D00039950000F0B4002401254FF6FF76094FBB
:1097E000076004710476C48104828476C461C575FF
:1097F0008575457686824682C1800281418182815B
:10980000F0BC70479C0601002DE9F04F85B006685A
:10981000BDF84450BDF93880CDF80080044601956C
:10982000D6F848B00392BDF93C60BDF94070894656
:109830009A46D84723680195009742465146D3F887
:10984000488020463346C0472068039B0E930F95FF
:10985000856C4B463A4631462046AC4605B0BDE8DD
:10986000F04F60472DE9F04F87B01746BDF94040F3
:1098700000912546E91D059344BF2B4603F10E01D7
:109880000268BDF8486053690294C91003912B49DE
:10989000BDF9444001968B42824645D1002C3CDD07
:1098A000029B3C445E1EB6B24FF0000923B2049303
:1098B00001364D46029B002B28DD059B002403EB5F
:1098C000090806E0EDB22B0604F1010411D4A6420A
:1098D0001CD0A1B211F0070F23B24FEA4505F1D118
:1098E000002BB8BF0733DB10013418F803502B06E8
:1098F000EDD5009BD2F818B019443A4609B2019B45
:109900005046D847A642DAF80020E2D1039B01373F
:109910009944049B3FB2BB42CCD1D36A074A9342DD
:1099200006D107B0BDE8F08F9847DAF80020B5E718
:10993000504607B0BDE8F04F184700BF399500000A
:1099400070B4BDF90C60BDF91050BDF81440039619
:109950000495059470BCFFF785BF00BF2DE9F04F5B
:1099600091B083460591C169BDF8680006909DF8E5
:109970007400BDF86C709DF870A003900292994637
:10998000002900F0CC800B7A48680A68C3EB090311
:10999000DBB2154600EBC30230F83360D37809938D
:1099A000BAF1010F92F9053092F802800E9392F904
:1099B000064079D9BDF93830089323B20B93A94BEF
:1099C000DBF800200F93194653698B4240F0A280C8
:1099D000099B002B53D0BDF808300C930021234481
:1099E00007910D930F460C46A946B8F1000F3FD0E2
:1099F000BDF81C100B9BBDF80C000297CB1813FB95
:109A000000F30C9803440D981BB2014404930BB26D
:109A10000A93002505E00135EBB264009845E4B2F5
:109A200023D9029B2B44590703D1731C19F8064014
:109A30009EB22306EFD5089BE918059B11FB0AF19E
:109A4000BAF1010F194402D1039B012B1ED0069BD2
:109A50000193039B0093D369049A1F4609B25346AE
:109A60005846B847DBF80020D5E7029F4744FFB2CD
:109A7000079B099901330793DBB29942B5D8D36AA2
:109A80000F9A934241D111B0BDE8F08F0E9B05991A
:109A9000591893690A9A29441F4609B2069B5846E9
:109AA000B847DBF80020B6E7039B012B82D80023E0
:109AB0000B93089383E70799099A0131013A49B258
:109AC00012F0FF020791099260D1069A4A454F466B
:109AD00017D0BAF1010F03D1039A012A00F0B58023
:109AE0000A9A089802EB8201039AD2008DE884005A
:109AF000084401B2DC69029A53465846A047DBF895
:109B00000030DB6A0F9A9342BDD0584611B0BDE8D1
:109B1000F04F184758469847DBF8002058E7BBF944
:109B20000A3005998B42AEDDBBF90C3002988342B6
:109B3000A9DD062313FB0A13002BA4DD039B00EB16
:109B4000C303002B9FDD9BF81A3033B9B9F1AF0F77
:109B500084BF09F101035FFA83F9424ADBF8003060
:109B60000F9211465A698A426AD1BDF814200892B0
:109B700005220992002207921FFA8AF20A92CDF872
:109B800030900FFA8AF2B946039F05920799BDF803
:109B90003040089D0522104610FB04120A98324CF2
:109BA0000646084601FB0651A65C15FA80F209B28A
:109BB00012B204910B92082400251CE0BAF1010FA7
:109BC00001D1012F24D0069A0192029A009705FB39
:109BD0000722D3F81C800499059B12B25846C0474F
:109BE000DBF80030013C013514F0FF046DB24FEAA0
:109BF00056063FF460AFF007E0D4069A4A45F1D02C
:109C0000BAF1010F01D1012F0ED0CDF80490DCE79D
:109C1000029AD3F818800B99069BAA1812B25846DC
:109C2000C047DBF80030DDE7029AD3F818800B99C3
:109C3000AA184B4612B25846C047DBF80030D1E7AD
:109C400058469047DBF800308FE70899CDF8009030
:109C500005311C6A029A082309B25846A047DBF86E
:109C600000304EE739950000EC060100F0B5C369FD
:109C700085B004463BB30A296FD00D294FD01A7A1C
:109C800091424CD3587A884249D38A1A5D68D2B23D
:109C900005EBC205AA78002A56D0E878002853D0F0
:109CA000607E00283ED095F905E0B4F90E00A67D4F
:109CB000B4F90A70724406FB0202BA4269DCE77D1D
:109CC000B4F9102034E00A295CD00D2927D0427E57
:109CD000002A50D0B0F90E00A57DB4F90A60062222
:109CE00012FB0502B242E67D42DD228AE38102EBED
:109CF000C60212B218462282B4F814E0678A0396AC
:109D00000B46029501468DE880402046FFF726FE6F
:109D1000A37DE28903EB430302EB4303E3810120CC
:109D200005B0F0BDA67DE77DB4F90E00B4F91020B2
:109D3000B4F814E00397678A02960B468DE88040DA
:109D400001462046FFF70AFE2979E389A27D01201A
:109D500001FB0233E38105B0F0BD0022C2819A7A93
:109D6000C17D038A01FB02330382012005B0F0BDEF
:109D7000B4F91020C0E7857DC67DB4F91020B0F994
:109D80000E00B9E7028AC17DC38102EBC1030382E1
:109D9000C5E70020E0819B7A228AE77D03FB07224A
:109DA00012B22282C4E700BF11B18175C17570473C
:109DB00001218175C1757047844641EA000313F0A3
:109DC00003036DD1403A41D351F8043B40F8043BC2
:109DD00051F8043B40F8043B51F8043B40F8043B85
:109DE00051F8043B40F8043B51F8043B40F8043B75
:109DF00051F8043B40F8043B51F8043B40F8043B65
:109E000051F8043B40F8043B51F8043B40F8043B54
:109E100051F8043B40F8043B51F8043B40F8043B44
:109E200051F8043B40F8043B51F8043B40F8043B34
:109E300051F8043B40F8043B51F8043B40F8043B24
:109E400051F8043B40F8043B403ABDD2303211D3C4
:109E500051F8043B40F8043B51F8043B40F8043B04
:109E600051F8043B40F8043B51F8043B40F8043BF4
:109E7000103AEDD20C3205D351F8043B40F8043BC4
:109E8000043AF9D2043208D0D2071CBF11F8013BC2
:109E900000F8013B01D30B8803806046704700BF88
:109EA000082A13D38B078DD010F003038AD0C3F197
:109EB0000403D21ADB071CBF11F8013B00F8013B79
:109EC00080D331F8023B20F8023B7BE7043AD9D338
:109ED000013A11F8013B00F8013BF9D20B7803700D
:109EE0004B7843708B78837060467047374A3849A7
:109EF00013681B06FCD40B6813F08003F8D172B60C
:109F000034490A78002A5FD0334A3448F0B4344CDC
:109F1000176806682568D4680C303E44143200681F
:109F20001268304F35442C4420440244C2F34E02A0
:109F30002D4E2E482E4D2F4C42F400423A60376889
:109F400006682D682C4A24680C303E44006812686C
:109F50002A4F35442C4420440244C2F34E02284E7A
:109F60002848294D294C42F400423A603768066877
:109F70002D68274A24680C303E4400681268254F3B
:109F800035442C4420440244C2F34E02224E23485E
:109F9000234D244C42F400423A60376806682D682D
:109FA000214A24680C303E440068126835442C4431
:109FB00020440244C2F34E021C4842F400420260B4
:109FC0000B7062B6F0BC704762B6704724B00340B5
:109FD00024B00B408E9EFF1F38B003403CB00340BE
:109FE00040B003402CB0034058B003405CB0034085
:109FF00060B0034064B003406CB0034030B0034035
:10A0000038B00B403CB00B4040B00B4044B00B406C
:10A010004CB00B402CB00B4058B00B405CB00B4028
:10A0200060B00B4064B00B406CB00B4030B00B40E4
:10A0300030B42948294A2A4B2A4D6024E121047072
:10A0400011701B78284C082B30D00A2B2748284940
:10A0500037D00C2B0CBF35223D2212232A602360FF
:10A0600002600B60234B24491B78244ABBB10123B7
:10A070000B601360224B23491B78234A012B26D9FE
:10A08000042B0FD9082B1ED9102B94BF86238723AE
:10A090000B6013601D4B01221A7030BC70470B60BF
:10A0A0001360E7E784230B601360F3E700F58E206D
:10A0B0000F490830012213232A60236002600B60DD
:10A0C000D0E73922F7E785230B601360E2E78023AE
:10A0D0000B601360DEE700BF00400740014007400F
:10A0E000FC90FF1F08B003400CB0034008B00B40C9
:10A0F0000CB00B40919EFF1F20B0034020B00B40DE
:10A10000FD90FF1F24B0034024B00B408E9EFF1F24
:10A110000C2830B417D91023984228BF18461C4683
:10A12000104A114D1178181A8C42287018D00F4916
:10A1300013700B7823B10E490E4A00230B60136095
:10A1400030BCFFF775BF0A2802D90C231C46E7E78D
:10A15000082802D90A231C46E2E708231C46DFE749
:10A1600030BC7047FC90FF1F8D9EFF1F8E9EFF1F0F
:10A1700024B0034024B00B4028282FD8334B2DE9BE
:10A18000F0411E5CFF2E2BD0314B1B78002B2AD1C7
:10A1900032062CD472B62F4D2F4C2F460123266049
:10A1A0002B7062B672B623681B060CD43B781BB9C1
:10A1B000F4E72B78002BF1D062B602F0CBFA72B63E
:10A1C00023681806F5D5254B1B6800222A7062B655
:10A1D000234A107843FA00F0BDE8F0810020704770
:10A1E0000020BDE8F081FFF781FE3206D2D572B6BD
:10A1F0001C4DDFF87C801C4C06F04007FFB206F0D7
:10A200003F06D8F80030DFB123F01003C8F8003063
:10A2100001232660134A2B7062B672B623681906B2
:10A220000CD413781BB9ECE72B78002BE9D062B67D
:10A2300002F090FA72B623681B06F5D50B4BC3E704
:10A2400043F01003C8F80030E2E700BFEC0B010058
:10A250008E9EFF1F909EFF1F00B0034010B0034072
:10A260008D9EFF1F8F9EFF1F00B00B4010B00B4054
:10A270000CB00B400A4A0B49136843F48053136037
:10A280000B7843B9084BC0221A70084B80F30C00BE
:10A2900000B218807047044B80221A70F5E700BFA7
:10A2A0002C800440919EFF1F21C00C4000C00C4038
:10A2B000F0B51B4B1B4E596818689A68DB6885B06F
:10A2C0006C460FC4337899071DD5174A174C13787D
:10A2D000174913F0700318BF1370164A164B8027E6
:10A2E000177000263320032226706D4608701A70FE
:10A2F00072B6043C45F001052046A84762B62378B3
:10A3000013F0700309D10D4B064901E0013B02D067
:10A310000A78D207FAD505B0F0BD237005B0F0BDBC
:10A32000180C01000100024000000240040002403D
:10A330000B000240070002400A000240410D0300EA
:10A34000B0F5006F0AD210B5094B1B78DB07044645
:10A3500006D504F1A0500078C0B210BD00207047AF
:10A36000FFF7A6FF04F1A0500078C0B210BD00BFF7
:10A3700001000240B0F5006F17D238B50F4B1B78C3
:10A38000DA070D46044611D504F1A0500378AB421C
:10A390000AD00B4A137813F0700318BF1370074AE2
:10A3A00005701378DB07FCD538BD7047FFF780FFD9
:10A3B00004F1A0500378AB42EBD1F5E70100024075
:10A3C0000000024008B5104C08E0236859050DD480
:10A3D00023681A050FD42368DB0411D423685803BB
:10A3E000F3D500F067FE23685905F1D502F036FA7F
:10A3F00023681A05EFD502F0C7FA2368DB04EDD510
:10A4000000F0CAFCEAE700BF3480044008B5FFF75B
:10A41000D9FF00BF014B10221A8070470020054071
:10A42000704700BF094908B50B6830B16A46184447
:10A43000A2F58052904202D20860184608BD03F08F
:10A440005DFD0C2303604FF0FF3008BD0091FF1F3E
:10A45000FEE700BFEFF3138070B9EFF310836BB921
:10A46000EFF305825AB94FF48070EFF311832BB1EB
:10A47000984228BF184670474FF0FF3070470F2AA8
:10A4800001D81846F1E7014BD05CEEE7F0E300E0BD
:10A49000704700BF10B40F4B53F8302092F8804241
:10A4A0002CB1012369B182F8803010BC704703EBF6
:10A4B000C0035B681A6841B922F002021A6010BC3E
:10A4C000704782F8003110BC704742F003021A60F6
:10A4D00010BC7047280C01001C4A02EBC003012984
:10A4E0005B6811D004291BD052F83000002280F89C
:10A4F000802229B1022920D0032922D01A60704776
:10A500004FF480721A60704752F830004FF4A27214
:10A5100080F880121A601A6822F020021A607047D0
:10A5200052F830104FF4A272012081F880021A60B4
:10A530001A6842F020021A60704740F203121A6053
:10A5400070474FF481721A60704700BF280C0100F9
:10A55000212848D8F8B5042A44D8DFE802F0484B4F
:10A560004E0345004FF410262B4B03EBC0030D4662
:10A570005C68216811F4E06148D0284B284A2949D9
:10A58000C3F89C2104F140422748C3F8A411A2F566
:10A590009221264FC3F8A0017C292548C3F8A87151
:10A5A000C3F8AC012CD9A2F594237C2B2AD9A2F5AF
:10A5B00096237C2B28D9A2F598237C2B29D9A2F5A8
:10A5C0009A227C2A27D81B4872B6236823F470236A
:10A5D00043F08072C4F384011643236040F8215095
:10A5E000266062B6F8BD70474FF43026BCE74FF4E2
:10A5F0000026B9E74FF44026B6E74FF42026B3E72C
:10A600000D48E1E70D48DFE70D48DDE7FFF764FFA0
:10A61000B3E70C48D8E7F8BD280C01000082FF1F03
:10A62000F188FF1F9988FF1FC588FF1F6D88FF1FD6
:10A630004188FF1FDC91FF1F0491FF1F3C91FF1F0A
:10A640008C91FF1FBC91FF1F1A4B03EBC00010B48D
:10A65000426802F14043A3F592217C2923D9A3F556
:10A6600094217C290DD9A3F596217C291FD9A3F526
:10A6700098217C2919D9A3F59A237C2B11D80E4C4B
:10A6800000E00E4C72B613680D4823F08773C2F3D6
:10A69000840123F4803343F08073136044F8210075
:10A6A00062B610BC7047074CECE7074CEAE7074C72
:10A6B000E8E700BF280C0100DC91FF1F3C91FF1F61
:10A6C00091A400000491FF1FBC91FF1F8C91FF1FFC
:10A6D00030B4054B054D064C002210211A602A604B
:10A6E0002060196030BC704714D0034004D0034090
:10A6F00000D00340282838B52ED0002904464FDD6D
:10A700005F4B1B78012505FA03F28A4202D8212803
:10A7100037D938BD0338C2B2012A3AD9202C4AD0E1
:10A72000192C48D0574A126802FB011222FA03F38F
:10A730001D2800F29B80DFE800F0928B847D9999C0
:10A74000766F99999999999999999968615A5399B4
:10A750004C99999999999945494B1B780B2B08D994
:10A760000C2B1CBF0C3B19410846BDE83840FFF7D5
:10A7700081BDC3F10C0399400846BDE83840FFF79E
:10A7800079BD2946FFF786FE2946BDE83840FFF728
:10A79000A3BE3D4A126802FB011222FA03F3C7E787
:10A7A0002128B6D80021FFF775FE20460121BDE81B
:10A7B0003840FFF791BE354A126802FB011222FAB7
:10A7C00003F3B5E73249334A0B604FF4517313601A
:10A7D00038BD3149314A0B604FF45173136038BDB5
:10A7E0002F49304A0B6040F24443136038BD2E4974
:10A7F0002E4A0B6040F24443136038BD2C492D4A69
:10A800000B6040F24443136038BD2B492B4A0B6068
:10A8100040F24443136038BD29492A4A0B6040F294
:10A820004443136038BD2849284A0B6040F2444332
:10A83000136038BD2649274A0B6040F24443136039
:10A8400038BD2549254A0B6040F24443136038BDAA
:10A850002349244A0B604FF45173136038BD2249D9
:10A86000224A0B604FF45173136038BD212C3FF620
:10A8700050AF7F29D4BF00210121204693E700BFBC
:10A88000E491FF1F088003400890034008800B40BC
:10A8900010800B4048A0044018800B404CA004409E
:10A8A0001880034008B004401080034004B0044006
:10A8B0004080034018C004403880034014C0044066
:10A8C0002880034010B00440208003400CB00440B6
:10A8D0003080034010C00440488003401CC0044046
:10A8E000189003403490044010900340309004408E
:10A8F00038B1102828BF1020044AC3B21078137052
:10A900007047024A0123107813707047E491FF1FCB
:10A910002DE9F8430E4680463249334D304603F068
:10A9200073FA47F6122300281ABF1D464FF002099A
:10A930004FF00109002425FA04F003F06FF84FF0FE
:10A940005E51074603F0C2F80146304603F070FA44
:10A9500030B90134072CEED1E80903F05FF807465F
:10A960003146384603F066F94FF07C5102F0A4FFFF
:10A9700003F098FA4FF6FF729042A8F1030328BF44
:10A980001046012B29D9B8F1170F17D8174B23FA06
:10A9900008F303F0010383F0010223B9B8F1190FA2
:10A9A0000FD0BDE8F883124B124D13491A6044EAE8
:10A9B000C9042A6008601C60BDE8F883B8F1200F64
:10A9C000ECD10E4B0E4D0F49002244EAC9041A6027
:10A9D0002A6008601C60BDE8F8830B4B0B4D0C49E6
:10A9E000F2E700BF001BB740006CDC026006F0001D
:10A9F00000800340048003400880034000800B4037
:10AA000004800B4008800B400090034004900340FA
:10AA100008900340212801D8FFF73CBD704700BFD4
:10AA2000212806D8044B53F8303093F80002C0B206
:10AA300070470020704700BF280C0100212801D872
:10AA4000FFF74ABD704700BF72B60C490C4B0D4A68
:10AA50001B680868126862B6520102D5322B88BFA3
:10AA600001300949C3F5BB334FF47A72FF33A1FBC0
:10AA7000031302FB00F000EB93107047949EFF1F3E
:10AA800018E000E004ED00E0ABAAAAAA2DE9F84323
:10AA9000054672B6204F214B214A1B683C6812685C
:10AAA00062B6520102D5322B88BF013495B3C3F58B
:10AAB000BB331C4EDFF86490DFF86480FF334FF443
:10AAC0007A72A6FB031302FB04F404EB931472B630
:10AAD000D9F800103A68D8F800E062B6C1F5BB3387
:10AAE000FF33A6FB03031EF0806FC4EB93134FF4F8
:10AAF0007A7002D0322988BF013200FB0233B3F5ED
:10AB00007A7F04D3013D05D004F57A74DFE701F0C4
:10AB100021FEDCE7BDE8F883949EFF1F18E000E00B
:10AB200004ED00E0ABAAAAAAF8B52D4B2D49DFF839
:10AB3000D0E0DFF8D0C02C4E2C4D2D4C2D4A2E4F9E
:10AB40004FF4000018604FF0807018604FF00070F4
:10AB500018604FF0806018604FF0006018600020AF
:10AB6000086028234BF6FF71CCF80010CEF80030B7
:10AB7000336013602B6023603B60B36293620922F1
:10AB800045F8242CC4F8D80F05F57F65C7F8D41F05
:10AB900007F5FF2707F5FA67C6F8F83F2B6006F5BB
:10ABA000FF26C4F8D42F05F5FD2504F5FF243860F1
:10ABB00006F2F4761148316005F5FF6504F5FD6491
:10ABC0002B6023600260FFF733FA1920FFF75EFF66
:10ABD00000F0B6FF40F21310BDE8F840FFF756BF93
:10ABE00008E100E004800340148003402480034017
:10ABF0002C8003401C8003403480034000800B40C5
:10AC00000C800340088003402DE9F84F214B1B685E
:10AC100007460BB101221A70DFF888901E4D99F893
:10AC20000040DFF884801D4E0134272C8ABF4FF08E
:10AC3000000A5FFA84FA5446AB462B78A34216D139
:10AC4000FFF708FC40281FDC33791B06F5D59BF87D
:10AC500000300133272B86BF00221346DAB218F8E2
:10AC60000330DBB2F3712A702B78A342E8D00C4991
:10AC70000A4BFFB208F804700120AC22087089F872
:10AC800000A0DA70BDE8F88FFF28D6DD01F062FD84
:10AC9000D3E700BF0C9FFF1F099FFF1F00C00640A6
:10ACA000089FFF1F109FFF1FA09EFF1F1C4BDFF878
:10ACB00094C01A681B49F0B542F480521A4D1A60CC
:10ACC000DFF884E0194F1A4E1A4C00238CF800303C
:10ACD0004FF451722B701F2840F213358EF800305C
:10ACE0003B70337025600A6012D819460124124A5D
:10ACF000124D11701248547000212C274026937277
:10AD00004FF4003491701174D7702E700460F0BD50
:10AD1000C0F34431C0F3471400F01F03E7E700BF5E
:10AD2000348004400CC004409D9EFF1F099FFF1FFC
:10AD3000089FFF1F08C0044000C0064031E400E047
:10AD400004E100E09C9EFF1F109FFF1F034B1B6848
:10AD5000DB0401D5FFF758BF704700BF34800440C3
:10AD600010B5044C237823B101F0F4FC2378002BB8
:10AD7000FAD110BD089FFF1F054A064B10781B78BB
:10AD8000C0B2DBB2984238BF4030C01A704700BF33
:10AD90009C9EFF1F9D9EFF1F30B42B4B1A7994067B
:10ADA0001FD52A48DA790378294901333F2B0978DE
:10ADB000C8BF00238B42D2B203D0264CD9B2E25492
:10ADC0000170254A116861B1244A1278D2B29342C7
:10ADD00036BFC2F140029B1A9B18272BC4BF012328
:10ADE0000B70194AD378DBB2180611D45A060DD568
:10ADF000154B1B795B0609D5194B1A491B680022B4
:10AE00000A7003B11A70104B2C22DA7030BC7047F4
:10AE100011790906EAD5144910480C780178C9B2AD
:10AE20008C420DD04A1C272A84BF00210A460F4DB0
:10AE3000054C98BFD1B2AA5CD2B2E2710170D5E7DD
:10AE40006C21D170D2E700BF00C006409C9EFF1F5E
:10AE50009D9EFF1FC89EFF1F989EFF1F099FFF1FFB
:10AE60000C9FFF1F089FFF1F109FFF1FA09EFF1F2B
:10AE700021282FD8184B195CFF292BD0174B184AC3
:10AE8000DFF870C003EBC000F0B54368DFF868E09E
:10AE9000144F154D154E00241C60DEF800300120C3
:10AEA00043F020038840CEF8003014604FF4A073C4
:10AEB00038602E60C2F800C0013BFDD113689B05CD
:10AEC000FCD42023013BFDD1094B09B233F811001A
:10AED00080B2F0BD00207047380D0100280C010041
:10AEE0000050044008500440045004400000020395
:10AEF0000051044080014A0038800440431E032B67
:10AF000014D872B60A4951F8230068B170B4094CDC
:10AF1000058834F81320466841F82360521B24F852
:10AF2000132062B670BC704762B67047002070474D
:10AF30006C9FFF1FD0A1FF1F013803280BD872B6EA
:10AF4000074B53F8203043B100205B680130002BE1
:10AF5000FBD162B67047002070471846F9E700BF82
:10AF6000C09FFF1F30B472B62B4A13781D0706D559
:10AF70002A4B196A002936D0996A002941D05378A2
:10AF80001C0706D5254B196C00293ED0996C002969
:10AF900039D09378190705D5204B196E002936D082
:10AFA000996E89B1D3781B0707D51C4BD3F8802045
:10AFB0007AB3D3F8882011213AB162B6184B002237
:10AFC0001A7030BC00F048BE0D21154C154D22788A
:10AFD00043F8315003EBC1030830013A5860227046
:10AFE00062B630BC704704220D4C0F4D217843F8F7
:10AFF000325003EBC20308304A1E5860227062B61A
:10B00000EFE70521E1E70921DFE70822ECE70C2261
:10B01000EAE71022E8E700BF600D01000080FF1F93
:10B02000E99FFF1FC800400088004000431E032B1B
:10B030001DD81B4A400140F0100030B4104472B6D5
:10B04000184CE25C032A1BD8DFE802F00212151745
:10B0500003220D88E25410F0080F14BFC823882380
:10B0600043EA054308310360416062B630BC704773
:10B0700008300222EDE70522EBE708300422E8E77A
:10B08000094A52F8230038B1084A52F823004160B7
:10B0900042F8231062B6E9E742F82310034AF7E7C3
:10B0A0000080FF1FF89FFF1FC09FFF1FD09FFF1F43
:10B0B00000BE70472DE9F04FDFF818B3DFF818A392
:10B0C00087B044E0AD4F4FEA930807EBC809013E53
:10B0D000D9F8042003F00803F6B2A2F1080003F047
:10B0E000FF04002B40F0018157F838301B0C99B257
:10B0F00022F8081C002B00F0EF80A14B22F8064C30
:10B1000042F8044C53F82620002A00F0CF819D4DD0
:10B1100055F8263058609C4C45F8260034F8163017
:10B12000194424F8161000F077FD002800F0C281C1
:10B13000964A974B19F0080F00F1080018BF134604
:10B14000C9F8040047F8383008238BF800309BF822
:10B150000040E4B265071CD58E4B1B78B3B18E4915
:10B160000A7802F0FF0322B1013BDBB20B7003B996
:10B1700000BE8A490A7802F0FF032AB1013BDBB224
:10B180000B70002B00F0688100F064FE04238BF844
:10B19000003004F0080303F0FF02002B00F0C98028
:10B1A0009AF80030DBB21E098CD19A08DFF8CC91F6
:10B1B00059F8321009EBC200C1F38301013940682C
:10B1C0000C2900F28580DFE801F07A7A838383839B
:10B1D00083834683838307000168714D4068714F04
:10B1E000714E6860296088B240F281610024674B2B
:10B1F00049F832304FF0010E88423C60C9F81040E7
:10B20000C9F8184086F800E05C4A00F2E780B0F523
:10B21000D06F80F01B82B0F5817F00F0D98100F201
:10B220006981802800F02A82822840F0D781A9888D
:10B2300001F07F01042900F2D1815C485C4A890059
:10B2400008441470547001788C0740F1608382F8D0
:10B2500000E0022173E1534F3A682AB3554B524E36
:10B26000554819883478057840298E4645F00208FB
:10B2700028BF4FF0400E002C84F001043470CEEB58
:10B2800001010CBF8824C82409EBC80689B285F0E7
:10B29000010544EA0E447260198049F8384072444E
:10B2A0000570002965D03A603D4B1A88B2F5A06F51
:10B2B0000ED100219A785970404B1A7008E0384935
:10B2C0003F4C0D68A54200F09880304949F8321093
:10B2D0003C4A0123137037E72C4A2D4B19F0080F15
:10B2E00018BF134647F838302EE700F0B5FC364A51
:10B2F000364952F82630002B00F0E38058688C5D08
:10B3000042F8260003F10802C9F80420032C05D8EE
:10B31000DFE804F02C02292602228A551A8819F047
:10B32000080F0CBF8823C82343EA024347F838308C
:10B330000AE7E00700F19380210600F1D180A2071F
:10B3400006D5234A234913780220DBB21370087014
:10B35000E30602D51F4B10221A7007B0BDE8F08F2C
:10B3600004228A55DAE705228A55D7E703228A554F
:10B37000D4E7BEF1400F18BF002294E70080FF1F02
:10B380006C9FFF1F189FFF1FD0A1FF1FC800400028
:10B3900088004000F49FFF1F7D9FFF1F68A0FF1FD4
:10B3A000E09FFF1F149FFF1F7C9FFF1FC0200740CF
:10B3B000EC9FFF1F289FFF1FE89FFF1F982007405B
:10B3C0002109000394200740C09FFF1FF89FFF1F23
:10B3D000882007408020074090200740B0F5106F7C
:10B3E00000F07C8140F2A38040F62112904240F0B0
:10B3F0007B82A54A012313706AE74C68A3498C42FB
:10B400007FF463AF0178A9297FF45FAF41784529C4
:10B410007FF45BAF8178C2297FF457AFC1786B2985
:10B420007FF453AF9A489B4E0178347881F0010540
:10B43000002C41F0020105700CBF8820C82084F068
:10B44000010449F8310009EBC1019348347000252B
:10B4500005244D60047038E700F062FF94E68F4BDE
:10B4600089488B491A614FF0020E80F800E08C4F3A
:10B470000A708C49196099608B4E8C4D8C4C9A6186
:10B480000D213970FF213170DFF84CE229702270F4
:10B49000884D894A8EF800109F27012406F8047C05
:10B4A0005D600470DA6007B0BDE8F08F43F82600F5
:10B4B000824D30E6824A47F8380013780133137022
:10B4C00042E68B5D032B00F2BA8001A252F823F012
:10B4D00049B1000049B1000029B5000023B50000C2
:10B4E0006F49724B80220D2008701A70A2077FF5F9
:10B4F0002FAF26E740F20232904240F0ED81AA8859
:10B5000002F07F02042A69D86D88002D66D1644953
:10B51000CDF804E0920011440A7842F002020A7069
:10B52000C1E101238B550FE600238B550CE6B0F5E6
:10B53000086F53D16349644A097811707146ED88E8
:10B540008D4280F0E88252480478402DAE4644F0A7
:10B55000020C28BF4FF0400E02EB0E0309EBCC01AA
:10B56000029301234A604FEA0E48CEEB0501019396
:10B570000025C82242EA080384F0010249F83C3061
:10B5800035700270DFF814C1424BDFF8048149BB0B
:10B59000BEF1400F7FF42DAF42F0020C09EBCC035B
:10B5A000029ADFF8F8E05A608DBB0D0445F088057B
:10B5B0009DF804304EF83C500A4433700470134632
:10B5C00040297FF416AF0021404A3B60118010E70C
:10B5D000AA8802F07F02042A40F28B81304A0F23AE
:10B5E000137006E74029D7D942F002020CEBC200E3
:10B5F000029E4660BDB19DF8045035481D7033462B
:10B60000403988F8004040334CF83200DCE79DF8C0
:10B61000043033700D04029B047045F0C8050B44E0
:10B620004EF83C50CCE79DF804501D70029B1D481D
:10B6300088F80040403940334CF83200C4E719F034
:10B64000080F0CBF022303238B557DE521494A686F
:10B65000002AC3D06C88B5F804E003E00C314A68D6
:10B66000002ABBD00B88A342F8D14B887345F5D193
:10B67000240A032C0CBF1178098960E7124A0221C1
:10B68000147054705BE700BF942007400100040071
:10B69000E89FFF1F7C9FFF1F7D9FFF1F0080FF1FF4
:10B6A000C0200740880040008820074080200740D5
:10B6B000982007402C9FFF1F809FFF1F189FFF1F90
:10B6C000E99FFF1FF49FFF1FEC9FFF1F289FFF1F95
:10B6D000C8004000640D01008C200740B248116A88
:10B6E000AC7804700C0600F19881D9F82820AF4995
:10B6F000100600F1DB81D9F83020AC49120600F1C8
:10B70000D081D9F83820A949130600F1C581D9F8AC
:10B710004020A649150600F1BA81D9F84820A3496E
:10B72000140600F1AF81D9F85020A049100600F1AD
:10B73000A481D9F858209D49120600F19981D9F8C1
:10B7400060209A49130600F18E81D9F86820974944
:10B75000150600F18381D9F870209449140600F190
:10B760007881D9F878209149100600F16D81D9F8D7
:10B7700080208E49120600F16181D9F888208B491A
:10B78000130600F15581D9F890208849150600F17B
:10B790004981D9F898208549140600F1FF80844832
:10B7A000844A854901908548854D864C049700233D
:10B7B0000596029580460F4616461D46039430684E
:10B7C00028B1446800F048FA2046002CF9D1002343
:10B7D0003360029B38681A46002342F8253028B1AE
:10B7E000446800F039FA2046002CF9D100223A6072
:10B7F000019A98F800301146002241F8042B039A70
:10B800000191023B4FF0000122F81510032B07D8DD
:10B81000DFE803F05D025D024FF0010388F80030BD
:10B820000135042D06F1040607F1040708F10108AB
:10B83000C5D1654C654D2278654B049F059E00215E
:10B84000100729701A7000F19280624962780A70BC
:10B850000021C9F83010C9F838101107DFF84C8101
:10B860006ED4A2785C49DFF844810A700021120787
:10B87000C9F85010C9F858104BD4E27857494B4CCE
:10B880000A7013074FF00001C9F87010C9F878105A
:10B8900000F1AE8033780193002283F00105C9F8EE
:10B8A0009020C9F898200021029188468E460A46C9
:10B8B0004B48047844F0020C09EBCC030393019B42
:10B8C000002B039B5A600CBF8822C82252E64FF01F
:10B8D000000388F80030A3E7B0F5A06F7FF47EAED8
:10B8E000012300250193DEE740F621229042F7D0A4
:10B8F00074E66D88002D7FF471AE3A49CDF804E00E
:10B90000920011440A7822F002020A70CBE7022169
:10B9100015E600F081F9002800F0EB800830324A8B
:10B92000C8F86400C8F8602000F076F9002800F03C
:10B93000DA8008302D4AC9F86C00C9F868209CE705
:10B9400000F06AF9002800F0E0800830264AC8F8C4
:10B950004400C8F8402000F05FF9002800F0CF80D4
:10B960000830224AC9F84C00C9F8482079E700F0AD
:10B9700053F9002800F0A58008301B4AC9F82400BC
:10B98000C9F8202000F048F9002800F09480083021
:10B99000164AC9F82C00C9F8282056E7D1F89C00AF
:10B9A000083800F059F9FAE6F49FFF1F0080FF1FE6
:10B9B000D09FFF1F6C9FFF1FC09FFF1FF89FFF1F9F
:10B9C000189FFF1FD0A1FF1F600D0100E99FFF1FFF
:10B9D000C4200740C8200740CC200740D0200740A3
:10B9E000E89FFF1FC020074088004000C8004000BB
:10B9F00000F012F9002870D008304F4AC4F88400D3
:10BA0000C4F8802000F008F9002860D008304B4AC4
:10BA1000C9F88C00C9F888203CE7506A083800F063
:10BA20001BF962E6D1F89400083800F015F9B0E689
:10BA3000D1F88C00083800F00FF9A4E6D1F88400A2
:10BA4000083800F009F998E6C86F083800F004F9E2
:10BA50008DE6486F083800F0FFF882E6C86E0838B7
:10BA600000F0FAF877E6486E083800F0F5F86CE672
:10BA7000C86D083800F0F0F861E6486D083800F04D
:10BA8000EBF856E6C86C083800F0E6F84BE6486C70
:10BA9000083800F0E1F840E6C86B083800F0DCF840
:10BAA00035E6486B083800F0D7F82AE6C86A083847
:10BAB00000F0D2F81FE62A78C9F8280001322A706F
:10BAC000C3E62A78C9F8200001322A705AE72A789A
:10BAD000C9F8880001322A70DCE62A78C4F88000B0
:10BAE00001322A708EE72A78C9F8680001322A707C
:10BAF000C3E62A78C8F8600001322A7014E72A7871
:10BB0000C9F8480001322A70ABE62A78C8F840002C
:10BB100001322A701FE740298E4628BF4FF0400EA1
:10BB200002EB0E0302930123CEEB01014FEA0E4814
:10BB300000250193BCE600BF88004000C80040001B
:10BB4000F8B500F0A7FF294B29482A4C2A4F2B4D66
:10BB5000DFF8BCC0DFF8BCE0294E00221A605A6052
:10BB60009A60DA601A615A619A61DA611A625A62FD
:10BB70009A62DA621A635A639A63DA631A645A64DD
:10BB80009A64DA641A655A659A65DA651A665A66BD
:10BB90009A66DA661A675A679A67DA67C3F8802086
:10BBA0000168C3F8842041F480210160C3F30721B8
:10BBB0002170C3F30740134938701B0E2B70FF230D
:10BBC0008CF80030104D8EF8003010480B700123B7
:10BBD000337084F8642070264FF40074102207F844
:10BBE0002C3C2E70046081F8F820F8BD0080FF1F07
:10BBF000348004409C200740B0200740B420074018
:10BC0000942007401020074049E400E008E100E0EC
:10BC1000802007408820074072B60D480268B2FABB
:10BC200082F30F2B10DC4FF00041D94022EA0102D1
:10BC3000026062B6074803EBC303DB00C2180021B1
:10BC4000C15010465160704762B60020704700BF77
:10BC5000E891FF1FBC83FF1F0D4B0E4AC31AA2FBC6
:10BC600003231B090F2B0CD80B4A127852B972B65A
:10BC70000A484FF00041026821FA03F31A430260B8
:10BC800062B67047064A1278002AF0D0FFF76AB908
:10BC9000BC83FF1F398EE338E99FFF1FE891FF1F28
:10BCA000F49FFF1F38B50E4B0E4C1B6821880546CC
:10BCB0008BB1B1F5917F05D20B4A4B1C55549BB209
:10BCC000238038BD0022084898470021064A555471
:10BCD0000123238038BDB1F5917FEDD338BD00BF7E
:10BCE00020A0FF1FDAA1FF1FE0A1FF1F2DE9F843ED
:10BCF000214E224F3168012380463B70B1B1204D67
:10BD00004B8801EB8302013300240F2BC2F808801B
:10BD10002C7004D84B8000233B70BDE8F88340238F
:10BD20000B800320FFF782F93460F4E7DFF85490CA
:10BD300099F80030002BF0D0114D45F6215408E061
:10BD4000013C12D02B7883B900F004FD99F8003043
:10BD50007BB10320FFF7F0F80528F1D8FFF75CFF6F
:10BD6000014630600028EBD0CAE701232B70BDE804
:10BD7000F883BDE8F88300BF3CA0FF1F10A0FF1FA1
:10BD800040A0FF1FF49FFF1F1201F8B5D5B2A1B369
:10BD9000012943D04378044600781B0643EA00405B
:10BDA00040F4704045F004068F1E3043FFF79EFFBD
:10BDB000022F04F1020314D9053414F8023C14F8DC
:10BDC000032C14F8010C1B0443EA0223334343EA17
:10BDD0000060033FFFF78AFF022F234604F10304AC
:10BDE000EBD8022F23D0012F0DD045F4774040F03F
:10BDF0000500BDE8F840FFF779BF14482843BDE8C7
:10BE0000F840FFF773BF187845F4770545F006054D
:10BE100045EA0020BDE8F840FFF768BF03780C480A
:10BE200045EA03452843BDE8F840FFF75FBF1A78AD
:10BE3000587845F0774545F0070545EA022545EA7B
:10BE40000040BDE8F840FFF751BF00BF06F0F70023
:10BE500007F000F738B5084B1C7824B9074D29685E
:10BE600009B14B8803B938BD9B000B800320FFF755
:10BE7000DDF82C6038BD00BF10A0FF1F3CA0FF1FE5
:10BE80002DE9F041AD4E33680746002B00F092805B
:10BE90001D885A88910803EB81010432AA428C68FC
:10BEA00042D25A8004F00F064FEA1428A449A6F1A2
:10BEB000080208F00F00C4F30313062A00F101057D
:10BEC0000B701AD9B31E012B5FFA88F04ED9052EDC
:10BED00048D0042E00F0A481731F022B7FD90F2EAF
:10BEE0000ED1F72842D8F02802D0964B1B883BB1E0
:10BEF000FFF7D8FE0020BDE8F08127B1BD4202D097
:10BF00000020BDE8F081082EC4F3033300F08780E1
:10BF1000092E11D00A2E40F094800A2BF0D18A4BC2
:10BF20008A4A1B68A02181E01846FFF795FE04208D
:10BF3000FEF7E4FF3060B5E7092BE1D1270E00F0F2
:10BF40007B81834B814A1B689021C4F307461170A3
:10BF5000EDB2FCB2002B00F09D802246314628460F
:10BF6000984797E0F02843D9F72841D0F1380E28B8
:10BF7000C6D801A353F820F02FC1000013C1000060
:10BF800001C1000001BF000001BF0000F3C00000BC
:10BF900001BF0000D3C1000001BF00009DC100002F
:10BFA000B7C10000DBC0000001BF0000C3C000003B
:10BFB000A7C00000674B1B78002BA1D00420FEF720
:10BFC0009DFF0346306000289AD00588002D7FF43D
:10BFD00060AFFFF741FE35602846BDE8F081FFF70E
:10BFE00061FEC4F30740FFF75DFE072E02D1200E6D
:10BFF000FFF758FE534B584A198858481468584D53
:10C00000524A017000270E0AF0201F802E70107017
:10C010000CB301225348A0470120BDE8F081082B52
:10C020007FF46EAF504B494A1B688021C4F307462A
:10C030001170EDB2240E6BB3284622463146984764
:10C0400028E00B2E11D10B2B7FF45AAF474B3F4A00
:10C050001B68B021EAE7464B1B68002B00F0FB8011
:10C06000404898470120BDE8F0810C2E40F0008147
:10C070000C2B7FF445AF3F4B344A1B68C021117035
:10C08000EDB2C4F30746002B00F0C88028463146C5
:10C09000240E98473849314A314B0D7016701C7088
:10C0A0000120BDE8F081354B1B68002B00F0D680E5
:10C0B0009847C4F30746254BEDB2240E83F8008061
:10C0C000E8E72F4B1B68002BF2D12E4B1B68A3B166
:10C0D000FE209847C4F30746EDE72B4B1B68002B67
:10C0E000E6D1284B1B6843B1FC209847C4F30746B0
:10C0F000E1E7264B1B68002BDAD1C4F30746DAE7E9
:10C10000234B1B68C4F30746002BD4D03046984716
:10C11000D1E7204B1A68002AEFD0260C630C06F0FA
:10C120007F0003F47E531843F6B29047C3E71A4BDF
:10C130001B68C4F30746002BE8D1BCE748A0FF1FEB
:10C14000DEA1FF1FDAA1FF1F24A0FF1FD8A1FF1F40
:10C1500058A0FF1FF49FFF1F20A0FF1FDCA1FF1F9F
:10C16000DDA1FF1FE0A1FF1F50A0FF1F54A0FF1F74
:10C1700038A0FF1F14A0FF1FDFA1FF1F00A0FF1F9B
:10C1800004A0FF1F08A0FF1F44A0FF1F34A0FF1F33
:10C190004CA0FF1F1CA0FF1F30A0FF1F3F4B1B68C0
:10C1A000002B85D13E4B1B68002BA6D0FA20984768
:10C1B000C4F307467FE73B4B1B68002B7FF478AF47
:10C1C000374B1B68002B98D0FB209847C4F30746D9
:10C1D00071E7354B1B68002B7FF46AAF304B1B684F
:10C1E000002B8AD0F8209847C4F3074663E70E2B4C
:10C1F0007FF486AE2D4A2E4B1268E0211970002A7A
:10C2000047D0260C610C06F07F0301F47E511943E0
:10C21000EDB2A1F5005128469047F6B2240E39E759
:10C22000FFF740FDC4F30740FFF73CFD200EFFF78A
:10C2300039FD0020BDE8F0811E4B1D4A1B6880219E
:10C240001170EDB2C4F3074683B1314628463A4631
:10C2500098473C461EE70120BDE8F081104B1B6863
:10C26000002B3FF44AAFFF20984746E71C4611E7F2
:10C270000D2EBCD10D2B7FF443AE0F4B0C4A1B6827
:10C28000D0211170EDB2C4F30746002B7FF4FEAE4F
:10C29000C4E7C4F30746EDB2240EFBE62CA0FF1F53
:10C2A00008A0FF1F0CA0FF1FFC9FFF1F18A0FF1F6F
:10C2B000D8A1FF1F50A0FF1F28A0FF1F38B5164DA3
:10C2C0002868E0B101884488A14213DD03191B7A74
:10C2D00083B104F10803C2180C1B002302E012F81A
:10C2E000011F21B10133A342F9D1204638BD1C46BC
:10C2F000204638BDFFF7B0FC0020286038BD074B52
:10C300001B780BB9002038BD0220FEF7F7FD28602E
:10C310000028D7D1F6E700BF64A0FF1FF49FFF1FDE
:10C320000D4B1B78BBB910B50C4C216803F0FF0214
:10C330004B883F2B07DC07330B4401F1470003F820
:10C34000012F8342FBD140230B800120FEF76EFEBC
:10C350000023236010BD70475CA0FF1F60A0FF1F7B
:10C3600010B4EFF3108272B6437F33B9017F012915
:10C3700007D003290FD00123437702B962B610BC5E
:10C380007047124C2168A1B1114943610B68836168
:10C3900008605861EFE70F4C216881B10E49436195
:10C3A0000B688361086058610C4B4FF08051196035
:10C3B000E1E7074B4161816120601860DBE7064BD4
:10C3C0004161816120601860EEE700BF7CA0FF1F23
:10C3D00078A0FF1F6CA0FF1F70A0FF1F04ED00E0FE
:10C3E00070B5EFF3108272B60C4C206880B10C4E21
:10C3F00000254369236073B19D6102B962B6457738
:10C4000083689847EFF3108272B620680028F0D155
:10C4100002B962B670BD3360EFE700BF6CA0FF1FCA
:10C4200070A0FF1FFFF7DCBF184A30B41468002C5F
:10C4300027D0036821688B420ED2CB1A002184607A
:10C44000C1602360E06010600223037530BC704758
:10C4500011688B42144608D3A2685B1A0360002A55
:10C46000F6D18260C460A060EEE7D268C2608460EA
:10C47000E060C568CB1A0222A8602360027530BC58
:10C4800070478460C4601060DEE700BF74A0FF1FC7
:10C49000F8B5224E34682CB32368002B3AD1204FD4
:10C4A0001D4604E03468ECB12368002B32D1A36848
:10C4B00003B1DD6020693360036825751B68BB42EA
:10C4C00021D1037F4560022BC46020D0FFF748FFD5
:10C4D0006368002BE6D023602046FFF7A5FF346891
:10C4E000002CE1D1EFF3108372B60E4A00211068E0
:10C4F000116003B962B628B18468FFF795FF204642
:10C500000028F9D1F8BD224600219847E0E783686A
:10C510009847DDE7013B2360E4E700BF74A0FF1FFD
:10C520004186000084A0FF1F024A13680133136094
:10C53000FFF7AEBF949EFF1F704700BF0368F0B4C3
:10C54000FBB1002501249D60DC601B4C1A601C447B
:10C55000241104F144056A11032692009E60174FCE
:10C560000679174B47F8241002F1604202F5614248
:10C5700005F01F05012000FA05F5E6541560F0BC32
:10C580007047104C236843F40003236000BF0E4B38
:10C590000E4DA4F58734A4F59E7401261E60234633
:10C5A00004609C68002CD0D01033AB420360F8D1FB
:10C5B000002303601846E2E7008FFCBFEC91FF1FE9
:10C5C00044E400E03C8004400070034040710340BC
:10C5D0000168A9B10B4BF0B40B441B110A4E0B4F71
:10C5E0000B4D46F8237003F1440202F01F040123AF
:10C5F0005211A340002445F822308C600460F0BC46
:10C60000704700BF008FFCBFEC91FF1F39C50000D1
:10C6100080E100E0024A034B012111601B681847CA
:10C620000C710340EC91FF1F024A034B0121116082
:10C630005B6818471C710340EC91FF1F024A034BD3
:10C64000012111609B6818472C710340EC91FF1F7A
:10C65000024A034B01211160DB6818473C7103401B
:10C66000EC91FF1FF8B50E4671B17AB1074614463A
:10C6700000253B6816F8011B1B6838469847013CAB
:10C680000544F6D12846F8BD0846F8BD1046F8BD69
:10C6900000B5064A036812885B6883B001A9ADF84B
:10C6A00004200222984703B05DF804FB5C0D0100F2
:10C6B000F0B507468BB0002A33D0012A08BF0A2202
:10C6C00051B3212400E0F4B2B1FBF2F502FB1511E5
:10C6D000C8B2092900F1300198BFC8B20AA988BFC1
:10C6E0003730214488BFC0B201F8240C661E2946A9
:10C6F000002DE8D133B1013CE4B20AAB23442D2232
:10C7000003F8242C3B6801AA11195B683846C4F170
:10C71000220298470BB0F0BD30228DF8252021244D
:10C72000E8E70368C9B21B6898470BB0F0BD00BFCB
:10C730000029BABF49422D2300230A22FFF7B8BFC0
:10C7400008B5F3F7B1FFF5F78FFD00F003F8FAE74E
:10C75000704700BF38B5224C237803B138BD0123A0
:10C760002370FFF7ABFD70BB00F068F840BB00F032
:10C77000FBF810BBFEF700FBE0B900232370EFF3DA
:10C780000583002BEAD1EFF3108172B6154B1868C0
:10C79000E0B1154C2278CAB945691D6001232370A8
:10C7A000C5B1AA6101B962B600254577836898478B
:10C7B0002570D3E700F0B4F9DFE700F0AFF9D9E76F
:10C7C00000F0AAF9D3E7FFF7C3FFCDE70029C5D1F1
:10C7D00062B638BD054B1D600029E5D1E3E700BF17
:10C7E00088A0FF1F7CA0FF1F80A0FF1F78A0FF1F55
:10C7F000F0B44D1E2E46002400E00134B0FBF2F3ED
:10C8000002FB1300092800F130078ABF3730F8B265
:10C81000C0B206F8010F1846002BEED10A1953706A
:10C820004CB1107815F8016F28700133E01A83427B
:10C8300002F80169F5DB0846F0BC7047054A064B73
:10C8400010781B78C0B2DBB2984238BF4030C01AB3
:10C85000704700BF90A0FF1F91A0FF1FF0B4384B9E
:10C860001A7912F0300F2CD072B6997D01F0FF02C8
:10C8700000293DD062B6334F334938780D78334EB6
:10C880001C46C0B2EDB2431C402BE17928BF002307
:10C89000AB4202F1FF32C9B21CBFF154184612F08C
:10C8A000FF02F0D12A4B1B68C2B23A704BB1A842CA
:10C8B00036BFC5F14005401B40192728C4BF0122DF
:10C8C0001A701F49CA78D2B2150616D452060DD571
:10C8D0001B4B1B795B0609D51E4B1F491B680022A9
:10C8E0000A7003B11A70164B3C22DA70F0BC704724
:10C8F0004022D9795A7462B6E3E70B791C06E5D574
:10C90000164B174E1C783378E4B2DBB29C420ED043
:10C91000144D01E0A3420AD00133402B28BF00236D
:10C920000879E85CC0B2C871087D0728F2D9DBB28B
:10C93000034933700B79180644BF7C23CB70C5E7DD
:10C9400000A0064090A0FF1F91A0FF1FD4A0FF1FD2
:10C950008CA0FF1F18A1FF1F14A1FF1F1CA1FF1F08
:10C9600015A1FF1F94A0FF1F054A064B10781B78E6
:10C97000C0B2DBB2984238BF4030C01A704700BF27
:10C9800090A1FF1F25A1FF1FF0B4384B1A7912F0B8
:10C99000300F2CD072B6997D01F0FF0200293DD0F6
:10C9A00062B6334F334938780D78334E1C46C0B2E7
:10C9B000EDB2431C402BE17928BF0023AB4202F1CA
:10C9C000FF32C9B21CBFF154184612F0FF02F0D179
:10C9D0002A4B1B68C2B23A704BB1A84236BFC5F1B0
:10C9E0004005401B40192728C4BF01221A701F4967
:10C9F000CA78D2B2150616D452060DD51B4B1B7938
:10CA00005B0609D51E4B1F491B6800220A7003B143
:10CA10001A70164B3C22DA70F0BC70474022D9796C
:10CA20005A7462B6E3E70B791C06E5D5164B174E30
:10CA30001C783378E4B2DBB29C420ED0144D01E096
:10CA4000A3420AD00133282B28BF00230879E85CD1
:10CA5000C0B2C871087D0728F2D9DBB20349337030
:10CA60000B79180644BF7C23CB70C5E700B00640A5
:10CA700090A1FF1F25A1FF1F50A1FF1F20A1FF1F95
:10CA800094A1FF1F24A1FF1F98A1FF1F91A1FF1FC9
:10CA900028A1FF1F70B584B072B6194B194D1A4802
:10CAA000702241260F2480211A702E701A460470BD
:10CAB000197013781B06FCD5144B186862B6144B1A
:10CAC000144C984298BF00EB800001A998BF400029
:10CAD0000A22FFF78DFE01A92046002311F8012B41
:10CAE00001333AB10A2B20F8022FF7D11623237015
:10CAF00004B070BD5B00DBB2237004B070BD00BF3A
:10CB00000000024007000240060002400800024008
:10CB10007F969800C492FF1F704700BF704700BF08
:10CB2000704700BFFFFFFFFF2DE9F043DFF8EC8007
:10CB30008BB006460F4600F073F898F900300133C9
:10CB400004460D4637D03046394600F0DFF900285C
:10CB500031D02BA3D3E900233046394600F026FE1E
:10CB6000814668BB28A3D3E900233046394600F04C
:10CB7000FFFD00B398F90030254ACDF82090042439
:10CB800000200021022BCDE90467CDE90267009463
:10CB90000192CDE906012CD0684600F0BDF940B302
:10CBA000089B1BB101F0AAF9089B0360DDE90601AF
:10CBB0000BB0BDE8F083204629460BB0BDE8F083FA
:10CBC000134A98F90030019203210022CDE904674D
:10CBD000CDE90267009108922BB90E4B4FF06042ED
:10CBE000CDE90623D8E70C490020022BCDE9060148
:10CBF000D2D101F083F922230360D1E7AFF30080A3
:10CC0000EF39FAFE422E864051302DD5104987C0AB
:10CC1000D00D0100FFFFEF470000F07FDA92FF1F09
:10CC20002DE9F04FB04F21F00042BA4283B00C46DC
:10CC30004FEAD17605460DD9AC4FBA4225D9C1F39A
:10CC40001303034340F0EF800EB10020014603B010
:10CC5000BDE8F08FA64B9A4200F2CC80A54B9A42D9
:10CC600000F2DE808AA3D3E9002300F05DF9002200
:10CC7000A14B00F09BFD002800F0058128462146CD
:10CC800000229D4B00F050F9E1E783A3D3E9002394
:10CC900000F08CFD002840F0CB802846214680A380
:10CCA000D3E9002300F064FD0028CED1934B284641
:10CCB00003EBC60821467CA3D3E9002300F0E6FA83
:10CCC000D8E9002300F030F900F07AFD804600F04A
:10CCD00077FA77A3D3E9002306460F4600F0D6FA89
:10CCE00002460B462846214600F01CF972A3D3E900
:10CCF0000023CDE900013046394600F0C7FA8246EC
:10CD00008B4652465B46DDE9000100F00BF9054613
:10CD10000C462A4623462846214600F0B7FA68A367
:10CD2000D3E9002306460F4600F0B0FA66A3D3E924
:10CD3000002300F0F7F832463B4600F0A7FA64A360
:10CD4000D3E9002300F0F0F832463B4600F09EFAAB
:10CD500061A3D3E9002300F0E5F832463B4600F03A
:10CD600095FA5FA3D3E9002300F0DEF832463B4694
:10CD700000F08CFA02460B462846214600F0D2F815
:10CD800006460F462846214632463B46B8F1000F7C
:10CD900056D000F07BFA324604460D463B46002052
:10CDA0004FF0804100F0BEF802460B46204629466F
:10CDB00000F096FB02460B465046594600F0B2F88A
:10CDC000DDE9002300F0AEF80B4602464A49002098
:10CDD00000F0A8F86FF47F7398454FDA08F57A7879
:10CDE00001EB085100224FF0B87300F04FFA03B086
:10CDF000BDE8F08F424B9A423FF658AF414BF400EA
:10CE00002344D3E9002300F08DF83F4BC6F101081D
:10CE10001C44CDE90001D4E900ABC6EB080870E77B
:10CE20004FF0000875E702460B4600F07DF80EE76C
:10CE300017A3D3E900231046194600F027FA06E7A6
:10CE400000F024FA0022804689464FF080433046A5
:10CE5000394600F067F802460B464046494600F066
:10CE60003FFB2A46234600F05DF802460B460020B1
:10CE7000214900F057F803B0BDE8F08F01EB0851ED
:10CE800003B0BDE8F08F804643E700BFAFF30080FA
:10CE90009C7500883CE4377EEF39FAFE422E8640CE
:10CEA00051302DD5104987C0FE822B654715F73FBD
:10CEB0000000E0FE422EE63F763C7935EF39EA3D50
:10CEC000D0A4BE726937663EF16BD2C541BDBB3E90
:10CED0002CDE25AF6A56113F93BDBE166CC1663F6E
:10CEE0003E5555555555C53F412E8640FFFFEF7FB6
:10CEF000422ED63FFFFF2F3E0000F03FD80D01002D
:10CF0000B1A2F03FF80D0100E80D010041F0004131
:10CF100001F58010C00F70470020704781F000417C
:10CF200002E000BF83F0004330B54FEA41044FEA0E
:10CF3000430594EA050F08BF90EA020F1FBF54EAA9
:10CF4000000C55EA020C7FEA645C7FEA655C00F045
:10CF5000E2804FEA5454D4EB5555B8BF6D420CDD16
:10CF60002C4480EA020281EA030382EA000083EA99
:10CF7000010180EA020281EA0303362D88BF30BD39
:10CF800011F0004F4FEA01314FF4801C4CEA11318F
:10CF900002D0404261EB410113F0004F4FEA0333EE
:10CFA0004CEA133302D0524263EB430394EA050F79
:10CFB00000F0A780A4F10104D5F1200E0DDB02FAE8
:10CFC0000EFC22FA05F2801841F1000103FA0EF27C
:10CFD000801843FA05F359410EE0A5F120050EF142
:10CFE000200E012A03FA0EFC28BF4CF0020C43FA73
:10CFF00005F3C01851EBE37101F0004507D54FF080
:10D00000000EDCF1000C7EEB00006EEB0101B1F5CF
:10D01000801F1BD3B1F5001F0CD349085FEA300015
:10D020004FEA3C0C04F101044FEA445212F5800F20
:10D0300080F09A80BCF1004F08BF5FEA500C50F1BD
:10D04000000041EB045141EA050130BD5FEA4C0CA0
:10D05000404141EB010111F4801FA4F10104E9D129
:10D0600091F0000F04BF01460020B1FA81F308BF20
:10D070002033A3F10B03B3F120020CDA0C3208DDEC
:10D0800002F1140CC2F10C0201FA0CF021FA02F1C7
:10D090000CE002F11402D8BFC2F1200C01FA02F137
:10D0A00020FA0CFCDCBF41EA0C019040E41AA2BF5C
:10D0B00001EB0451294330BD6FEA04041F3C1CDA24
:10D0C0000C340EDC04F11404C4F1200220FA04F044
:10D0D00001FA02F340EA030021FA04F345EA0301EE
:10D0E00030BDC4F10C04C4F1200220FA02F001FAB0
:10D0F00004F340EA0300294630BD21FA04F0294632
:10D1000030BD94F0000F83F4801306BF81F48011CA
:10D110000134013D4EE77FEA645C18BF7FEA655C3D
:10D1200029D094EA050F08BF90EA020F05D054EA0F
:10D13000000C04BF1946104630BD91EA030F1EBF14
:10D140000021002030BD5FEA545C05D14000494118
:10D1500028BF41F0004130BD14F580043CBF01F50B
:10D16000801130BD01F0004545F0FE4141F47001F1
:10D170004FF0000030BD7FEA645C1ABF19461046CC
:10D180007FEA655C1CBF0B46024650EA013406BFCD
:10D1900052EA033591EA030F41F4002130BD00BF8C
:10D1A00090F0000F04BF0021704730B54FF4806449
:10D1B00004F132044FF000054FF0000150E700BFCA
:10D1C00090F0000F04BF0021704730B54FF4806429
:10D1D00004F1320410F0004548BF40424FF0000116
:10D1E0003EE700BF42004FEAE2014FEA31014FEA59
:10D1F00002701FBF12F07F4393F07F4F81F06051A8
:10D20000704792F0000F14BF93F07F4F704730B516
:10D210004FF4607401F0004521F0004120E700BFA9
:10D2200050EA010208BF704730B54FF000050AE030
:10D2300050EA010208BF704730B511F0004502D531
:10D24000404261EB41014FF4806404F132045FEA33
:10D25000915C3FF4DCAE4FF003025FEADC0C18BFD8
:10D2600003325FEADC0C18BF033202EBDC02C2F1CE
:10D27000200300FA03FC20FA02F001FA03FE40EA60
:10D280000E0021FA02F11444C1E600BF70B54FF060
:10D29000FF0C4CF4E06C1CEA11541DBF1CEA135542
:10D2A00094EA0C0F95EA0C0F00F0DEF82C4481EAAA
:10D2B000030621EA4C5123EA4C5350EA013518BFCA
:10D2C00052EA033541F4801143F4801338D0A0FBB7
:10D2D00002CE4FF00005E1FB02E506F00042E0FB64
:10D2E00003E54FF00006E1FB03569CF0000F18BF6A
:10D2F0004EF0010EA4F1FF04B6F5007F64F5407412
:10D3000004D25FEA4E0E6D4146EB060642EAC621A4
:10D3100041EA55514FEAC52040EA5E504FEACE2E11
:10D32000B4F1FD0C88BFBCF5E06F1ED8BEF1004F14
:10D3300008BF5FEA500E50F1000041EB045170BD90
:10D3400006F0004646EA010140EA020081EA0301D4
:10D35000B4EB5C04C2BFD4EB0C0541EA045170BDD0
:10D3600041F480114FF0000E013C00F3AB8014F14A
:10D37000360FDEBF002001F0004170BDC4F1000493
:10D38000203C35DA0C341BDC04F11404C4F1200514
:10D3900000FA05F320FA04F001FA05F240EA02006F
:10D3A00001F0004221F0004110EBD37021FA04F6A5
:10D3B00042EB06015EEA430E08BF20EAD37070BD5F
:10D3C000C4F10C04C4F1200500FA04F320FA05F0BE
:10D3D00001FA04F240EA020001F0004110EBD370C0
:10D3E00041F100015EEA430E08BF20EAD37070BD30
:10D3F000C4F1200500FA05F24EEA020E20FA04F309
:10D4000001FA05F243EA020321FA04F001F00041B7
:10D4100021FA04F220EA020000EBD3705EEA430E28
:10D4200008BF20EAD37070BD94F0000F0FD101F057
:10D430000046400041EB010111F4801F08BF013C90
:10D44000F7D041EA060195F0000F18BF704703F0CE
:10D450000046520043EB030313F4801F08BF013D55
:10D46000F7D043EA0603704794EA0C0F0CEA135511
:10D4700018BF95EA0C0F0CD050EA410618BF52EACB
:10D480004306D1D181EA030101F000414FF00000D1
:10D4900070BD50EA410606BF1046194652EA4306DF
:10D4A00019D094EA0C0F02D150EA013613D195EA53
:10D4B0000C0F05D152EA03361CBF104619460AD19B
:10D4C00081EA030101F0004141F0FE4141F47001A5
:10D4D0004FF0000070BD41F0FE4141F4780170BD95
:10D4E00070B54FF0FF0C4CF4E06C1CEA11541DBFFA
:10D4F0001CEA135594EA0C0F95EA0C0F00F0A7F8FC
:10D50000A4EB050481EA030E52EA03354FEA013128
:10D5100000F088804FEA03334FF0805545EA13133B
:10D5200043EA12634FEA022245EA111545EA106503
:10D530004FEA00260EF000419D4208BF964244F19A
:10D54000FD0404F5407402D25B084FEA3202B61AB9
:10D5500065EB03055B084FEA32024FF480104FF48D
:10D56000002CB6EB020E75EB030E22BFB61A754601
:10D5700040EA0C005B084FEA3202B6EB020E75EB94
:10D58000030E22BFB61A754640EA5C005B084FEAFC
:10D590003202B6EB020E75EB030E22BFB61A7546C9
:10D5A00040EA9C005B084FEA3202B6EB020E75EBD4
:10D5B000030E22BFB61A754640EADC0055EA060E95
:10D5C00018D04FEA051545EA16754FEA06164FEAD8
:10D5D000C30343EA52734FEAC2025FEA1C1CC0D184
:10D5E00011F4801F0BD141EA00014FF000004FF011
:10D5F000004CB6E711F4801F04BF01430020B4F1D2
:10D60000FD0C88BFBCF5E06F3FF6AFAEB5EB030C89
:10D6100004BFB6EB020C5FEA500C50F1000041EB86
:10D62000045170BD0EF0004E4EEA113114EB5C0453
:10D63000C2BFD4EB0C0541EA045170BD41F4801126
:10D640004FF0000E013C90E645EA060E8DE60CEA2E
:10D65000135594EA0C0F08BF95EA0C0F3FF43BAF4B
:10D6600094EA0C0F0AD150EA01347FF434AF95EA02
:10D670000C0F7FF425AF104619462CE795EA0C0FE6
:10D6800006D152EA03353FF4FDAE1046194622E7B3
:10D6900050EA410618BF52EA43067FF4C5AE50EA8D
:10D6A00041047FF40DAF52EA43057FF4EBAE12E77D
:10D6B0004FF0FF3C06E000BF4FF0010C02E000BF5E
:10D6C0004FF0010C4DF804CD4FEA410C7FEA6C5C41
:10D6D0004FEA430C18BF7FEA6C5C1BD001B050EAE4
:10D6E000410C0CBF52EA430C91EA030F02BF90EACF
:10D6F000020F0020704710F1000F91EA030F58BF8E
:10D70000994208BF90422CBFD8176FEAE37040F0EF
:10D71000010070474FEA410C7FEA6C5C02D150EA8D
:10D72000013C07D14FEA430C7FEA6C5CD6D152EA48
:10D73000033CD3D05DF8040B704700BF844610460D
:10D7400062468C461946634600E000BF01B5FFF70C
:10D75000B7FF002848BF10F1000F01BD4DF808EDDC
:10D76000FFF7F4FF0CBF012000205DF808FB00BFAD
:10D770004DF808EDFFF7EAFF34BF012000205DF807
:10D7800008FB00BF4DF808EDFFF7E0FF94BF012054
:10D7900000205DF808FB00BF4DF808EDFFF7CEFF55
:10D7A00094BF012000205DF808FB00BF4DF808ED94
:10D7B000FFF7C4FF34BF012000205DF808FB00BF65
:10D7C0004FEA410212F5001215D211D56FF47873A9
:10D7D000B3EB625212D94FEAC12343F0004343EA4C
:10D7E000505311F0004F23FA02F018BF4042704727
:10D7F0004FF00000704750EA013005D111F00040B1
:10D8000008BF6FF0004070474FF00000704700BF46
:10D810004FEA4102B2F1E04324BFB3F5001CDCF152
:10D82000FE5C0DD901F0004C4FEAC0024CEA50708A
:10D83000B2F1004F40EB830008BF20F001007047B9
:10D8400011F0804F21D113F13872BCBF01F00040BC
:10D85000704741F480114FEA5252C2F11802C2F1EE
:10D86000200C10FA0CF320FA02F018BF40F001006F
:10D870004FEAC1234FEAD32303FA0CFC40EA0C0021
:10D8800023FA02F34FEA4303CCE77FEA625307D15E
:10D8900050EA01331EBF4FF0FE4040F44000704795
:10D8A00001F0004040F0FE4040F40000704700BF2F
:10D8B00080F0004002E000BF81F0004142001FBF45
:10D8C0005FEA410392EA030F7FEA226C7FEA236C4E
:10D8D0006AD04FEA1262D2EB1363C1BFD218414043
:10D8E00048404140B8BF5B42192B88BF704710F0D9
:10D8F000004F40F4000020F07F4018BF404211F07C
:10D90000004F41F4000121F07F4118BF494292EAE3
:10D91000030F3FD0A2F1010241FA03FC10EB0C000F
:10D92000C3F1200301FA03F100F0004302D549429C
:10D9300060EB4000B0F5000F13D3B0F1807F06D349
:10D9400040084FEA310102F10102FE2A51D2B1F141
:10D95000004F40EBC25008BF20F0010040EA030036
:10D960007047490040EB000010F4000FA2F10102E3
:10D97000EDD1B0FA80FCACF1080CB2EB0C0200FA6D
:10D980000CF0AABF00EBC25052421843BCBFD040BB
:10D990001843704792F0000F81F4000106BF80F435
:10D9A00000000132013BB5E74FEA41037FEA226CF8
:10D9B00018BF7FEA236C21D092EA030F04D092F0C3
:10D9C000000F08BF0846704790EA010F1CBF0020F7
:10D9D000704712F07F4F04D1400028BF40F0004054
:10D9E000704712F100723CBF00F50000704700F074
:10D9F000004343F0FE4040F4000070477FEA22629B
:10DA000016BF08467FEA23630146420206BF5FEA6B
:10DA1000412390EA010F40F4800070474FF000036B
:10DA200004E000BF10F0004348BF40425FEA000C32
:10DA300008BF704743F0964301464FF000001CE0DA
:10DA400050EA010208BF70474FF000030AE000BF30
:10DA500050EA010208BF704711F0004302D540426E
:10DA600061EB41015FEA010C02BF844601460020E0
:10DA700043F0B64308BFA3F18053A3F50003BCFAFB
:10DA80008CF2083AA3EBC25310DB01FA02FC6344A8
:10DA900000FA02FCC2F12002BCF1004F20FA02F2AF
:10DAA00043EB020008BF20F00100704702F12002A2
:10DAB00001FA02FCC2F1200250EA4C0021FA02F203
:10DAC00043EB020008BF20EADC7070474FF0FF0C08
:10DAD0001CEAD0521EBF1CEAD15392EA0C0F93EA03
:10DAE0000C0F6FD01A4480EA010C400218BF5FEAA5
:10DAF00041211ED04FF0006343EA501043EA511118
:10DB0000A0FB01310CF00040B1F5000F3EBF490011
:10DB100041EAD3715B0040EA010062F17F02FD2A15
:10DB20001DD8B3F1004F40EBC25008BF20F00100F8
:10DB3000704790F0000F0CF0004C08BF49024CEA0F
:10DB4000502040EA51207F3AC2BFD2F1FF0340EAA1
:10DB5000C250704740F400004FF00003013A5DDC12
:10DB600012F1190FDCBF00F000407047C2F1000253
:10DB7000410021FA02F1C2F1200200FA02FC5FEA40
:10DB8000310040F1000053EA4C0308BF20EADC708A
:10DB9000704792F0000F00F0004C02BF400010F4FC
:10DBA000000F013AF9D040EA0C0093F0000F01F0A9
:10DBB000004C02BF490011F4000F013BF9D041EACB
:10DBC0000C018FE70CEAD15392EA0C0F18BF93EACD
:10DBD0000C0F0AD030F0004C18BF31F0004CD8D1F7
:10DBE00080EA010000F00040704790F0000F17BF7E
:10DBF00090F0004F084691F0000F91F0004F14D0C4
:10DC000092EA0C0F01D142020FD193EA0C0F03D11B
:10DC10004B0218BF084608D180EA010000F000401E
:10DC200040F0FE4040F40000704740F0FE4040F4F9
:10DC3000400070474FF0FF0C1CEAD0521EBF1CEA98
:10DC4000D15392EA0C0F93EA0C0F69D0A2EB0302B6
:10DC500080EA010C49024FEA402037D04FF0805350
:10DC600043EA111143EA10130CF000408B4238BF15
:10DC70005B0042F17D024FF4000C8B4224BF5B1A23
:10DC800040EA0C00B3EB510F24BFA3EB510340EA71
:10DC90005C00B3EB910F24BFA3EB910340EA9C001F
:10DCA000B3EBD10F24BFA3EBD10340EADC001B018F
:10DCB00018BF5FEA1C1CE0D1FD2A3FF650AF8B4233
:10DCC00040EBC25008BF20F0010070470CF0004C40
:10DCD0004CEA50207F32C2BFD2F1FF0340EAC2506B
:10DCE000704740F400004FF00003013A37E792F02C
:10DCF000000F00F0004C02BF400010F4000F013A8A
:10DD0000F9D040EA0C0093F0000F01F0004C02BF84
:10DD1000490011F4000F013BF9D041EA0C0195E7ED
:10DD20000CEAD15392EA0C0F08D142027FF47DAF86
:10DD300093EA0C0F7FF470AF084676E793EA0C0F76
:10DD400004D14B023FF44CAF08466EE730F0004C74
:10DD500018BF31F0004CCAD130F000427FF45CAF04
:10DD600031F000437FF43CAF5FE700BF4FF0FF3C72
:10DD700006E000BF4FF0010C02E000BF4FF0010CC5
:10DD80004DF804CD4FEA40024FEA41037FEA226C8E
:10DD900018BF7FEA236C11D001B052EA530C18BFB0
:10DDA00090EA010F58BFB2EB030088BFC81738BF15
:10DDB0006FEAE17018BF40F0010070477FEA226C03
:10DDC00002D15FEA402C05D17FEA236CE4D15FEAFF
:10DDD000412CE1D05DF8040B704700BF8446084633
:10DDE0006146FFE70FB5FFF7C9FF002848BF10F1F4
:10DDF000000F0FBD4DF808EDFFF7F4FF0CBF012039
:10DE000000205DF808FB00BF4DF808EDFFF7EAFFC2
:10DE100034BF012000205DF808FB00BF4DF808ED7D
:10DE2000FFF7E0FF94BF012000205DF808FB00BF72
:10DE30004DF808EDFFF7D2FF94BF012000205DF8F8
:10DE400008FB00BF4DF808EDFFF7C8FF34BF012005
:10DE500000205DF808FB00BF4FEA4002B2F1FE4F20
:10DE60000FD34FF09E03B3EB12620DD94FEA00239C
:10DE700043F0004310F0004F23FA02F018BF404275
:10DE800070474FF00000704712F1610F01D142025C
:10DE900005D110F0004008BF6FF0004070474FF010
:10DEA0000000704742000ED2B2F1FE4F0BD34FF08C
:10DEB0009E03B3EB126209D44FEA002343F0004300
:10DEC00023FA02F070474FF00000704712F1610F23
:10DED00001D1420202D14FF0FF3070474FF00000F5
:10DEE000704700BF0B460146184600F001B800BF5E
:10DEF00013460A460146022000F0B4BE014B1868E2
:10DF0000704700BF0897FF1F70B50F4E0F4D761B6F
:10DF1000B61018BF002405D0013455F8043B9847CB
:10DF2000A642F9D10A4E0B4D761B02F06FFFB610D8
:10DF300018BF002406D0013455F8043B9847A64288
:10DF4000F9D170BD70BD00BF180E0100180E0100A0
:10DF50002C0E0100180E0100024B0146186800F05B
:10DF60000BB800BF0897FF1F024B0146186800F06E
:10DF70003DBF00BF0897FF1F2DE9F04F01F10B05D2
:10DF8000162D83B0064640F29F8035F0070500F15C
:10DF9000BF80A94200F2BC8000F058FBB5F5FC7FC1
:10DFA000C0F09C826B0A00F0BA80042B00F28381DF
:10DFB000A80900F1390E4FEA4E033830C44F07EB81
:10DFC0008303A3F108015C68A14207D1ACE0002AF9
:10DFD00080F2AC80E468A14200F0A680636823F080
:10DFE00003035A1B0F2AF2DDB9493C6901F1080EFF
:10DFF000744500F0B381636823F003035A1B0F2AB2
:10E0000000F39981002AC1F814E0C1F810E080F211
:10E010009E80B3F5007F80F06781DB0803F1010C7F
:10E0200001229B1002FA03F34A6851F83C80C4F8BD
:10E03000088001EBCC091A43A9F10803E3604A60A8
:10E0400041F83C40C8F80C40831001249C409442A5
:10E0500000F28A80144206D120F0030064001442CA
:10E0600000F10400FAD007EBC009CC468046DCF88A
:10E070000C108C4507D173E1002A80F28181C968B8
:10E080008C4500F06D814B6823F003035A1B0F2A67
:10E09000F2DD0C46D1F80CC054F8088F4B1945F04E
:10E0A00001054D6042F00101C8F80CC03046CCF8C3
:10E0B00008807B613B61C3F80CE0C3F808E059605D
:10E0C0009A5000F0C5FA1FE0102921D800F0BEFADE
:10E0D0001025062302207E4F07EB8303A3F10802DD
:10E0E0005C68944200F045816368E168A56823F0AC
:10E0F0000303234430465A68E96042F001028D6010
:10E100005A6000F0A5FA0834204603B0BDE8F08F4D
:10E1100000240C232046336003B0BDE8F08F802339
:10E120004FF0400E3F2049E770465DE72344E16829
:10E130005A68A56842F00102E96030468D605A6075
:10E1400000F086FA0834204603B0BDE8F08F23447F
:10E1500030465A6842F001025A6000F079FA0834F9
:10E16000204603B0BDE8F08FBC68636823F0030865
:10E17000A84504D3C5EB08030F2B00F38C80554B47
:10E18000DFF860911A68D9F8003001332A4404EBB3
:10E19000080A00F0608102F580520F3222F47F629B
:10E1A00022F00F0211463046019200F04BFCB0F114
:10E1B000FF3F8346019A00F05881824500F2FC80BF
:10E1C000454B1968DA451144196000F05381D9F8BC
:10E1D0000000DFF810E101301BBFCAEB0B0A51440D
:10E1E000CEF800B019601BF0070100F01781C1F1F3
:10E1F0000800C1F58051834408315A44C2F30B0230
:10E20000C2EB010949463046019300F01BFC431C58
:10E21000019B00F03F81CBEB00024A4442F0010237
:10E220001968C7F808B04944BC42CBF8042019600B
:10E23000DFF8A49016D0B8F10F0F40F2FD806268AD
:10E24000A8F10C0323F00703E01802F001024FF0DD
:10E25000050E1A430F2B6260C0F804E0C0F808E016
:10E2600000F21C811D4BBC681A68914288BF19607E
:10E270001B4B1A689142626888BF196022F0030242
:10E280009542A2EB050301D80F2B04DC304600F0C9
:10E29000DFF9002438E7621943F0010345F0010576
:10E2A00065603046BA60536000F0D2F90834204609
:10E2B00003B0BDE8F08F142B71D9542B00F2A48069
:10E2C000280B00F16F0E4FEA4E036E3076E600BF6A
:10E2D0000C97FF1FA4A1FF1FA8A1FF1FA0A1FF1F54
:10E2E0009CA1FF1F189BFF1F5A0A042A5ED9142AFB
:10E2F00000F2B38002F15C0149005B3207EB810C54
:10E3000057F82110DFF8DC81ACF1080C8C4500F0E7
:10E3100088804A6822F00302934202D289688C45C1
:10E32000F7D1D1F80CC07A68C4F80CC0A160CCF861
:10E330000840CC6088E6631942F0010745F001050A
:10E34000656030464B610B61C3F80CE0C3F808E030
:10E350005F609A50083400F07BF9D5E64A6873E6AE
:10E3600008F1010818F0030F0CF1080C7FF47FAEE0
:10E3700030E0DC68A34208BF02303FF435AEB3E6BC
:10E380000B440C465A68C96854F8085F42F0010211
:10E390005A603046E9608D6000F05AF9B4E603F146
:10E3A0005C0E03F15B004FEA4E0307E69A0902F1A7
:10E3B000390149003832A1E7BC424A4B3FF400AF73
:10E3C0009C68626822F003025AE759F808399945B7
:10E3D00040F0828010F0030F00F1FF30F5D17B6830
:10E3E00023EA04037B6064009C423FF6BDAE002C30
:10E3F0003FF4BAAE1C4240467FF435AE64001C4286
:10E4000000F10400FAD02EE6B3F5AA7F18D8E80B85
:10E4100000F1780E4FEA4E037730CFE54FF480518C
:10E42000EBE60121D8F80430921001FA02F21A4307
:10E43000C8F80420614677E70123CBF8043025E7CC
:10E4400040F25452934220D8A80C00F17D0E4FEABE
:10E450004E037C30B2E51032A4E6542A26D81A0BBB
:10E4600002F16F0149006E3248E7BC68626822F031
:10E47000030205E7CAF30B0000287FF4A8AE42446C
:10E48000BB6842F001025A60ECE6FE234FF07F0EBB
:10E490007E2093E501224FF00009C1E604F1080156
:10E4A000304600F0A3FCD9F80010DBE6B2F5AA7FF5
:10E4B00005D8DA0B02F17801490077321EE740F205
:10E4C00054518A4205D89A0C02F17D0149007C32F0
:10E4D00014E7FE217E2211E77B6884E7E808431CED
:10E4E0005B00F8E50C97FF1F8842F0B50DD98B183B
:10E4F00098420AD28118002A51D09A1A13F8014D75
:10E5000001F8014D9342F9D1F0BD0F2A48D941EAF3
:10E5100000039B0746D100F1100401F110031546DA
:10E5200053F8106C44F8106C53F80C6C44F80C6CF5
:10E5300053F8086C44F8086C103D53F8046C44F828
:10E54000046C0F2D03F1100304F11004E8D8A2F1BC
:10E55000100323F00F0302F00F0E1033BEF1030F70
:10E560001944034421D91E1F0D467446043C55F836
:10E57000047B46F8047F032CF8D8AEF1040424F0A1
:10E58000030404342344214402F0030262B1013B3A
:10E590000A4411F8014B03F8014F8A42F9D1F0BD4A
:10E5A0000346F3E70346F2E7F0BD7246EEE700BF2D
:10E5B00070B4840746D0541E002A41D0CDB2034621
:10E5C00002E0621EE4B3144603F8015B9A07F8D137
:10E5D000032C2ED9CDB245EA05250F2C45EA054579
:10E5E00019D903F110022646103E0F2E42F8105C96
:10E5F00042F80C5C42F8085C42F8045C02F110023C
:10E60000F2D8A4F1100222F00F0204F00F0410322D
:10E61000032C13440DD91E462246043A032A46F819
:10E62000045BFAD8221F22F003020432134404F0E0
:10E6300003042CB1C9B21C4403F8011BA342FBD153
:10E6400070BC704714460346C2E700BF704700BF66
:10E65000704700BF024B0A460146186800F002B836
:10E660000897FF1F2DE9F04F174683B0002900F0EF
:10E67000C1800E46814607F10B05FFF7E7FF56F80C
:10E6800004EC162D2EF00304A6F1080840D8102241
:10E690001546AF4241D8944275DAC94B996808EBE8
:10E6A00004008842416800F0D98021F0010303444E
:10E6B0005B68DB077DD51EF0010F35D03946484633
:10E6C000FFF75AFC0746E0B156F8043C23F001037B
:10E6D0004344A0F108029A4200F04481221F242AF8
:10E6E00000F23181132A00F2048103463246116898
:10E6F00019605168596092689A603146484600F046
:10E7000075FB4846FFF7A4FF384603B0BDE8F08F1D
:10E7100025F00705002D2A46BBDA0C230020C9F896
:10E72000003003B0BDE8F08F56F8083CC3EB080A90
:10E73000DAF8043023F0030C04EB0C039342BDDB46
:10E740005746DAF80C1057F8080F221F242AC16028
:10E75000886000F21781132A40F212813168CAF8EA
:10E7600008107168CAF80C101B2A00F22B810836B9
:10E770000AF110023168116071685160B1689160EE
:10E780003E461C46D046631B0F2B1DD8D8F80430DC
:10E7900003F0010323434444C8F80430636843F0A2
:10E7A000010363604846FFF753FF304603B0BDE8FE
:10E7B000F08F21F003012144914221DBC36882687C
:10E7C0000C46D3609A60DEE7D8F8042008EB050118
:10E7D00002F00102154343F001020B44C8F8045053
:10E7E0004A605A6842F0010208315A60484600F017
:10E7F000FDFAD7E7114603B0BDE8F04FFFF7BCBB09
:10E800001EF0010F7FF45AAF56F8083CC3EB080A1C
:10E81000DAF8043023F0030C01EB0C0E96458BDB89
:10E82000C36882685746D3609A6057F8081FDAF8C1
:10E830000C30CB60221F242A996000F29980132AA1
:10E8400062D93368CAF808307368CAF80C301B2ADA
:10E8500000F2A08008360AF1100356E021F0030B05
:10E86000A34405F11000834559DA1EF0010F7FF42F
:10E8700025AF56F8081CC1EB080ADAF8041021F09D
:10E88000030CE34458453FF757AF5746DAF80C10EE
:10E8900057F8080F221F242AC160886000F2B48054
:10E8A000132A40F2A5803168CAF808107168CAF8C6
:10E8B0000C101B2A00F2AF8008360AF110023168F2
:10E8C000116071685160B16891600AEB0501C5EB98
:10E8D0000B0242F0010299604A60DAF8043003F05A
:10E8E00001031D434846CAF80450FFF7B1FE3846FD
:10E8F0005CE733680360736843601B2A27D800F124
:10E90000080306F10802F2E63B4632681A607268B4
:10E910005A60B2689A603E467446D04633E708EBC8
:10E920000501C5EB0B0B4BF0010299604A6056F8EC
:10E93000043C03F001031D43484646F8045CFFF71E
:10E9400087FE304632E73146FFF7CEFDD5E6B368A5
:10E950008360F368C360242A28D000F1100306F115
:10E960001002C4E650F8043C23F003031C440AE7F9
:10E97000314638467446D046FFF7B6FD3E4602E7BC
:10E980003A46F7E6314638461C46D046FFF7ACFD1E
:10E990003E46F8E6B368CAF81030F368CAF8143097
:10E9A000242A1BD010360AF11803AEE7336903613D
:10E9B0007369436106F1180200F1180397E600BF7E
:10E9C0000C97FF1FB168CAF81010F168CAF814104C
:10E9D000242A0FD010360AF11802CBE63369CAF8A0
:10E9E00018307369CAF81C3018360AF120038CE716
:10E9F0003A4664E73269CAF818207269CAF81C20DE
:10EA000018360AF12002B5E6314638460193FFF781
:10EA10006BFD019B59E7B168CAF81010F168CAF89C
:10EA20001410242A03D010360AF1180247E732697D
:10EA3000CAF818207269CAF81C2018360AF1200298
:10EA40003DE700BF38B5074C002305460846236064
:10EA5000FBF7E8FC431C00D038BD2368002BFBD03B
:10EA60002B6038BD04A3FF1FFFFFFFFFFFFFFFFF69
:10EA7000FFFFFFFFFFFFFFFFFFFFFFFFFFFFFFFFA6
:10EA800090F800F06DE9024520F007016FF0000CEE
:10EA900010F0070491F820F040F049804FF0000496
:10EAA0006FF00700D1E9002391F840F000F1080071
:10EAB00082FA4CF2A4FA8CF283FA4CF3A2FA8CF3A9
:10EAC0004BBBD1E9022382FA4CF200F10800A4FA10
:10EAD0008CF283FA4CF3A2FA8CF3E3B9D1E9042364
:10EAE00082FA4CF200F10800A4FA8CF283FA4CF39B
:10EAF000A2FA8CF37BB9D1E9062301F1200182FA55
:10EB00004CF200F10800A4FA8CF283FA4CF3A2FA5A
:10EB10008CF3002BC6D0002A04BF04301A4612BA68
:10EB2000B2FA82F2FDE8024500EBD2007047D1E96B
:10EB3000002304F00305C4F100004FEAC50514F0FA
:10EB4000040F91F840F00CFA05F562EA05021CBFCB
:10EB500063EA050362464FF00004A9E7002A41D0AA
:10EB600040EA010313F00303F0B425D1032A23D9AB
:10EB700004680D68AC421FD1043A35D0A4F10135C8
:10EB800025EA040414F0803F31D1071D0D1D0DE06E
:10EB900057F8043B0E68A3F10134B34224EA03049E
:10EBA0000AD1043A20D014F0803F23D1032A294609
:10EBB000384605F10405EBD803780C789C4202F145
:10EBC000FF320CD182B114B916E06AB17BB110F8F2
:10EBD000013F11F8014FA34202F1FF32F5D0181B9B
:10EBE000F0BC7047104670471046F0BC704718469E
:10EBF000F0BC70470020F3E72046F1E740EA01034C
:10EC00009B0770B42BD1032A29D90C460346214611
:10EC100054F8046BA6F1013525EA060515F0803F8E
:10EC200006D1043A032A43F8046B2146EFD8A2B177
:10EC30000C781C70013A013301313CB16AB111F812
:10EC4000014B03F8014B013A002CF7D12AB11A44C9
:10EC5000002103F8011B9A42FBD170BC70470346A8
:10EC6000E5E700BF2DE9F047254C2568D5F8484178
:10EC70000646884692469946C4B360681F2817DC4A
:10EC8000431C76B104EB80050122C5F888A0D4F8B6
:10EC9000881182401143022EC4F88811C5F80891EA
:10ECA0001ED00230636044F820800020BDE8F08769
:10ECB000144B03B34FF4C870FFF74EF90446D0B1BC
:10ECC000D5F84831002780E88800C5F84841384623
:10ECD0000123C4F88871C4F88C71002EE1D0D1E70B
:10ECE000D4F88C110A43C4F88C21DAE705F5A67430
:10ECF000C5F84841C1E74FF0FF30BDE8F08700BFDD
:10ED0000080E010059DF0000024B13B1024800F069
:10ED100005B870470000000029ED000000230146FF
:10ED20001A461846FFF79EBF38B5074D074C2C1BF7
:10ED3000A41005D0013C55F8043D9847002CF9D1AA
:10ED4000BDE8384002F072B800000000000000008A
:10ED5000F8B5234F0C460646FFF778FCBB685D68A4
:10ED600025F00305291B01F6EF7121F47F6121F0E5
:10ED70000F01A1F58054B4F5805F07DB0021304618
:10ED8000FFF760FEBB682B44984204D03046FFF783
:10ED90005FFC0020F8BD61423046FFF753FE0130B2
:10EDA0000DD0104BBA6819682D1B45F0010530468F
:10EDB000091B55601960FFF74BFC0120F8BD0021CD
:10EDC0003046FFF73FFEBA68831A0F2BDEDD064C94
:10EDD0000449246843F00103001B53600860D5E731
:10EDE0000C97FF1FA8A1FF1F189BFF1F002945D0EC
:10EDF0002DE9F0410D468046FFF728FC55F8047CCC
:10EE00006A4927F00103A5F10804E2188E685068EA
:10EE1000B24220F0030062D0FE0750600BD455F8D8
:10EE2000087CE41B01F1080EA56875453B446FD0D2
:10EE3000E768EF60BD6015186D68ED0742D543F0D7
:10EE400001026260E350B3F5007F18D2DB085A1C60
:10EE50004D6851F83270A76001209B1000FA03F34F
:10EE600001EBC2001D430838E0604D6041F83240BC
:10EE7000FC604046BDE8F041FFF7EABB70475A0A24
:10EE8000042A53D89A0902F139077F0002F13805A4
:10EE900001EB870051F827204449083890424DD0B3
:10EEA000516821F003018B4202D292689042F7D15F
:10EEB000D068E060A2608460D4604046BDE8F04164
:10EEC000FFF7C6BB95683A4FBD4203443FD0D068B8
:10EED000E86043F0010285606260E350B3E7FF073A
:10EEE000034407D455F8082CA41A1344A068E26818
:10EEF000C26090602F4A126843F001009342606044
:10EF00008C60B6D32C4B40461968FFF721FFB0E761
:10EF100011184968C90744D49168D268CA6003448B
:10EF200043F0010091606060E350A2E7142A17D813
:10EF300002F15C077F0002F15B05A9E7AA104B68AC
:10EF4000012505FA02F213434B600246B1E743F094
:10EF500001024C610C61E560A5606260E35088E7E6
:10EF6000542A06D81A0B02F16F077F0002F16E05D2
:10EF70008EE7B2F5AA7F06D8DA0B02F178077F0098
:10EF800002F1770584E740F25450824206D89A0C89
:10EF900002F17D077F0002F17C0579E7FE277E25DF
:10EFA00076E743F001026260E35062E70C97FF1FCF
:10EFB0001497FF1F149BFF1FA4A1FF1FF2FFFFFF69
:10EFC000F3FFFFFFF4FFFFFFF4FFFFFFF5FFFFFF7D
:10EFD000F6FFFFFFF7FFFFFFF8FFFFFFF9FFFFFF5F
:10EFE000FAFFFFFFFBFFFFFFFCFFFFFFFDFFFFFF3F
:10EFF000FDFFFFFFFEFFFFFFFFFFFFFF0000000020
:10F00000000078053408540B800C3C0F5C12E015AE
:10F01000FA19141E6022AC265C2B0C30BC34023A68
:10F02000FF3FFFFF90F300006CF3000048F3000087
:10F0300024F300000CF1000058F000007CF0000008
:10F04000A0F00000C4F0000010F2000034F2000054
:10F0500000F00000ECF100000000580246056608D0
:10F06000540BD80E5C12E015FA19141E6022AC265F
:10F070005C2B0C30BC34023AFF3FFFFF00009001D4
:10F0800020031405D0075A0AAC0DCC10B4146A182A
:10F09000E81C342180252A2B70301437FF3FFFFFF6
:10F0A0000000C800F4018403140508072E091C0C95
:10F0B000D80EF811AE159619401F1C25F22B5834A6
:10F0C000FF3FFFFF00006400C8009001BC021A046B
:10F0D000DC059E07F609800CA00F2413A2174C1D17
:10F0E0005424442FFF3FFFFF40067805B004E80397
:10F0F00084032003BC025802F40190012C01FA00A1
:10F10000C8009600640032001900FFFF0000FF03F2
:10F11000FF07FF0BFF0FFF13FF17FF1BFF1FFF234F
:10F12000FF27FF2BFF2FFF33FF37FF3BFF3FFFFF83
:10F1300001020101020101010201010102010100BC
:10F1400001010102000101020101010101010200AE
:10F15000010102010102010101020100010201019C
:10F16000020101010000000102010102010101018F
:10F17000000001020101020101000202020102017C
:10F180000102010002020202010201010200010269
:10F190000202020102010100000002020202010259
:10F1A000010101000002020202010201000202024A
:10F1B0000202020201020002020102020202020134
:10F1C0000100020202020202020201000002020029
:10F1D0000202020202000201020202020202020212
:10F1E0000002000202020202020202FF0000D00737
:10F1F000800CD80E0010C012EC130C17FA19141E54
:10F200006022AC265C2B0C30BC34023AFF3FFFFF7F
:10F210000000580246056608540BD80E5C127017A1
:10F22000FC21F82A70305834DC37663A8C3C803E3A
:10F23000FF3FFFFF0000580246056608540BA00F71
:10F24000D4172823F82A442F643284354038663A8C
:10F250008C3C803EFF3FFFFF2C011301FA00E100D0
:10F26000C800AF0096007D0064004B00320019001A
:10F2700000000000CDCC4C3DCDCCCC3D9A99193E40
:10F28000CDCC4C3E0000803E9A99993E3333B33E3C
:10F29000CDCCCC3E6666E63E0000000007000000D4
:10F2A0000C00000010000000130000001600000019
:10F2B0001800000000000000070000000C00000023
:10F2C00013000000180000001F00000024000000D0
:10F2D000000000000C0000001800000024000000E6
:10F2E000300000003C00000048000000000000006A
:10F2F000FBFFFFFFF4FFFFFFEFFFFFFFE8FFFFFF54
:10F30000E3FFFFFFDCFFFFFF00000000F4FFFFFF53
:10F31000E8FFFFFFDCFFFFFFD0FFFFFFC4FFFFFFA1
:10F32000B8FFFFFF00007805220B0410B414321957
:10F33000B01DFC214826FE29822D3831263446375F
:10F34000663A223DFF3FFFFF0000D007100E8813F2
:10F350003219AA1E282374275C2B442F643284356B
:10F360004038663A8C3C803EFF3FFFFF0000540B64
:10F37000EC13FA1908201C253629EC2C0C302C3300
:10F38000E8357238663AF63B863D163FFF3FFFFF91
:10F390000000CC10581BFC21AC26C62A7C2E38312C
:10F3A000F4334C36A438983A5A3C543D803E7A3F68
:10F3B000FF3FFFFF24F40000FA9BFF1F0000FF0F38
:10F3C000A09DFF1F0000FF0F4D3B0000F0F3000069
:10F3D0009C9DFF1F32005E01000000000000000045
:10F3E000ED3A000054485200534E53004D4158002E
:10F3F000544F5543482053454E53450045585452A9
:10F400004120434F4E54524F4C4C45520000000097
:10F4100050495443482042454E4400004249544517
:10F420000000000042524541544800FFFCF3000038
:10F43000F49CFF1FF401A00FEE9CFF1FF401A00F2E
:10F44000F93A00001CF40000B29BFF1FBC025C12E2
:10F45000749DFF1FBC025C12313B000010F40000E1
:10F46000469DFF1FF401A00F809BFF1FF401A00F1A
:10F47000153B000054FC00005CFC000048FC000050
:10F480004CFC000050FC0000ECFA00000CFC0000FA
:10F4900028FC00002CFC000030FC000034FC0000C4
:10F4A00038FC00003CFC000040FC000014FC0000A4
:10F4B00044FC0000ECFA0000E8FA00001CFC00002C
:10F4C00020FC000024FC0000ECFA00000CFC000012
:10F4D00010FC000014FC000018FC0000F8FB000009
:10F4E000FCFB000000FC000004FC000008FC000025
:10F4F000E8FB0000ECFB0000F0FB0000F80001005E
:10F50000F4FB000064FC000068FC00006CFC0000E0
:10F5100070FC000074FC000078FC00007CFC000023
:10F5200080FC000084FC000088FC00008CFC0000D3
:10F5300090FC000094FC00000100000098FC00001A
:10F5400007000000000000000100000099480000D2
:10F5500010FE00000000050108000000AC8DFF1F38
:10F56000C94700000600000009000000308FFF1F9F
:10F570000000000000FF0000F4FE0000589DFF1F87
:10F580000000300000000000A9550000D546000032
:10F59000000000009CFD00000000010108000000C8
:10F5A000C88EFF1FFCFC0000000002010C000000E0
:10F5B000788FFF1F00000000D0FE0000DCFE00007E
:10F5C000949BFF1F0000010001000000994B000008
:10F5D00009450000000000000100000018FE0000C6
:10F5E0000600000098FC0000000004050800000070
:10F5F000C48BFF1F0100000010FE00000900000086
:10F60000000000000100000069610000010000002E
:10F6100038FE0000030000000000000018FF00009A
:10F62000F4FE0000549DFF1F0000300000000000A9
:10F63000A9550000D54600000000000000000000B1
:10F64000010000003D5200000000000040FE0000EC
:10F6500048FE0000FC9CFF1F010010000600000097
:10F66000955D000029450000A14F0000000000004A
:10F67000E8FE0000F4FE00005A9DFF1F000030006D
:10F6800000000000A9550000D54600000000000061
:10F69000000000000000000000000000000000006A
:10F6A000000000000000000000000000000000005A
:10F6B000000000000000000000000000000000004A
:10F6C000000000000000000000000000000000003A
:10F6D000000000000000000000000000000000002A
:10F6E000000000000000000000000000000000001A
:10F6F000000000000000000000000000000000000A
:10F7000000000000000000000000000000000000F9
:10F7100000000000000000000000000000000000E9
:10F7200000000000000000000000000000000000D9
:10F7300000000000000000000000000000000000C9
:10F7400000000000000000000000000000000000B9
:10F7500000000000000000000000000000000000A9
:10F760000000000000000000000000000000000099
:10F770000000000000000000000000000000000089
:10F780000000000000000000000000000000000079
:10F790000000000000000000000000000000000069
:10F7A0000000000000000000000000000000000059
:10F7B00000000000007FFFFF000003F9FFFFFC00D6
:10F7C00000000000007FFFFF800007F9FFFFFE0040
:10F7D0000000000000600001C0000E19800007005A
:10F7E00000000000006FFFFCC0001DD9BFFFF30048
:10F7F00000000000006FFFFEC0003BD9BFFFFB0010
:10F8000000000000006C0006C00077D9B0001B00AB
:10F8100000000000006C0006C000EED9B0001B0024
:10F8200000000000006C0006C001DCD9B0001B0025
:10F8300000000800006C0006C003B8D9B0001B002F
:10F8400000001800006FFFFEC0077FD9B0001B004A
:10F8500000001800006FFFFCC00EFFD9B0001B00B5
:10F8600000C0180000600001C01C0019B0001B009F
:10F8700000C03800006FFBFF803BFFD9B0001B00C9
:10F8800000C03000006FFDFF0077FFD9B0001B0003
:10F8900001E03000006C0EE000EE00D9B0001B006B
:10F8A00001E03000006C077001DC00D9B0001B00E3
:10F8B00001B03000006C03B803B800D9B0001B00E1
:10F8C00001B03000006C01DC077000D9B0001B00F3
:10F8D000019820C0406C00EE0EE000D9B0001B0083
:10F8E000030C20C0C06C00771DC000D9BFFFFB0017
:10F8F000030C20C0C06C003BBB8000D9BFFFF300ED
:10F90000030620C1C06C001DF70000D9800007006D
:10F9100003032083806C000EEE0000D9FFFFFE0081
:10F920000303B183806C00075C0000D9FFFFFC007B
:10F930000301F187800000000000000000000000CB
:10F940000300F18D800000000000000000000000B6
:10F95000030071B9800000000000000000000000FA
:10F96000030031F1800000000000000000000000F2
:10F97000030000C180000000000000000000000043
:10F980000300000000000000000000000000000074
:10F990000300000000000000000000000000000064
:10F9A0000200000000000000000000000000000055
:10F9B0000000000000000000000000000000000047
:10F9C0000000000000000000000000000000000037
:10F9D0000000000000000000000000000000000027
:10F9E0000000000000000000000000000000000017
:10F9F0000000000000000000000000000000000007
:10FA000000000000000000000000000000000000F6
:10FA100000000000000000000000000000000000E6
:10FA200000000000000000000000000000000000D6
:10FA300000000000000000000000000000000000C6
:10FA400000000000000000000000000000000000B6
:10FA500000000000000000000000000000000000A6
:10FA60000000000000000000000000000000000096
:10FA70000000000000000000000000000000000086
:10FA80000000000000000000000000000000000076
:10FA9000C0FE00000000030106000000948DFF1F5F
:10FAA0000000000024FF0000F4FE0000789BFF1F10
:10FAB00000003000000000009955000019450000CA
:10FAC0000000000000000000F4FC0000C0FC00008A
:10FAD000689BFF1F0000090000000000BD4B0000F4
:10FAE00049450000000000004F4E00004F46460010
:10FAF00055534200424154004C4F57200000000033
:10FB00004D454E5520202020202020202058585898
:10FB100020592E595600000058000000524F540042
:10FB20004D454C0044594E006D730000425448004E
:10FB3000424954004C5652004E524D005245560018
:10FB4000312F0000415400004D4F4400504244000A
:10FB500045434200454353004C564C004C56500020
:10FB6000474C440045434800762E0000312E342E89
:10FB70003600000053455400434C52004E7552412C
:10FB8000440000006669726D7761726520762E0010
:10FB900055534220706F776572000000416C6B61B5
:10FBA0006C696E6520626174746572790000000092
:10FBB00030202520617420004E694D482062617418
:10FBC00074657279000000004C69506F20626174A6
:10FBD0007465727900000000444F4E275400000005
:10FBE00050414E49430000004557490045575800D1
:10FBF0005341580045565200484D53003554480073
:10FC00004F43540035444E004F444E004D570000C2
:10FC10004650000043460000535000005357000078
:10FC200053454C005345450042520000564C0000DD
:10FC3000455800004D572B0042522B00564C2B00CC
:10FC400045582B00554E4F00414C4B004E4D48003F
:10FC50004C49500042525448000000005054434860
:10FC6000000000002D3400002D3300002D32000074
:10FC70002D3100004C494E002B3100002B3200008A
:10FC80002B3300002B3400005331000053320000AE
:10FC90005A3100005A3200005649425241544F0036
:10FCA000444952454354494F4E000000434F4E547F
:10FCB000524F4C00535155454C43482042000000E0
:10FCC0004C4556454C00000053454E534520425488
:10FCD00045000000535155454C4348204C0000005E
:10FCE00053454E5345204C56520000005245545542
:10FCF000524E0000444550544800000053455455AE
:10FD000050204354524C5300455854524120504BBC
:10FD10004559000046494E474552494E47000000AC
:10FD20004C4556454C204343000000004D4F4420B5
:10FD30004B4559004445474C495443480000000096
:10FD40004841524D2053454C000000005345524954
:10FD50004553000045584354204841524D0000008F
:10FD60004841524D2052414E4745000045584354AA
:10FD70002043432042000000455843542043432081
:10FD800041000000504954434842454E44000000A1
:10FD9000504F52542F474C440000000053455455D7
:10FDA00050204252454154480000000056454C2026
:10FDB000424F4F535400000056454C2044454C419F
:10FDC00059000000435552564500000056454C4F1F
:10FDD00043495459000000004252454154482041D3
:10FDE0005400000043432042205249534500000084
:10FDF000425254482043432042000000425254489B
:10FE0000204343204100000041424F555400000070
:10FE10004558545241530000524F5441544F5200E0
:10FE200053455455502043544C00000053455455FD
:10FE3000502042520000000041444A5553540000F3
:10FE40004D494449204348004D4944492043484EC8
:10FE50004C0000004241542054595045000000001D
:10FE6000574C204348414E00574C20504F57455265
:10FE7000000000004641535420424F4F5400000000
:10FE8000444143204F55540053504543204B45595E
:10FE9000000000004C4547414359204252000000F9
:10FEA0004C45474143592050420000004F435441C4
:10FEB000564500005452414E53504F5345000000E8
:10FEC000524F5441544F5220534554555000000056
:10FED0005052494F52495459000000004D4F4E4F67
:10FEE000205052494F000000524F54415445203495
:10FEF0000000000053454D49544F4E45530000004B
:10FF0000524F54415445203300000000524F544199
:10FF10005445203200000000524F544154452031D6
:10FF200000000000504152414C4C454C00FFFFFF87
:10FF3000010000002CFE0000040000002C01000065
:10FF4000000000000CFF0000F4FE0000569DFF1FA3
:10FF50000000300000000000A9550000D546000058
:10FF6000000000000100000020FE0000050000006D
:10FF700000000000C4FD0000C4FD00006C9BFF1FDA
:10FF800000000C0003000000B55C000039450000D3
:10FF9000000000000100000008FE00000800000052
:10FFA0000021110202000000002111020504FFFFE0
:10FFB000003E7FFF4E75455649633031000000001A
:10FFC0007676764E75455649636363007676764E4F
:10FFD00075455649633034656576767676767676FD
:10FFE00076000000496E76616C696420636F6E660E
:10FFF000696720666F726D6174000000496E7661FA
:020000021000EC
:100000006C696420636865636B73756D0000000044
:10001000496E76616C696420636F6E6669672073F0
:10002000697A6500496E76616C696420636F6E66FB
:1000300069672076657273696F6E00004E7545566C
:1000400049000000496E76616C6964206D657373C8
:100050006167652E000000006530300063303000BD
:1000600053656E64696E6720636F6E6669672E2ED6
:100070002E000000436F6E6669672073656E742EF4
:10008000000000006330330053656E64696E6720C2
:1000900076657273696F6E2E000000006330320067
:1000A000526563656976696E6720636F6E6669671E
:1000B0002E2E2E004E657720636F6E666967207363
:1000C000617665642E000000556E6B6E6F776E2052
:1000D0006D6573736167652E000000006530310047
:1000E000436F6E666967206D676D7400506F77654A
:1000F00072206F6666204E7545564900746F206504
:100100007869740052656164792E00FF3480044080
:10011000400000001211FFFFFF0202000000131058
:10012000FFFFFF02020000001800000034800440BE
:10013000800000001EFFFFFFFF02000000001DFF07
:10014000FFFFFF0200000000190000000000000097
:1001500000000000517D0000157D0000C97C0000FA
:10016000117D0000CD7C0000D97C0000F97C0000EE
:10017000000103070F1F3F7F2200FF2100FFFFFF49
:100180000080C0E0F0F8FCFE00000000000000006D
:100190006D9C000065C60000C97C0000D58600008B
:1001A0006D87000039950000ED9400002195000056
:1001B000F99400000D9500000994000039950000A5
:1001C0006195000059890000999100003591000067
:1001D000319600003D95000095960000359700008F
:1001E00000006000000000000000000000000000AF
:1001F00000E000000000000000000000000000011E
:10020000E00000000000000000000000000001F01D
:100210000000000000000000000000000003F000EB
:1002200000000000000000000000000007F00000D7
:10023000000000000000000000000007F8000000BF
:10024000000000000000000000000FF800000003A4
:10025000C0007E000001E0007F0FF800000003C036
:1002600000FE000001E000FFEFF800000003C00006
:10027000FE000001E000FFFFF800000003C000F0F6
:100280000000000F007FFE7FC0000003C000F000F0
:1002900000000F003FFE7FF83FF1FBCFFCFEF3BCF8
:1002A0003DEFE01FFE7FFF7FFBFFDFFEFEFFBC3D5B
:1002B000EFE01FC6FFFF7FFBFFDFFEFEFFBC3DEF51
:1002C000E00FE3C7FE787BC3DE1EF0FFBC3DEF000E
:1002D00007FF87FC787BC3DE1EF0F83C3DEF000192
:1002E000FFFFF0007BC3C01EF0F03C3DEF0001F3C8
:1002F0007FE03FFBC3CFFEF0F03C3DEF0003E33F68
:10030000807FFBC3DFFEF0F03C3DEF0007E73C00E1
:10031000787BC3DE1EF0F03C3DEF0007FFBE0078A7
:100320007BC3DE1EF0F03C3DEF0007FFFE00787B54
:10033000C3DE1EF0F03C3DEF000FFFFE007FFBFF31
:10034000DFFEF0F03FFDEFE00FFFFF007FFBFFDF80
:10035000FEF0F03FFDEFE00FF9FF003E79F9CF9E90
:10036000F0F01F3DE7E01FF1FF000000000000007B
:1003700000000000001F80FF007FFFFFFFFFFFFF66
:10038000FFFFFFE01C007F007FFFFFFFFEB46D88D2
:100390008D18E000001F007FFFFFFFFE95AD7DB5CB
:1003A00077E000000F007FFFFFFFFEA5AD9D8D19D8
:1003B000E0000006007FFFFFFFFEB5ADEDB57EE07B
:1003C000AED580A8D300408D2000A1C8DB40A4A6F4
:1003D0002EAFFFFF000000000001800000000000C1
:1003E0000000000003800000000000000000000783
:1003F000C000000000000000000007C00000000076
:1004000000000000000FC00000000000000000001D
:100410001FE00000000000000000001FE0000000DE
:100420000000000000003FE00000000000000000AD
:10043000003FF00000000000000000007FF000001E
:1004400000000000001FF87FF00000000000000026
:100450003FFE7FF0000000000000003FFF7FF00043
:100460000000000000001FFFFBE000000000000093
:10047000000FFFF9FFC00000000000000FFFF9FFB0
:10048000F800000000000007FFF1FFFF000000007F
:10049000000003FC73FFFF80000000000001FE3F2E
:1004A000FFFF80000000000000FF1E0FFF000000A3
:1004B000000000007FFE1FFC000000000000003F65
:1004C000FFFFF8000000000000000FDFFFE0000069
:1004D00000000000001F19FFC00000000000000025
:1004E0003F3CFF00000000000000007E7CF80000A0
:1004F0000000000000007FFE7C0000000000000003
:1005000000FFFFFC0000000000000000FFFFFE00F5
:1005100000000000000000FFFFFE000000000000DF
:100520000001FFEFFE0000000000000001FFCFFE11
:100530000000000000000003FF07FE0000000000B4
:10054000000003FC07FE0000000000000003F003B1
:10055000FE00000000000000018000FE000000001E
:100560000000000000007E0000000000000000000D
:10057000003E000000000000000000000C00000031
:10058000000000078000FC000003C000000007809E
:1005900001FC000003C0000000078001FC00000314
:1005A000C0000000078001E00000001E00000007FE
:1005B0008001E00000001E007FE3F79FF9FDE7786F
:1005C0007BDFC0FFF7FFBFFDFDFF787BDFC0FFF7DC
:1005D000FFBFFDFDFF787BDFC0F0F787BC3DE1FF8B
:1005E000787BDE00F0F787BC3DE1F0787BDE000031
:1005F000F787803DE1E0787BDE007FF7879FFDE1B4
:10060000E0787BDE00FFF787BFFDE1E0787BDE006E
:10061000F0F787BC3DE1E0787BDE00F0F787BC3D7A
:10062000E1E0787BDE00F0F787BC3DE1E0787BDE3F
:1006300000FFF7FFBFFDE1E07FFBDFC0FFF7FFBF7B
:10064000FDE1E07FFBDFC07CF3F39F3DE1E03E7B1B
:10065000CFC00000000000000000000000FFFFFF0E
:10066000FFFFFFFFFFFFFFC0FFFFFFFFFD68DB1184
:100670001A31C0FFFFFFFFFD2B5AFB6AEFC0FFFFDF
:10068000FFFFFD4B5B3B1A33C0FFFFFFFFFD6B5BC2
:10069000DB6AFDC000000000000000006D9C00004F
:1006A00065C60000C97C0000D586000051A400008A
:1006B00039950000ED94000021950000F9940000A8
:1006C0000D95000009940000399500006195000027
:1006D0005D95000085950000DD95000031960000D5
:1006E0003D95000095960000359700000000000041
:1006F000003E5B4F5B3E3E6B4F6B3E1C3E7C3E1CA8
:10070000183C7E3C181C577D571C1C5E7F5E1C00ED
:10071000183C1800FFE7C3E7FF0018241800FFE7A4
:10072000DBE7FF30483A060E2629792926407F0567
:100730000507407F05253F5A3CE73C5A7F3E1C1C7D
:1007400008081C1C3E7F14227F22145F5F005F5F3D
:1007500006097F017F006689956A60606060609429
:10076000A2FFA29408047E040810207E201008082E
:100770002A1C08081C2A08081E101010100C1E0C39
:100780001E0C30383E3830060E3E0E0600000000CB
:100790000000005F00000007000700147F147F14B2
:1007A000242A7F2A122313086462364956205000F7
:1007B00008070300001C2241000041221C002A1CE3
:1007C0007F1C2A08083E08080080703000080808CE
:1007D0000808000060600020100804023E514945EE
:1007E0003E00427F400072494949462141494D330C
:1007F0001814127F1027454545393C4A4949314173
:10080000211109073649494936464949291E000040
:100810001400000040340000000814224114141495
:100820001414004122140802015909063E415D5981
:100830004E7C1211127C7F494949363E414141228A
:100840007F4141413E7F494949417F090909013EB4
:10085000414151737F0808087F00417F41002040DB
:10086000413F017F081422417F404040407F021CED
:10087000027F7F0408107F3E4141413E7F09090904
:10088000063E4151215E7F091929462649494932D0
:1008900003017F01033F4040403F1F2040201F3F96
:1008A0004038403F6314081463030478040361591B
:1008B000494D43007F41414102040810200041415D
:1008C000417F040201020440404040400003070809
:1008D0000020545478407F28444438384444442805
:1008E000384444287F385454541800087E090218AC
:1008F000A4A49C787F0804047800447D4000204034
:10090000403D007F1028440000417F40007C047877
:1009100004787C080404783844444438FC182424BF
:100920001818242418FC7C0804040848545454243F
:1009300004043F44243C4040207C1C2040201C3CBC
:100940004030403C44281028444C9090907C4464B3
:10095000544C440008364100000077000000413646
:10096000080002010204023C2623263C1EA1A161CC
:10097000123A4040207A38545455592155557941FE
:100980002254547842215554784020545579400CD3
:100990001E527212395555555939545454593955B6
:1009A0005454580000457C410002457D42000145F9
:1009B0007C407D1211127DF0282528F07C5455458D
:1009C000002054547C547C0A097F493249494932F9
:1009D0003A4444443A324A4848303A4141217A3A0A
:1009E00042402078009DA0A07D3D4242423D3D40D6
:1009F00040403D3C24FF2424487E4943662B2FFC85
:100A00002F2BFF0929F620C0887E09032054547932
:100A1000410000447D413048484A32384040227A03
:100A2000007A0A0A727D0D19317D2629292F282680
:100A30002929292630484D40203808080808080888
:100A40000808382F10C8ACBA2F102834FA00007BE1
:100A5000000008142A142222142A140855005500F4
:100A600055AA55AA55AAFF55FF55FF000000FF00E3
:100A7000101010FF00141414FF001010FF00FF10DE
:100A800010F010F0141414FC001414F700FF000010
:100A9000FF00FF1414F404FC141417101F10101F8F
:100AA000101F1414141F00101010F0000000001F7D
:100AB000101010101F10101010F010000000FF1088
:100AC0001010101010101010FF10000000FF140084
:100AD00000FF00FF00001F10170000FC04F41414B6
:100AE0001710171414F404F40000FF00F714141482
:100AF00014141414F700F7141414171410101F1002
:100B00001F141414F4141010F010F000001F101F24
:100B10000000001F14000000FC140000F010F01092
:100B200010FF10FF141414FF141010101F00000009
:100B300000F010FFFFFFFFFFF0F0F0F0F0FFFFFF0D
:100B40000000000000FFFF0F0F0F0F0F3844443864
:100B500044FC4A4A4A347E02020606027E027E02B3
:100B600063554941633844443C04407E201E2006BE
:100B7000027E020299A5E7A5991C2A492A1C4C72FB
:100B800001724C304A4D4D303048784830BC625A82
:100B9000463D3E494949007E0101017E2A2A2A2A12
:100BA0002A44445F444440514A444040444A5140EE
:100BB0000000FF0103E080FF000008086B6B0836AF
:100BC00012362436060F090F060000181800000020
:100BD0001010003040FF0101001F01011E00191D0F
:100BE0001712003C3C3C3C0000000000050E0809C8
:100BF0000D0C06070F0400130393050E08090D0CD6
:100C000006070F04FFFFC585848687C4FFFF001316
:100C100003931A9217FFFFFF6FF07F0303700378AF
:100C200013F0800FFBD070474008FE4340A0044003
:100C30004408FE4344A004400018FE4300C00440A2
:100C40003000FE43309004403400FE4334900440B2
:100C50001C18FE431CC004401018FE4310C0044082
:100C60000818FE4308C004400C18FE430CC00440A2
:100C70000C10FE430CB004401010FE4310B00440B2
:100C80001810FE4318B004401C10FE431CB0044072
:100C90001410FE4314B004400418FE4304C0044082
:100CA0000010FE4300B004400008FE4300A00440D2
:100CB0000408FE4304A004400C08FE430CA00440BA
:100CC0000808FE4308A004401418FE4314C0044062
:100CD0001818FE4318C004400410FE4304B004403A
:100CE0000810FE4308B004401400FE431490044072
:100CF0004C08FE434CA004400420FE4304D00440B2
:100D00002410FE4324B004402010FE4320B00440D1
:100D10002810FE4328B004402C10FE432CB00440A1
:100D20000020FE4300D004404808FE4348A0044091
:100D30001000FE4310900440090AFFFFFFFFFFFF71
:100D4000FFFFFFFFFFFFFF0D00060807FFFF0E0F6D
:100D5000FF0CFFFFFFFFFFFF0B05FFFF0D0AFFFF6B
:100D60001519151900010000FC91FF1F1200000069
:100D7000000200002892FF1F730000000022010003
:100D80009C92FF1F21000000002101008492FF1FA0
:100D90000900000000030000C092FF1F00000000D7
:100DA000010309041092FF1F000000000203090460
:100DB0002089FF1F0000000003030904C492FF1FE5
:100DC0000000000000000000000000000000000023
:100DD00065787000FFFFFFFF000000000000E03FAB
:100DE000000000000000E0BF763C7935EF39EA3DB5
:100DF000763C7935EF39EABD0000E0FE422EE63F51
:100E00000000E0FE422EE6BFE092FF1FF8B500BFF3
:100E1000F8BC08BC9E46704709ED00003504000090
:0C0E2000913A0000515600005579000086
:040E2C00F8B500BF56
:100E300038B5084B1C681C6054B1074D94FAA4F3F4
:100E4000B3FA83F355F823309847631E1C40F5D15D
:100E500038BD00BFA0D00440DC91FF1F38B5084B5F
:100E60001C681C6054B1074D94FAA4F3B3FA83F3E1
:100E700055F823309847631E1C40F5D138BD00BF9C
:100E8000A0C00440BC91FF1F38B5084B1C681C6013
:100E900054B1074D94FAA4F3B3FA83F355F8233011
:100EA0009847631E1C40F5D138BD00BFA0B0044078
:100EB0008C91FF1F38B5084B1C681C6054B1074D5E
:100EC00094FAA4F3B3FA83F355F823309847631EDA
:100ED0001C40F5D138BD00BFA0A004403C91FF1FCD
:100EE00038B5084B1C681C6054B1074D94FAA4F344
:100EF000B3FA83F355F823309847631E1C40F5D1AD
:100F000038BD00BFA09004400491FF1F0000000006
:100F100016034E00750045005600490020004D00A4
:100F20004900440049000000002000000000F0419A
:100F3000280000000C0000005A000000F3FFFFFF33
:100F4000DFFFFFFFA3FFFFFFAEFFFFFF7300000007
:100F5000760000000200000004000000D8FFFFFF40
:100F6000B5FFFFFFA2FFFFFF02000000FBFFFFFF36
:100F70000000000000000000000000000000000071
:100F80000000000000000000000000000000000061
:100F90000100000000200000002000000010000000
:100FA000AB0A0000000800006606000055050000BE
:100FB00092040000000400008E03000033030000D0
:100FC000E8020000AB020000002000001405000051
:100FD000000102070B0102070B4A140002000C007B
:100FE00024000000A8FFFFFFBCFFFFFFE1FFFFFFA1
:100FF0000D000000040000007800000079000000EF
:10100000BCFFFFFFABFFFFFFDEFFFFFF170000008D
:1010100057000000100000000A0000000800000057
:101020001500000018000000290000000200FFFF6A
:10103000FFFF0000B4F3000044F400005CF4000083
:101040002CF40000CCF300000000000008FD0000BC
:1010500008FD0000C89DFF1F0000190000000000EF
:101060000000000000000000000000000000000080
:10107000A0FC0000A0FC0000E09BFF1F000001009E
:10108000010000000000000000000000000000005F
:1010900000000000ACFC0000ACFC0000EA9CFF1F5C
:1010A000000002000100000000000000000000003D
:1010B0000000000000000000D4FC0000C0FC0000A4
:1010C000EE89FF1F01001E0000000000000000006C
:1010D000000000000000000001000000000000000F
:1010E00014FD000014FD0000449BFF1F00000400DD
:1010F00001000000000000000000000000000000EF
:101100000000000090FD000090FD0000FE9BFF1F0E
:1011100000000400010000000000000000000000CA
:10112000000000000000000040FD00004CFD000039
:101130006C9DFF1F00000400010000000000000083
:1011400000000000000000000000000020FD000082
:1011500020FD0000CC9BFF1F00007F00010000006D
:10116000000000000000000000000000000000007F
:10117000C8FC0000C0FC00003C8AFF1F01001100F9
:10118000000000000000000000000000000000005F
:1011900000000000D8FD0000D8FD0000F29BFF1FFA
:1011A000000001000100000000000000000000003D
:1011B00000000000A08AFF1FC4FA0000A88FFF1FD4
:1011C0007C8AFF1F088CFF1FC48AFF1F7C8BFF1FB8
:1011D000A48EFF1F00000000FCFD0000FCFD0000CD
:1011E000389DFF1F00000A00010000000000000001
:1011F000000000000000000000000000E0FC000013
:10120000C0FC0000EC89FF1F01000C000000000082
:1012100000000000000000000000000000000000CE
:1012200094FE000094FE0000EE9BFF1F00000100F2
:1012300001000000000000000000000000000000AD
:1012400000000000B8FD0000B8FD0000EC9BFF1F8F
:1012500000001E000100000000000000000000006F
:101260000000000000000000E4FD0000E4FD0000BC
:10127000549BFF1F01000A00010000000000000055
:1012800000000000000000000000000074FE0000EC
:1012900074FE0000429DFF1F0000010000000000DE
:1012A000000000000000000000000000000000003E
:1012B00084FD000084FD00009E9BFF1F00000C00C9
:1012C000000000000000000000000000000000001E
:1012D0000000000088FE000088FE00004E9DFF1FF9
:1012E00000000100010000000000000000000000FC
:1012F000000000000000000060FE000060FE000032
:10130000FC8FFF1F040050000000000000000000E0
:1013100000000000000000000000000068FE000067
:1013200068FE0000509EFF1F000003000000000048
:1013300000000000000000000000000000000000AD
:10134000B4FE0000B4FE0000589BFF1F0000180010
:10135000000000000000000000000000000000008D
:1013600000000000ACFD0000ACFD0000489BFF1F2A
:101370000000090001000000000000000000000063
:1013800000000000A0FA000018F6000040FF000076
:1013900070F500006CF60000B4F50000F08DFF1F42
:1013A0002C8CFF1FE08CFF1F0090FF1F5C8EFF1F27
:1013B000988CFF1F288DFF1F048DFF1F0000000069
:1013C00054FD000060FD0000A49DFF1F000006000A
:1013D000010000000000000000000000000000000C
:1013E00000000000A0FE0000A0FE0000B09BFF1F58
:1013F00000000100010000000000000000000000EB
:1014000000000000000000002CFD00002CFD00008A
:10141000769DFF1F00001E0000000000000000007D
:1014200000000000000000000000000078FD000047
:1014300078FD0000969BFF1F0000040001000000E3
:10144000000000000000000000000000000000009C
:1014500054FE000054FE0000DE9CFF1F000002004E
:10146000010000000000000000000000000000007B
:1014700000000000ACFE0000ACFE0000509DFF1F0D
:101480000000060000000000000000000000000056
:101490000000000000000000B4FC0000C0FC0000E0
:1014A0004489FF1F01001E00000000000000000032
:1014B0000000000000000000E48BFF1FE88EFF1F0B
:1014C000748CFF1FA08BFF1F548FFF1F70FF000045
:1014D000508CFF1F708DFF1F00000000F0FD00000A
:1014E000F0FD00007A9DFF1F00007F00010000005A
:1014F00000000000000000000000000000000000EC
:1015000034FD000034FD0000869DFF1F00004600F2
:1015100000000000000000000000000000000000CB
:101520004C8DFF1F808EFF1F48F600000CF6000058
:1015300030FF000064FF0000D8F50000F4F5000063
:1015400094FF000000000000CCFD0000CCFD000076
:101550005C9BFF1F00007F000100000000000000F6
:101560000000000000000000108BFF1F388EFF1FDE
:10157000D88FFF1FCC8DFF1F348BFF1F38F5000065
:101580000C8FFF1F148EFF1F588BFF1F588AFF1FE1
:10159000EC8AFF1FBC8CFF1F00000000ECFC000069
:1015A000C0FC00007889FF1F00000400000000005C
:1015B000000000000000000000000000000000002B
:1015C0000100000000000000000000006CFD0000B1
:1015D0006CFD0000889DFF1F00007F0001000000DF
:1015E00000000000000000000000000004000000F7
:1015F0000000000080FE000080FE00004C9DFF1FE8
:1016000000000100000000000000000000000000D9
:10161000000000005401010000000000E803000089
:1016200000000000006006400C0101000000000006
:1016300000000000000000000000000000000000AA
:10164000000000000000000000000000000000009A
:10165000000000000000000000000000000000008A
:10166000000000000000000000000000000000007A
:10167000000000000000000000000000000000006A
:101680005401010000000000E80300000000000019
:10169000007006402C010100000000000000000066
:1016A000000000000000000000000000000000003A
:1016B000000000000000000000000000000000002A
:1016C000000000000000000000000000000000001A
:1016D000000000000000000000000000000000000A
:1016E0000000000000000000000000000A040000EC
:1016F00008A3FF1F91A4000091A4000091A4000082
:1017000091A4000091A4000091A4000091A4000005
:1017100091A4000091A4000091A4000091A40000F5
:1017200091A4000091A4000091A4000091A40000E5
:1017300091A4000091A4000091A4000091A40000D5
:1017400091A4000091A4000091A4000091A40000C5
:1017500091A4000091A4000091A4000091A40000B5
:1017600091A4000091A4000091A4000091A40000A5
:1017700091A4000091A4000091A4000091A4000095
:1017800091A4000091A4000091A4000091A4000085
:1017900091A4000091A4000091A4000091A4000075
:1017A00091A4000091A4000091A4000091A4000065
:1017B00091A4000091A4000091A4000091A4000055
:1017C00091A4000091A4000091A4000091A4000045
:1017D00091A4000008000000FFFFFFFF39C50000D2
:1017E00039C5000039C5000039C5000012011001DB
:1017F00000000040C01685047502010203010000CC
:1018000018035400650065006E00730079006400E1
:10181000750069006E006F0009027300020100C0CC
:101820003209040000020103000007240100012521
:10183000000624020101000624020202000924031A
:10184000010301020100092403020401010100094E
:10185000050402400000000005250101010905837F
:1018600002400000000005250101030904010002F7
:101870000300000009211101000122210007058158
:1018800003400001070502032000020006C9FF090A
:1018900004A15C7508150026FF00954009758102BA
:1018A00095200976910295040976B102C0000000E6
:1018B000040309040C030000000000000000000005
:1018C0000000000000000000000001000000000017
:1018D00000000000CC95FF1F3496FF1F9C96FF1F51
:1018E00000000000000000000000000000000000F8
:1018F00000000000000000000000000000000000E8
:1019000000000000000000000000000000000000D7
:1019100000000000000000000000000000000000C7
:1019200000000000000000000000000000000000B7
:1019300000000000000000000000000000000000A7
:101940000000000000000000000000000000000097
:101950000000000000000000000000000000000087
:101960000000000000000000000000000000000077
:101970000000000000000000010000000000000066
:101980000E33CDAB34126DE6ECDE05000B0000002B
:101990000000000000000000000000000000000047
:1019A0000000000000000000000000000000000037
:1019B0000000000000000000000000000000000027
:1019C0000000000000000000000000000000000017
:101CF0000000000000000000E092FF1F0000000054
:101D0000000000000C97FF1F0C97FF1F1497FF1F88
:101D10001497FF1F1C97FF1F1C97FF1F2497FF1F7F
:101D20002497FF1F2C97FF1F2C97FF1F3497FF1F2F
:101D30003497FF1F3C97FF1F3C97FF1F4497FF1FDF
:101D40004497FF1F4C97FF1F4C97FF1F5497FF1F8F
:101D50005497FF1F5C97FF1F5C97FF1F6497FF1F3F
:101D60006497FF1F6C97FF1F6C97FF1F7497FF1FEF
:101D70007497FF1F7C97FF1F7C97FF1F8497FF1F9F
:101D80008497FF1F8C97FF1F8C97FF1F9497FF1F4F
:101D90009497FF1F9C97FF1F9C97FF1FA497FF1FFF
:101DA000A497FF1FAC97FF1FAC97FF1FB497FF1FAF
:101DB000B497FF1FBC97FF1FBC97FF1FC497FF1F5F
:101DC000C497FF1FCC97FF1FCC97FF1FD497FF1F0F
:101DD000D497FF1FDC97FF1FDC97FF1FE497FF1FBF
:101DE000E497FF1FEC97FF1FEC97FF1FF497FF1F6F
:101DF000F497FF1FFC97FF1FFC97FF1F0498FF1F1E
:101E00000498FF1F0C98FF1F0C98FF1F1498FF1FCA
:101E10001498FF1F1C98FF1F1C98FF1F2498FF1F7A
:101E20002498FF1F2C98FF1F2C98FF1F3498FF1F2A
:101E30003498FF1F3C98FF1F3C98FF1F4498FF1FDA
:101E40004498FF1F4C98FF1F4C98FF1F5498FF1F8A
:101E50005498FF1F5C98FF1F5C98FF1F6498FF1F3A
:101E60006498FF1F6C98FF1F6C98FF1F7498FF1FEA
:101E70007498FF1F7C98FF1F7C98FF1F8498FF1F9A
:101E80008498FF1F8C98FF1F8C98FF1F9498FF1F4A
:101E90009498FF1F9C98FF1F9C98FF1FA498FF1FFA
:101EA000A498FF1FAC98FF1FAC98FF1FB498FF1FAA
:101EB000B498FF1FBC98FF1FBC98FF1FC498FF1F5A
:101EC000C498FF1FCC98FF1FCC98FF1FD498FF1F0A
:101ED000D498FF1FDC98FF1FDC98FF1FE498FF1FBA
:101EE000E498FF1FEC98FF1FEC98FF1FF498FF1F6A
:101EF000F498FF1FFC98FF1FFC98FF1F0499FF1F19
:101F00000499FF1F0C99FF1F0C99FF1F1499FF1FC5
:101F10001499FF1F1C99FF1F1C99FF1F2499FF1F75
